:100000000C94080A0C94270A0C94270A0C94E20B0F
:100010000C941C0C0C94270A0C94270A0C94270AA5
:100020000C94270A0C94270A0C94270A0C94270A8C
:100030000C94270A0C94270A0C94270A0C944B0F53
:100040000C94270A0C94270A0C94270A0C94270A6C
:100050000C945D730C94106B0C94270A0C94270A73
:100060000C94270A0C94E56B0C94270A0C94D96B1A
:100070000C94270A0C94270A0C94270A0C94270A3C
:100080000C94907E0C94270A0C94270A0C94270A4F
:100090000C94236C0C94270A0C94176C0C94270A6C
:1000A0000C94270A0C94270A0C94270A0C94270A0C
:1000B0000C94270A0C94270A0C94270A0C94270AFC
:1000C0000C94270A0C94270A0C94270A0C94270AEC
:1000D0000C94270A0C94270A0C94270A0C94270ADC
:1000E0000C94270A0C9416730C9420730C940C73C4
:1000F0000C94CC720C9451730C9442730C94367320
:100100000C942A730C94270A0C94270A0C94270A3F
:100110000C94270A0C94270A0C94270A0C94270A9B
:10012000C787E68765885489748994899C89498939
:10013000084AD73B3BCE016E84BCBFFDC12F3D6C4E
:1001400074319ABD56833DDA3D00C77F11BED9E4B4
:10015000BB4C3E916BAAAABE000000803F076342E1
:1001600036B79BD8A71A39685618AEBAAB558C1D4E
:100170003CB7CC5763BD6DEDFD753EF6177231BFD0
:10018000000000803F08000000BE922449123EABF0
:10019000AAAA2ABECDCCCC4C3E00000080BEABAAA1
:1001A000AAAA3E00000000BF000000803F0000003F
:1001B0000000084178D3BB4387D1133D190E3CC3DF
:1001C000BD4282AD2B3E68EC8276BED98FE1A93E5E
:1001D0004C80EFFFBE01C4FF7F3F00000000000025
:1001E00025630025630025730A005854414C5F5471
:1001F00052494D3D25640025730A0025730A0054B9
:1002000065737420362025730A0054657374203595
:100210002025730A005465737420342025730A0066
:100220005465737420332025730A00546573742059
:10023000322025730A005465737420312025730A17
:10024000006368616E3D25640A0074787077723DC2
:1002500025640A003530306B0A003235306B0A00F5
:100260003131356B0A0035366B0A0033386B0A00C2
:1002700025730A00765F6C6F773D252D332E32662D
:100280000A0025730A0073656E743D252D75206480
:1002900075703D252D752069676E6F7265643D250B
:1002A0002D752074746C5F7A65726F3D252D750A0B
:1002B0000025372E33662025372E33660025352E50
:1002C000326620004572726F72203020566F6C7457
:1002D000004E6F7420737570706F727465640A00DD
:1002E0004572726F72203020566F6C7400457272C6
:1002F0006F72203020566F6C740062756C6B5F6497
:10030000656C61793D252D750062756C6B3D252D01
:10031000750056616C7565206E6F7420616C6C6F32
:100320007765640062756C6B3A206D61783D257568
:100330002073746172743D25752C20656E643D25B3
:10034000752C20696E5F7573653D25750A007062B6
:10035000323D25730A007062313D25730A00256C19
:100360007500416C6C6F77656420737065656420FF
:10037000312F31302F3130302F343030206B6269E3
:10038000742F730025630074746C3D252D64200068
:1003900074746C3D252D6420004E65772074746C58
:1003A0003D252D6420002563004D53353631312025
:1003B000503D252D372E326620252D372E32666D85
:1003C0000A00424D5030383520256C6420506120A1
:1003D00020252D372E32666D00256300545F484579
:1003E00041545F4944583D252D352E326620005436
:1003F0005F4445573D252D352E3266200041483D4E
:10040000252D352E32662000545F53485432583D16
:10041000252D352E3266200052485F5348543258FD
:100420003D252D352E32662000545F52483D252D46
:10043000342E3166200052483D252D342E31662061
:100440000025630025630025630025630025630004
:100450007265706F72745F616C6C3D007265706F75
:1004600072743D0025630025630025630025630049
:10047000204F534343414C3D256420002046757373
:10048000653A2065653D253032782068663D253027
:100490003278206C663D25303278206C623D253004
:1004A0003278004D43553D2530366C780025630089
:1004B00074785F6C656E3D252D6C752C765F6C6F66
:1004C000773D252D6C752C73687432783D252D6C25
:1004D000752C62756C6B3D252D6C75002563004F86
:1004E0004B0A002563002563002563002563002572
:1004F00063002563002563002563006465627567FA
:100500005F616C6C3D0064656275673D00646562A7
:1005100075673D0025730A00646565700A006E6F9B
:100520006E650A00707772733D007062323D25730C
:100530000A007062313D25730A00696E74725F7340
:1005400065635F70313D252D372E33660A00696E75
:1005500074725F70313D252D6C640A00696E74728F
:100560005F7365635F70303D252D372E33660A005B
:10057000696E74725F70303D252D6C640A00765F81
:100580006D63753D252D352E32660A00745F6D63EF
:10059000753D252D352E32660A00707077723D2527
:1005A000730A0064656275673D0072636D643D2582
:1005B000730A0025730A006175746F0A006C6F6717
:1005C0005F6D6F64653D007573625F7077723D2586
:1005D000730A0072656C61793D25730A0074746C4E
:1005E0003D252D640A0052494D455F616464723DAA
:1005F000252D642E252D640A006E65696768626F7B
:10060000725F7461626C655F73697A653D25640A27
:1006100000765F6C6F773D252D332E32660A0074AD
:100620007870773D25640A006368616E3D25640A31
:100630000069643D006932635F6275733D00693231
:10064000635F73706565643D252D6C750A00747871
:10065000743D25730A0053797374656D2053756D6D
:100660006D6172790A002530366C780041744D65F1
:100670006761323536524652320041744D656761CA
:10068000313238524652320041744D65676136341A
:10069000524652320041744D6567613132385246DC
:1006A0004131004D43553D006D61736B3D002C00A1
:1006B000696E74657276616C3D252D750023252D5C
:1006C000642C00745F686561745F69647800745FAE
:1006D00064657700616800705F6D73353631310095
:1006E00072685F736874327800745F73687432780C
:1006F0000070610070006164340061643300616403
:100700003200616431006133006132006131007692
:100710005F696E0072680065727200757074696D51
:10072000650070315F6C73740070315F74007031FC
:100730000070305F6C73740070305F740070300054
:10074000765F6D637500745F6D637500743100745E
:100750000069640065363400747874002D002B0045
:100760006175746F006E6F6E650062756C6B007002
:100770006F7765725F736176655F6C65647279002F
:1007800072656C61795F6C65647900636F6D70612F
:10079000737300616363656C007072657300705FF2
:1007A000707772006165730070315F6C6564790009
:1007B00070305F6C656472006576656E74006C65A0
:1007C00064006F7700706B740074785F6C65647997
:1007D0000072785F6C656472006F706572006E6F96
:1007E0006E65002530327800765F6164343D252DDA
:1007F000382E3666002000765F6164333D252D3843
:100800002E3666002000765F6164323D252D382E3D
:100810003666002000765F6164313D252D382E3626
:1008200066002000765F6C696768743D252D382E60
:100830003666002000765F61323D252D372E336607
:10084000002000765F61313D252D372E3366002074
:1008500000765F696E3D252D352E326600204E658F
:100860007665722D7573656420737461636B203EC9
:100870002025642062797465730A00757074696D4F
:10088000653D252D642D646179732D253032643AE0
:10089000253032643A253032642D686F7572730AE0
:1008A0000074657374205B6F66667C317C327C33C8
:1008B0007C347C355D20202020202020202D2074B9
:1008C000657374206D6F6465730A0D007478205B26
:1008D000706B74207061796C6F61645D20202020E2
:1008E00020202020202020202D2073656E6420727F
:1008F0006164696F20706B74206B6579626F6172DF
:10090000640A0D00776474205B6F6E7C6F66667C92
:10091000746573745D20202020202020202020205A
:100920002D207761746368646F670A0D00765F6CD1
:100930006F77205B765F6C6F775D20202020202012
:100940002020202020202020202D206C6F77657310
:1009500074207265706F727420766F6C7461676555
:100960000A0D007570677220202020202020202092
:100970002020202020202020202020202020202D6A
:10098000207265626F6F742076696120626F6F7488
:100990006C6F616465720A0D0075617274205B335F
:1009A000386B7C35366B7C3131356B7C3235306B56
:1009B0007C3530306B5D202D20736574207465723A
:1009C0006D2F756172742073706565640A0D006225
:1009D0006F6F742020202020202020202020202025
:1009E00020202020202020202020202D2072656221
:1009F0006F6F740A0D0070777273205B64656570A9
:100A00007C6E6F6E655D202020202020202020201D
:100A100020202D206D637520736C656570206D6FCF
:100A200064650A0D007265737420656570726F6D80
:100A300020202020202020202020202020202020B6
:100A4000202D20726573746F726520656570726FFA
:100A50006D0A0D0070707772205B6F6E7C6F66663A
:100A60005D20202020202020202020202020202049
:100A70002D2070726F6772616D6D61626C652070A0
:100A800077720A0D0070623220205B6F6E7C6F6699
:100A9000665D2020202020202020202020202020D3
:100AA000202D2070726F6772616D6D61626C6520C0
:100AB00070696E2062320A0D0070623120205B6F17
:100AC0006E7C6F66665D2020202020202020202064
:100AD00020202020202D2062756C6B204750494F2C
:100AE0002070696E0A0D00747874205B73747269EB
:100AF0006E675D2020202020202020202020202024
:100B00002020202D20536574207265706F72742030
:100B10007465787420737472696E670A0D00747856
:100B20007077205B31352D305D2020202020202063
:100B3000202020202020202020202D20545820500C
:100B400077722E20486967686573742030202833D7
:100B500064426D290A0D0074746C205B302D3135B0
:100B60005D20202020202020202020202020202048
:100B70002020202D2074696D652D746F2D6C697691
:100B80006520666F72207061636B6574730A0D0077
:100B900073732020202020202020202020202020AF
:100BA0002020202020202020202020202D2073798C
:100BB0007374656D2073756D6D6172790A0D0072C5
:100BC00073202020202020202020202020202020D2
:100BD00020202020202020202020202D2072616431
:100BE000696F2073746174730A0D007269205B234E
:100BF0006E5D205B696E745D202020202020202007
:100C0000202020202020202D207265706F727420FB
:100C1000696E74657276616C0A0D0072636D642092
:100C20005B6F6E7C6F66665D202020202020202078
:100C3000202020202020202D20616C6C6F772063E5
:100C40006D642066726F6D206E65746F726B0A0D35
:100C5000007265205B236E5D205B2B7C2D5D205B2D
:100C60006D61736B7C6175746F2C6D61736B5D204E
:100C70002D206D6F7465207265706F7274207365BE
:100C8000742F6D6F646966790A0D006F77202020DC
:100C90002020202020202020202020202020202054
:100CA000202020202020202D206F6E652D77697256
:100CB000652073656E736F72730A0D006C6F672029
:100CC0005B6175746F7C6F6E7C6F66665D20202043
:100CD00020202020202020202D206D6F746573207F
:100CE00064617461206F6E205553420A0D006E6579
:100CF000205B666C7573685D2020202020202020FA
:100D0000202020202020202020202D206E656967B3
:100D100068626F72207461626C650A0D00657272A0
:100D200020202020202020202020202020202020C3
:100D30002020202020202020202D206572726F721C
:100D40002073746174730A0D006D63752020202078
:100D50002020202020202020202020202020202093
:100D600020202020202D206D637520696E666F0A7B
:100D70000D00693263205B70726F62657C73706511
:100D8000656420236E5D20202020202020202D203F
:100D90006932632070726F6265206275737C73655F
:100DA00074206275732073706565640A0D00696450
:100DB000205B72657365745D202020202020202038
:100DC000202020202020202020202D206964206841
:100DD000616E646C696E670A0D0068756D20202075
:100DE0002020202020202020202020202020202003
:100DF0002020202020202D2068756D696469747979
:100E00002073656E736F720A0D0072656C617920D4
:100E10005B6F6E7C6F66667C73746174735D20209B
:100E20002020202020202D2072656C6179206E65A5
:100E300074776F726B207265706F7274730A0D0035
:100E40006465205B6D61736B5D2020202020202075
:100E50002020202020202020202020202D206465FC
:100E60006275670A0D006368616E205B31312D3257
:100E7000365D20202020202020202020202020201F
:100E800020202D206368616E2031312D32362028DC
:100E9000322E3430352D32343830204D687A290ADC
:100EA0000D0063616C69205B5B765F696E7C61310C
:100EB0007C61325D20766F6C747C72657365747CC6
:100EC0006E6F6E655D202D2063616C696272617466
:100ED000650A0D0062756C6B205B5B73686F777CD5
:100EE000666C7573685D205B7365742074687273DB
:100EF000682064656C61795D5D20202D2062756CD1
:100F00006B696E67207061636B657473200A0D00F6
:100F10006164632020202020202020202020202009
:100F20002020202020202020202020202D20736819
:100F30006F7720765F696E2C2061312C2061322022
:100F4000766F6C74616765730A0D00752020202030
:100F50002020202020202020202020202020202091
:100F6000202020202020202D20757074696D650AB6
:100F70000D0076202020202020202020202020204E
:100F800020202020202020202020202020202D2054
:100F900076657273696F6E0A0D006820202020202C
:100FA0002020202020202020202020202020202041
:100FB0002020202020202D2068656C700A0D00253F
:100FC0006300756E6B6E6F776E20636D640A004808
:100FD0004D433538383300257300257300202573C1
:100FE000002025362E3266200025303278007465C8
:100FF0006D705F65787465726E3D252D362E326694
:1010000000202573002025362E3266204F6E2D429B
:101010006F61726400253032780074656D705F62B4
:101020006F6172643D252D362E3266000A004275CE
:101030006C6B2072656D3A2073746172743D257516
:101040002C20656E643D25752C20696E5F75736577
:101050003D25750A0042756C6B206164643A20730B
:10106000746172743D25752C20656E643D25752C68
:1010700020696E5F7573653D25750A0042756C6B5E
:10108000207468726573683A2074696D65723D25D5
:10109000750A00503A20256C642050612020252DCF
:1010A000372E3266206D0A004932433A200045202F
:1010B00025642E256420636C6F636B20256C75207E
:1010C00063707520256C75206C706D20256C752003
:1010D00069727120256C7520676C656420256C75BC
:1010E00020796C656420256C7520726C6564202500
:1010F0006C7520747820256C75206C697374656E2E
:1011000020256C752073656E736F727320256C7566
:101110002073657269616C20256C750A0053202567
:10112000642E256420636C6F636B20256C752074BE
:101130007820256C7520727820256C752072747863
:1011400020256C752072727820256C752072657868
:101150006D697420256C752061636B747820256C33
:1011600075206E6F61636B747820256C75206163E8
:101170006B727820256C752074696D65646F757469
:1011800020256C752062616461636B727820256C28
:101190007520746F6F6C6F6E6720256C7520746F8F
:1011A0006F73686F727420256C7520626164737947
:1011B0006E636820256C752062616463726320250C
:1011C0006C7520636F6E74656E74696F6E64726F98
:1011D0007020256C752073656E64696E6764726F2C
:1011E0007020256C75206C6C747820256C75206CD3
:1011F0006C727820256C750A00257325730A004FE0
:101200006E6C696E650A000A002C20636865636B6A
:10121000207261746520257520487A002573202589
:10122000732C206368616E6E656C20257520706F6D
:10123000776572202575000A0025783A004D4143F4
:101240002061646472657373200052616E646F6D17
:101250002045554936342061646472657373206794
:10126000656E6572617465640A000A2A2A2A2A2A50
:101270002A2A426F6F74696E672025732A2A2A2AE8
:101280002A2A2A0A00454550524F4D20697320638F
:101290006F72727570742C20726577726974696EE2
:1012A0006720776974682064656661756C74732E55
:1012B0000A006C6F63616C686F73740041544D4534
:1012C00047413132387266613100020000FFFE0092
:1012D00000016E616E00696E660000407A10F35A7C
:1012E00000A0724E18090010A5D4E80000E8764866
:1012F000170000E40B54020000CA9A3B000000E112
:10130000F505000080969800000040420F000000A4
:10131000A08601000000102700000000E803000084
:1013200000006400000000000A000000000001004E
:10133000000000002C76D888DC674F0823DFC1DF6F
:10134000AE59E1B1B796E5E3E453C63AE651997672
:1013500096E8E6C28426EB898C9B62ED407C6FFCAC
:10136000EFBC9C9F40F2BAA56FA5F490055A2AF7EE
:101370005C936B6CF9676DC11BFCE0E40D47FEF5F7
:1013800020E6B500D0ED902E03009435770500805F
:10139000841E080000204E0A000000C80C333333BE
:1013A000330F986E12831141EF8D2114893BE6555E
:1013B00016CFFEE6DB18D1844B381BF77C1D901D41
:1013C000A4BBE424203284725E228100C9F124ECA3
:1013D000A1E53D274E414E494E495459494E46CD0F
:1013E000CCCC3D0AD7233C17B7D13877CC2B3295DC
:1013F00095E6241FB14F0A000020410000C84200BA
:10140000401C4620BCBE4CCA1B0E5AAEC59D740083
:1014100011241FBECFEFD1E4DEBFCDBF1AE0A0E0A4
:10142000B2E0EEE1F9E301E00BBF02C007900D92DC
:10143000AA33B107D9F72DE3AAE3BAE001C01D92A0
:10144000A436B207E1F70E946B8A0C948D9C0C9431
:1014500000008115910511F00197F1F7089584E2DC
:1014600095E09F938F930E9472998091660290916C
:101470006702A0916802B09169020F900F9093FFEC
:1014800003C08EE195E002C088E195E09F938F93C1
:101490000E9472990F900F900895E091FD1BEF73D9
:1014A000F0E0E25BF34E80838091FD1B8F5F8093C1
:1014B000FD1B80919E34886080939E344CE452E002
:1014C00061E1CA010E94F05A80E090E00895CF9354
:1014D000DF93EC014091410A5091420A6091430A26
:1014E0007091440A46FF1DC08E811F928F938D819B
:1014F0001F928F938C811F928F938B811F928F935A
:101500008A811F928F9385E793E09F938F930E9428
:1015100060998DB79EB70C960FB6F8949EBF0FBE1C
:101520008DBFBE0182E89AE00E94225CBE0184E089
:1015300092E0DF91CF910C94975B1092B41C1092C3
:10154000B51C1092B31C0895CF92DF92EF92FF92D8
:101550000F931F93CF93DF93EC01FB018091B31C9A
:10156000843108F0B7C08091B51C64E10E94759287
:101570009093B51CC090D02FD090D12FE090D22F57
:10158000F090D32F092F10E06DE8969F9001112461
:101590002D54334ED9011396CD92DD92ED92FC92EB
:1015A00016974115510569F0DA018C91D901AA57B6
:1015B000BF4F8C93DA0111968C91D901A957BF4F77
:1015C0008C932097A1F029813DE8309FC001319F85
:1015D000900D11248D54934EDC01A657BF4F2C93D0
:1015E000119688818F708C9388818F708C9330973F
:1015F000B9F186819DE8909F9001919F300D112453
:101600002D54334ED901A757BF4F8C938581119725
:101610008C93A90144575F4F83859485A585B68532
:10162000C92EDA2EEB2EFF24DA01CD92DC9279015D
:10163000BEE8EB0EF11C2385348545855685A4E66E
:10164000B0E00E941593672F782F892F992724E601
:1016500030E040E050E00E94A992F701718360837E
:101660008DE8809FD001819FB00D1124A654B34E08
:10167000FE0132968FE701900D928A95E1F7209155
:10168000B51C2F5F2093B51C3091B31C3F5F309386
:10169000B31C8091410A9091420AA091430AB091F3
:1016A000440AA0FF2DC01F923F931F922F93809159
:1016B000B41C1F928F9385E590E19F938F930E94B6
:1016C00072998DB79EB708960FB6F8949EBF0FBE5D
:1016D0008DBF16C08091E02F9091E12FA091E22F55
:1016E000B091E32F0196A11DB11D8093E02F90933F
:1016F000E12FA093E22FB093E32F80E090E002C0AF
:1017000081E090E0DF91CF911F910F91FF90EF90DA
:10171000DF90CF9008952091B31C222369F180912E
:10172000B41C8F5F21502093B31C64E10E9475921A
:10173000392F9093B41C8091410A9091420AA09154
:10174000430AB091440AA0FF1AC01F922F938091C0
:10175000B51C1F928F931F923F938EE290E19F934F
:101760008F930E9472998DB79EB708960FB6F89422
:101770009EBF0FBE8DBF03C080E090E0089581E062
:1017800090E008958823B9F052985A981DBA809134
:101790006900806280936900EA9A53985B98EB9A9B
:1017A0008091690080688093690080916800816001
:1017B000809368000895109269005A9AEA985B9A9B
:1017C000EB9808951F920F920FB60F9211248F93EA
:1017D0009F93AF93BF938091680080FF24C0809156
:1017E000793490917A34A0917B34B0917C34019615
:1017F000A11DB11D8093793490937A34A0937B34EA
:10180000B0937C348091410A9091420AA091430A9E
:10181000B091440A87FF07C0749882E090E09093EB
:10182000930280939202BF91AF919F918F910F90FD
:101830000FBE0F901F9018951F920F920FB60F9228
:1018400011248F939F93AF93BF938091680080FF83
:1018500024C080917D3490917E34A0917F34B091EA
:1018600080340196A11DB11D80937D3490937E3408
:10187000A0937F34B09380348091410A9091420AC2
:10188000A091430AB091440A90FF07C0739882E088
:1018900090E09093930280939202BF91AF919F91B9
:1018A0008F910F900FBE0F901F90189580937C0022
:1018B00080917B00877F80937B0080917C00806C8F
:1018C00080937C0085E080937A0080917A00806824
:1018D00080937A0080917B0087FFFCCF80917B0012
:1018E00085FFFCCF80917A00806480937A0080919C
:1018F0007A0086FDFCCF109279001092780084E087
:1019000090E060E070E020917A00206420937A00FB
:1019100020917A0026FDFCCF20917800309179004B
:10192000620F731F0197009771F710927C008091EE
:101930007A008F7780937A0076956795769567958C
:1019400080E090E00E94C18F089580E00E94560CD4
:1019500020918A0230918B0240918C0250918D022D
:101960000E94A59121EE3AE744E95EE30E945A8E77
:1019700008950F931F93CF93DF93CFE1D0E00BE552
:101980001EE0C093510187EC90E00E94290A8091EB
:10199000510185FD0DC0C031D10521F02CF00B5453
:1019A000110904C004EC19E0025311092197E9CF91
:1019B000B80180E090E00E94C18F20E030E04AE76B
:1019C00054E40E94248FDF91CF911F910F910895CD
:1019D000CF93DF93EC0188819981009799F0873D3F
:1019E000914121F01982188283E011C0623171F4B3
:1019F0000E94B90C6093CC2F7093CD2F8093CE2F83
:101A00009093CF2F87ED91E19983888381E0DF91D7
:101A1000CF91089580917B00886080937B0089EC52
:101A200080937C0085E080937A0080917A008068C2
:101A300080937A0080917B0087FFFCCF80917B00B0
:101A400085FFFCCF80917A00806480937A0080913A
:101A50007A0086FDFCCF80917A00806480937A00C2
:101A600080917A0086FDFCCF6091780070917900BA
:101A700080917A008F7780937A0080E090E00E94D6
:101A8000C18F27ED33EA40E95FE30E94A59126E686
:101A900036E648E853E40E94598E0895BF92CF92EB
:101AA000DF92EF92FF920F931F93CF93DF93CDB707
:101AB000DEB729970FB6F894DEBF0FBECDBF6C011D
:101AC00010923A0A8FEF89870EE01CE1B12C7E015B
:101AD00089E0E80EF11C89858823E9F1E8E0BE166B
:101AE000E1F1BE016F5F7F4FC7010E948B64898562
:101AF0008F3F11F08E3F19F480933A0A2CC0CE012B
:101B00000196C114D10471F40E94A46480939B34A3
:101B1000FE013196A3E9B4E381918D93EE15FF05A3
:101B2000D9F71DC00E94A464F8018083FE0131969C
:101B300020E030E0A801485051098191DA01A20F5C
:101B4000B31F8C932F5F3F4F28303105B1F7B3940B
:101B5000075F1F4FC0CF8B2D03C088E001C081E01D
:101B600029960FB6F894DEBF0FBECDBFDF91CF919F
:101B70001F910F91FF90EF90DF90CF90BF9008954D
:101B80008CE290E19F938F930E9472990F900F9037
:101B900008952F923F924F925F926F927F928F9211
:101BA0009F92AF92BF92CF92DF92EF92FF920F93EC
:101BB0001F93CF93DF93EC014B01009711F427E0C3
:101BC00004C08130910549F426E04AE250E06BE21E
:101BD00070E089E290E00E946B63CE010E944E0D9E
:101BE0009E01255C354F5901D9018C93CD2B69F0AD
:101BF000AEE0CA2EACE1DA2EC6E0DCE1E12CF12C3D
:101C0000BDED2B2EBFE03B2EA6C083E994E30E94DE
:101C1000D965BC01882777FD8095982F0E94C38FD6
:101C20006B017C01892869F020E030E048EC52E447
:101C30000E94248F9F938F937F936F938AE190E10B
:101C4000ACC0C3E9D4E305E110E189911F928F9301
:101C50001F930F930E9472990F900F900F900F9007
:101C6000B4E3CB39DB0789F720E030E048EC52E4FD
:101C7000C701B6010E94248F9F938F937F936F9328
:101C800085E090E19F938F930E9472990F900F903F
:101C90000F900F900F900F9080919B34882319F034
:101CA00084EA93E002C088E194E09F938F9381E0FF
:101CB00090E19F938F930E9472990F900F900F90D5
:101CC0000F9075C000E010E0FE01E00FF11F808171
:101CD0001F928F93A9EEBFE0BF93AF930E947299BA
:101CE0000F5F1F4F0F900F900F900F90083011054E
:101CF00059F720E030E048EC52E4C301B2010E9401
:101D0000248F9F938F937F936F93A1EEBFE0BF9338
:101D1000AF930E9472990F900F900F900F900F90B9
:101D20000F90D6018C91882309F455C084EA93E082
:101D30009F938F933F922F920E9472990E94C00DA1
:101D4000BFEFEB1AFB0AE9E0CE0ED11C29960F90EB
:101D50000F900F900F90D5018C9190E0E816F90646
:101D6000ECF5CE010E94D965BC01882777FD8095EE
:101D7000982F0E94C38F2B013C018114910409F418
:101D8000A1CF20E030E048EC52E40E94248F9F93E2
:101D90008F937F936F938EEE9FE09F938F930E941C
:101DA00072990F900F900F900F900F900F90DF91FE
:101DB000CF911F910F91FF90EF90DF90CF90BF9048
:101DC000AF909F908F907F906F905F904F903F90DB
:101DD0002F900C94C00D88E194E0AACFDF91CF91B1
:101DE0001F910F91FF90EF90DF90CF90BF90AF9039
:101DF0009F908F907F906F905F904F903F902F902B
:101E00000895CF93DF9300D0CDB7DEB7809194349F
:101E1000898380919A348A83CE0101960E94E45886
:101E20000F900F90DF91CF910895CF93DF93EC0146
:101E3000209193343091943440919534509196345C
:101E400060919734709198348091993490919A343C
:101E5000AFEF0E94E194E1F427E04AE250E06BE248
:101E600070E089E290E00E946B6380E090E00E9465
:101E70004E0DC55CD54F888349E050E06EE070E0C0
:101E800083E994E30E94E49ADF91CF910C94010FCF
:101E9000DF91CF9108951F920F920FB60F921124E8
:101EA0000BB60F92FF920F931F932F933F934F9375
:101EB0005F936F937F938F939F93AF93BF93CF93D2
:101EC000DF93EF93FF9380919E34826080939E34E2
:101ED0008091660286FD2B9A8091660287FD2B9A7F
:101EE00080919202909193021816190614F4749A34
:101EF000739A8091410A9091420AA091430AB0914D
:101F0000440A85FF02C074987398809102029091F0
:101F1000030201979093030280930202892B09F038
:101F20004BC18091510A9091520A01969093520AA6
:101F30008093510A8091D02F9091D12FA091D22FD0
:101F4000B091D32F0196A11DB11D8093D02F9093F6
:101F5000D12FA093D22FB093D32F80E190E0909314
:101F60000302809302028091660280FD02C01D9BE5
:101F700005C010923F0A10923E0A06C081E090E030
:101F800090933F0A80933E0A8091410A9091420AC1
:101F9000A091430AB091440A97FF08C080913E0A7D
:101FA00090913F0A892B49F0749A7398CDEADBE14E
:101FB00005EE1FE2FF24F3941FC0739A7498F6CFC6
:101FC0008091510A9091520A01960E948192892B28
:101FD000C9F0688579856115710591F56885798500
:101FE0006115710509F03FC02A960B5F1F4FFBE199
:101FF000C53DDF0709F44DC0688579856115710518
:1020000041F3DECF4A81417020E030E050E060E0F3
:1020100070E080E090E0A0E00E94E194D1F2779837
:102020008091410A9091420AA091430AB091440ADA
:1020300092FFCFCF74981092930210929202C9CF60
:102040008091510A9091520A01960E948192892BA7
:1020500029F6F80114821382A80162E184E292E079
:102060000E94F05ABBCF8091510A9091520A0E946F
:102070008192892B09F0B8CFF801F082D283C18315
:1020800014821382A80162E182E492E00E94F05A75
:10209000ABCF60916C0270916D0261157105A1F179
:1020A0008091510A9091520A0E948192892B61F588
:1020B0008091793490917A34A0917B34B0917C34C2
:1020C0004091C2275091C3276091C4277091C527C2
:1020D000841B950BA60BB70B8093D51B9093D61B37
:1020E000A093D71BB093D81B8091793490917A3408
:1020F000A0917B34B0917C348093C2279093C32706
:10210000A093C427B093C52760916A0270916B02B7
:1021100061157105A1F18091510A9091520A0E94B6
:102120008192892B61F580917D3490917E34A091CC
:102130007F34B09180344091C6275091C727609179
:10214000C8277091C927841B950BA60BB70B8093EA
:10215000D91B9093DA1BA093DB1BB093DC1B8091FF
:102160007D3490917E34A0917F34B09180348093FF
:10217000C6279093C727A093C827B093C9278091FB
:10218000660286FD2B988091660290916702A0916D
:102190006802B091690291FF0FC00E948A6F8A3174
:1021A00019F0C1E0C80F01C0CBE00E94466E8C2F31
:1021B0000E94A26F0E948E6E40E050E060E084E9D1
:1021C00092E00E94F05AFF91EF91DF91CF91BF9181
:1021D000AF919F918F917F916F915F914F913F91BF
:1021E0002F911F910F91FF900F900BBE0F900FBE7C
:1021F0000F901F9018958091FD1B9091E42F891BE3
:1022000008950E94FB10882371F0E091E42FEF7392
:10221000F0E0E25BF34E808190E02091E42F2F5FAD
:102220002093E42F08958FEF9FEF0895CF93DF93CE
:10223000EC011092760A1092750A888199810097B4
:10224000B1F0843E934021F01982188283E0B6C039
:10225000613109F0B2C00E94011199279093710A6F
:102260008093700A8D3009F443C08F3F49F40E9477
:10227000FB108111F0CF84EE93E0998388839DC099
:102280008231910509F45AC08F37910509F052C087
:1022900080916E0A90916F0A181619060CF56091DC
:1022A0005E3D70915F3D88E090E00E942E996091C4
:1022B0005E3D70915F3D80E290E00E942E996091BA
:1022C0005E3D70915F3D88E090E00E942E99809184
:1022D0006E0A90916F0A019790936F0A80936E0A2D
:1022E00080916E0A90916F0A8F37910509F0BFCFE8
:1022F0001092E42F1092FD1B80916E0A90916F0A4C
:10230000FC01E750F04D10829093760A8093750A95
:1023100010926F0A10926E0A80919C3490919D34B5
:10232000009709F4A4CF40E050E0609184120E942D
:10233000F05A9DCF8830910571F5AACF60915E3D2E
:1023400070915F3D8DE090E00E942E9910926D0A91
:1023500010926C0A80916C0A90916D0A20916E0A1D
:1023600030916F0A821793070CF0BACFFC01E75047
:10237000F04D808160915E3D70915F3D90E00E94E4
:102380002E9980916C0A90916D0A019690936D0A36
:1023900080936C0ADFCF60915E3D70915F3D0E943B
:1023A0002E9980916E0A90916F0A2091700AFC011B
:1023B000E750F04D208301968FCF81E0DF91CF91E0
:1023C000089580913E0A90913F0A892BD1F0809127
:1023D000660290916702A0916802B091690293FD34
:1023E00010C00E94466E83B7817F866083BFF894D9
:1023F00083B7816083BF7894889583B78E7F83BFCE
:1024000078940895CF93DF93EC01888199810097A8
:1024100019F08A30924199F40E94036D0E94E111F3
:1024200040E050E065E880918812909189120E9406
:10243000F05A8AE092E19983888381E003C019828F
:10244000188283E0DF91CF910895CF93DF9300D07E
:10245000CDB7DEB7892B81F05F934F938AED9FE074
:102460009F938F9369837A830E9472990F900F9044
:102470000F900F907A8169817F936F9387ED9FE032
:102480009F938F930E9472990F900F900F900F90CF
:102490000F900F90DF91CF910895FF920F931F93AC
:1024A000CF93DF930E94036D80EB0E9466668111DB
:1024B0001CC00E94CA668091CA2B9091CB2B816070
:1024C0009093CB2B8093CA2B8DEA93E09F938F93AD
:1024D00087ED9FE09F938F930E9472990F900F90CA
:1024E0000F900F90C1E0D0E002C0C0E0D0E0FEB09D
:1024F0008F2D8470F82E729A0E94036D8EE40E94D4
:102500006666811116C00E94CA668091CA2B90919E
:10251000CB2B82609093CB2B8093CA2B8E010F5FC5
:102520001F4F4FE959E065EB73E0CE010E94251281
:10253000E801F11001C072980E94036D8EEE0E94B6
:102540006666811116C00E94CA668091CA2B90915E
:10255000CB2B84609093CB2B8093CA2B8E010F5F83
:102560001F4F4FE959E06DEB73E0CE010E94251239
:10257000E8010E94036D86EA0E946666811116C01A
:102580000E94CA668091CA2B9091CB2B8860909351
:10259000CB2B8093CA2B8E010F5F1F4F4FE959E061
:1025A00064EC73E0CE010E942512E8010E94036DE5
:1025B0008CE30E94666681111EC00E94CA668091EB
:1025C000CA2B9091CB2B80619093CB2B8093CA2BFD
:1025D0008E010F5F1F4F4FE959E06CEC73E0CE01A5
:1025E0000E9425128FEC9FE09F938F930E94729917
:1025F0000F900F90E8010E94036D82ED0E946666C5
:10260000811116C00E94CA668091CA2B9091CB2B73
:1026100080629093CB2B8093CA2B8E010F5F1F4F4C
:102620004FE959E064ED73E0CE010E942512E80104
:102630000E94036D80E80E946666811116C00E94A8
:10264000CA668091CA2B9091CB2B91609093CB2B33
:102650008093CA2B8E010F5F1F4F4FE959E06DED3C
:1026600073E0CE010E942512E8010E94036D80ED07
:102670000E946666811116C00E94CA668091CA2BAC
:102680009091CB2B80689093CB2B8093CA2B8E019B
:102690000F5F1F4F4FE959E063EE73E0CE010E94D8
:1026A0002512E8010E94036D8CEE0E94666681117E
:1026B00016C00E94CA668091CA2B9091CB2B926063
:1026C0009093CB2B8093CA2B8E010F5F1F4F4FE946
:1026D00059E06BEE73E0CE010E942512E80107E09D
:1026E00010E00E94036D8CE70E946666811113C0A2
:1026F0000E94CA668091CA2B9091CB2B80649093E4
:10270000CB2B8093CA2B4FE959E062EF73E0CE01E7
:102710000E94251205C0015011090115110509F784
:102720000E94CA66DF91CF911F910F91FF900C9488
:10273000C00DCF93DF9300D0CDB7DEB74A83698356
:102740000E94A1666981862F0E94D2664A81842FE9
:102750000E94D2660F900F90DF91CF910C94CA66C1
:10276000AF92BF92DF92EF92FF920F931F93CF939E
:10277000DF9300D01F92CDB7DEB7182FD22E4A8339
:102780005B8369830E94A1666981862F0E94D2665D
:10279000812F81600E94C8664A81A42E5B81B52E7C
:1027A00000E010E0ED2CF12C81E0E81AF1080D15A5
:1027B00080F40E151F0519F40E94ED6602C00E94F8
:1027C000E366F50180830F5F1F4FFFEFAF1ABF0A6B
:1027D000EECF0F900F900F90DF91CF911F910F913F
:1027E000FF90EF90DF90BF90AF900C94CA66AF92CD
:1027F000BF92CF92DF92EF92FF920F931F93CF93EE
:10280000DF93CDB7DEB760970FB6F894DEBF0FBE8B
:10281000CDBFB82EA42E6623E9F18E010F5F1F4FA6
:1028200080E1F80111928A95E9F728E0A80168E9AA
:1028300080EB0E94B013BB2041F02BEF33E03F93BD
:102840002F930E9460990F900F906E01F8E0CF0EC9
:10285000D11C92E0E92E94E0F92EF80181918F01CC
:102860001F928F93FF92EF920E9460990F900F90AA
:102870000F900F900C151D0581F788851F928F937F
:1028800027E534E03F932F930E9460990F900F90BB
:102890000F900F90AA20E9F18E010F5F1F4F80E18A
:1028A000F80111928A95E9F728E0A80160E880EB29
:1028B0000E94B013BB2041F087E094E09F938F9378
:1028C0000E9460990F900F906E01F0E1CF0ED11C25
:1028D00082E0E82E84E0F82EF80181918F011F92AA
:1028E0008F93FF92EF920E9460990F900F900F903C
:1028F0000F900C151D0581F788851F928F9387E532
:1029000094E09F938F930E9460990F900F900F9087
:102910000F9060960FB6F894DEBF0FBECDBFDF916B
:10292000CF911F910F91FF90EF90DF90CF90BF90CC
:10293000AF900895CF93DF9300D0CDB7DEB71A8262
:10294000198222E0AE014F5F5F4F6AEA8EEE0E946D
:10295000B013898190E0982F88272A81822B909349
:102960008F1C80938E1C22E0AE014F5F5F4F6CEA9C
:102970008EEE0E94B013898190E0982F88272A81DB
:10298000822B9093911C8093901C22E0AE014F5FAC
:102990005F4F6EEA8EEE0E94B013898190E0982F0F
:1029A00088272A81822B9093931C8093921C22E08B
:1029B000AE014F5F5F4F60EB8EEE0E94B0138981D6
:1029C00090E0982F88272A81822B9093A11C8093D6
:1029D000A01C22E0AE014F5F5F4F62EB8EEE0E94C3
:1029E000B013898190E0982F88272A81822B9093B9
:1029F000A31C8093A21C22E0AE014F5F5F4F64EBEB
:102A00008EEE0E94B013898190E0982F88272A814A
:102A1000822B9093A51C8093A41C22E0AE014F5FF3
:102A20005F4F66EB8EEE0E94B013898190E0982F85
:102A300088272A81822B9093951C8093941C22E0F6
:102A4000AE014F5F5F4F68EB8EEE0E94B01389813D
:102A500090E0982F88272A81822B9093971C80934F
:102A6000961C22E0AE014F5F5F4F6AEB8EEE0E9434
:102A7000B013898190E0982F88272A81822B909328
:102A80009B1C80939A1C22E0AE014F5F5F4F6CEB62
:102A90008EEE0E94B013898190E0982F88272A81BA
:102AA000822B90939D1C80939C1C22E0AE014F5F73
:102AB0005F4F6EEB8EEE0E94B013898190E0982FED
:102AC00088272A81822B90939F1C80939E1C0F90B5
:102AD0000F90DF91CF9108952F923F924F925F9286
:102AE0006F927F928F929F92AF92BF92CF92DF921E
:102AF000EF92FF920F931F93CF93DF93CDB7DEB783
:102B00006A970FB6F894DEBF0FBECDBF182F488F5F
:102B1000298F19821A821B828091B21C811107C0F1
:102B20006A8F0E949A1481E08093B21C6A8D66239A
:102B300009F46CC04EE264EF8EEE0E94991369E0D6
:102B40007AE180E090E00E94446622E0AE014F5FAF
:102B50005F4F66EF8EEE0E94B0132981822F90E0C6
:102B6000A0E0B0E02227382F492F5A2F8A81282B46
:102B70008091A41C9091A51C281B390B4109510977
:102B8000A091A21CB091A31C0E9415936B017C0123
:102B90008FE0F594E794D794C7948A95D1F7609124
:102BA0009C1C70919D1C882777FD8095982F2BE0A9
:102BB000660F771F881F991F2A95D1F720919E1CB9
:102BC00030919F1C442737FD4095542F2C0D3D1DFF
:102BD0004E1D5F1D0E94CB92C20ED31ED092991C37
:102BE000C092981C88E0C80ED11C34E0D594C794DC
:102BF0003A95E1F7EE24D7FCE094FE2CC092A61C97
:102C0000D092A71CE092A81CF092A91C012F02955B
:102C1000000F000F007C0C5CA12FB0E0BD8BAC8BD3
:102C2000A3E0B0E0012E02C0AA0FBB1F0A94E2F796
:102C300025E335E00E940E93DC01CB010296A11D35
:102C4000B11D8C879D87AE87BF8780E593ECA0E0A0
:102C5000B0E004C0B595A795979587951A95D2F7DA
:102C6000888B998BAA8BBB8B10E0188619861A86E5
:102C70001B86A8E02A2E312CAC89BD892A1A3B0A72
:102C8000988D191709F436C1402F64EF8EEE0E941B
:102C900099136C857D858E859F850E94446623E00F
:102CA000AE014F5F5F4F66EF8EEE0E94B013E09172
:102CB000981CF091991CE05AFF409F01DF010E948F
:102CC000F7926B017C018091901C9091911C9F8BDD
:102CD0008E8BA0908E1CB0908F1C2091921C3091F6
:102CE000931C0E94F7922B013C01ADE07594679410
:102CF00057944794AA95D1F7A091941CB091951C34
:102D0000A70196018CE055954795379527958A95AB
:102D1000D1F70E942093BB2797FDB095AB2F480EAB
:102D2000591E6A1E7B1E92E0490E511C611C711CCB
:102D300032E075946794579447943A95D1F7A0E898
:102D40005A0E611C711CA091A01CB091A11CA30182
:102D500092010E941593DC01CB014FE0B695A79537
:102D6000979587954A95D1F78C839D83AE83BF83D2
:102D700029818A8190E0A0E0B0E04424582E692E99
:102D80007A2E622A8B81482A022C04C0759467949B
:102D9000579447940A94D2F74501AA2497FCA0942B
:102DA000BA2C62E0880C991CAA1CBB1C6A95D1F74E
:102DB000A091961CB091971CA70196010E942093A8
:102DC0006B017C0177E1F594E794D794C7947A95E9
:102DD000D1F72E893F89DF010E94F792EBE09595AC
:102DE000879577956795EA95D1F7C60ED71EE81EA9
:102DF000F91E8C0C9D1CAE1CBF1C0C8804C0880CDA
:102E0000991CAA1CBB1C0A94D2F792E0890E911C53
:102E1000A11CB11CF2E0B594A79497948794FA95FD
:102E2000D1F7481859086A087B08A30192016889FC
:102E300079898A899B890E94659297FD0DC0660FEA
:102E4000771F881F991F2C813D814E815F810E94D1
:102E5000A99249015A010CC02C813D814E815F81AC
:102E60000E94A99249015A01880C991CAA1CBB1CFA
:102E70009927B7FC9A958B2D7A2D692D9B01AC0172
:102E80000E9465929B01AC01AEEDBBE00E941593E0
:102E90006C01FF24D7FCF094EF2CA3E4B3EEA50162
:102EA00094010E942393BB2797FDB095AB2FC80ECA
:102EB000D91EEA1EFB1EAFECCA0EAEE0DA1EE11C04
:102EC000F11C64E0F594E794D794C7946A95D1F720
:102ED000C80CD91CEA1CFB1C88859985AA85BB8572
:102EE0008C0D9D1DAE1DBF1D88879987AA87BB8746
:102EF0001F5FC6CE112391F0212F30E040E050E05B
:102F0000688579858A859B850E94A9922093AA1C51
:102F10003093AB1C4093AC1C5093AD1CA98DAA23DD
:102F200089F16091AA1C7091AB1C8091AC1C9091AE
:102F3000AD1C611571058105910521F10E94C38FBA
:102F400020E836EE45EC57E40E94248F21E03EED68
:102F500042E45EE30E9408929B01AC0160E070E0F5
:102F600080E89FE30E94598E2BE43AE34DEB57E350
:102F70000E94248F6093AE1C7093AF1C8093B01C92
:102F80009093B11C6A960FB6F894DEBF0FBECDBF0A
:102F9000DF91CF911F910F91FF90EF90DF90CF9035
:102FA000BF90AF909F908F907F906F905F904F9069
:102FB0003F902F9008950F931F93CF93DF9300D0EE
:102FC00000D000D0CDB7DEB78E010F5F1F4F86E077
:102FD000F80111928A95E9F78091A41B811113C021
:102FE00040E061E386EA0E9499134AE06CE286EAD7
:102FF0000E94991381E08093A41B6CE77EE380E03C
:1030000090E00E94446648E06DE286EA0E949913CF
:103010006CE77EE380E090E00E94446626E0A80131
:1030200062E386EA0E94B01347E06DE286EA0E94FE
:1030300099138A8190E0982F88272981822B909379
:103040009F1B80939E1B2C8130E0322F22274B81C7
:10305000242B3093A11B2093A01B4E8150E0542FB2
:1030600044276D81462B5093A31B4093A21B5F9373
:103070004F933F932F939F938F938BE094E09F9375
:103080008F930E9460990FB6F894DEBF0FBECDBF3C
:1030900026960FB6F894DEBF0FBECDBFDF91CF915D
:1030A0001F910F910895CF92DF92EF92FF920F93AD
:1030B0001F93CF93DF93CDB7DEB72A970FB6F8945F
:1030C000DEBF0FBECDBF8E010F5F1F4F86E0F80140
:1030D00011928A95E9F741E062E08CE30E9499132E
:1030E00048E560E08CE30E94991362E174E380E0BC
:1030F00090E00E94446626E0A80163E08CE30E9411
:10310000B01343E062E08CE30E949913098110E060
:10311000102F00278A81082B10937F1B00937E1BA2
:10312000EB80F12CFE2CEE248C81E82AF092811B9E
:10313000E092801BCD80D12CDC2CCC248E81C82A3F
:10314000D092831BC092821BB801882777FD80959F
:10315000982F0E94C38F9B01AC01B701882777FD90
:103160008095982F2F83388749875A870E94C38F6D
:103170002F81388549855A850E94CD8E20EE3EE20A
:1031800045E652E40E94A59120E030E044E353E498
:103190000E945A8E9F938F937F936F93DF92CF926B
:1031A000FF92EF921F930F9389E194E09F938F9387
:1031B0000E9460990FB6F894DEBF0FBECDBF2A966D
:1031C0000FB6F894DEBF0FBECDBFDF91CF911F9138
:1031D0000F91FF90EF90DF90CF900895CF93DF9302
:1031E000EC0188819981009759F1833F914121F049
:1031F0001982188283E06FC08BE59AE00E94965D89
:10320000892B41F18091410A9091420AA091430A91
:10321000B091440A93FD20C04091410A5091420A66
:103220006091430A7091440A54FD47C04091410A9D
:103230005091420A6091430A7091440A55FD44C07E
:1032400060E870E08BE59AE00E946F5D83EF91E1AA
:103250009983888381E03FC08091CA2B82FFDCCFB5
:1032600021E048E061E083E00E946C158091B11C90
:103270008F938091B01C8F938091AF1C8F9380911E
:10328000AE1C8F938091AD1C8F938091AC1C8F935B
:103290008091AB1C8F938091AA1C8F9383E990E15E
:1032A0009F938F930E9472998DB79EB70A960FB61F
:1032B000F8949EBF0FBE8DBFAFCF8091CA2B83FF06
:1032C000B5CF0E94DB17B2CF8091CA2B84FFB8CF55
:1032D0000E945318B5CFDF91CF910895CF93C82F97
:1032E0008CEE0E94C8668C2F0E94D26665E375E062
:1032F00080E090E00E9444668DEE0E94C8660E94C5
:10330000E366C82F0E94ED662C2F30E0322F222773
:10331000A901482BCA01CF910895CF93DF93C82FFD
:103320008CEE0E94C8668C2F0E94D26662E174E324
:1033300080E090E00E9444668CEE0E94C86680E0C7
:103340000E94D26665E375E080E090E00E944466EA
:103350008DEE0E94C8660E94E366C82F0E94E36655
:10336000D82F0E94ED664D2F50E060E070E0762F80
:10337000652F542F44276C2B482BCB01BA01DF91CA
:10338000CF9108952F923F924F925F926F927F92CA
:103390008F929F92AF92BF92CF92DF92EF92FF9265
:1033A0000F931F93CF93DF93CDB7DEB7CD54D109E1
:1033B0000FB6F894DEBF0FBECDBF80910002909192
:1033C0000102892BD1F110920102109200028CEEC1
:1033D0000E94C8668EE10E94D2666BE17EE480E0C6
:1033E00090E00E94446682EA0E946E199093500A0F
:1033F00080934F0A84EA0E946E1990934E0A80933C
:103400004D0A86EA0E946E1990934C0A80934B0AEB
:1034100088EA0E946E1990934A0A8093490A8AEAC0
:103420000E946E199093480A8093470A8CEA0E9482
:103430006E199093460A8093450A88E40E948D197C
:103440006FAB78AF89AF9AAF88E50E948D194B01B9
:103450005C018091470A9091480A20E030E040E00A
:1034600050E0BA0126962FAF269727963FAF2797B1
:1034700028964FAF289729965FAF29972A966FAF66
:103480002A972B967FAF2B979C0140E050E060E09D
:1034900070E080E090E008E00E9483940E943C94F9
:1034A0003901B42FA52FF62FE72F8C019401A50128
:1034B00060E070E080E090E05301CB2EDA2EEF2E3A
:1034C000FE2E0E94BA9429833A832A011B014C01E3
:1034D000B101C401315041095F4F6F4F7F4F8F4F92
:1034E0009F4FA1E0B0E02596BFAFAEAF2597211565
:1034F0003F4F4F4F5140610571058105910509F01E
:1035000020F425961FAE1EAE259725966EAC7FAC97
:1035100025978091450A9091460A5C01C12CD12CD7
:10352000E12CF12C00E010E029813A81A201B101E7
:10353000C4010E942893D22EE32EF42E052F162FBD
:10354000B72FF82FE92FA0E00E94E19484F42150D6
:10355000310940485F4F6F4F7F4F8F4F9F4FD22EA3
:10356000E32EF42E052F162FB72FF82FE92F2D2D30
:103570003E2D4F2D502F612F7B2F8F2F9E2F07E138
:103580000E949C942B8F3C8F4D8F5E8F6F8F78A302
:1035900089A39AA32053384F4F4F5F4F6F4F7F4FF0
:1035A0008F4F9F4F2B8B3C8B4D8B5E8B6F8B788F10
:1035B000898F9A8F2056304F4F4F5F4F6F4F7F4FFD
:1035C0008F4F9F4F243D30434105510561057105E3
:1035D0008105910541F038F025966EAC7FAC2597BA
:1035E000FFEF6F1A7F0A80914D0A90914E0A9C015D
:1035F00040E050E060E070E080E090E000E10E9498
:1036000083942B833C834D835E836A8779878F8382
:1036100098874091490A50914A0AA980BA8062016C
:10362000710184019A0140E050E060E070E080E0C8
:1036300090E00E942893D22EE32EF42E052F162F11
:10364000B72FF82FE92FA0E00E94E1945CF4AFE7D8
:103650000E94C394D22EE32EF42E052F162FB72FDF
:10366000F82FE92F2D2D3E2D4F2D502F612F7B2F21
:103670008F2F9E2F07E00E949C9459016A017B01C5
:103680008C012B813C814D815E816A8579858F819A
:1036900098850E94BA942B833C834D835E836F830D
:1036A00078878F87988B2E5F3F4F434051096E4F2D
:1036B0007F4F8F4F9F4F22303105494F5F4F6440FE
:1036C00071058105910521F018F01FEF611A710A4B
:1036D00080914F0A9091500ABC0180E090E020E078
:1036E00030E840E050E00E94819329873A874B8779
:1036F0005C876A8B798B8D879E8740914B0A5091AE
:103700004C0AA980BA806201710184019A0140E0EB
:1037100050E060E070E080E090E00E942893D22EBC
:10372000E32EF42E052F162FB72FF82FE92FA0E048
:103730000E94E19484F421503F4F4F4F5F4F6F4FF1
:103740007F4F8F4F9F4FD22EE32EF42E052F162F33
:10375000B72FF82FE92F2D2D3E2D4F2D502F612FF4
:103760007B2F8F2F9E2F08E00E949C9459016A01A5
:103770007B018C0129853A854B855C856A8979892D
:103780008D859E850E94BA9429873A874B875C87EE
:103790006D877E87898B9A8B2F5F3F4F4140510900
:1037A0006109710981099109213030484C4F5F4707
:1037B000614071058105910521F018F0BFEF6B1A8A
:1037C0007B0A2B893C894D895E896F89788D898D2B
:1037D0009A8D2F3C374041055105610571058105E2
:1037E000910511F00CF0A5C1A980BA8062017101A8
:1037F00084019501A201B101C4010E942893A12C6A
:10380000B12CC12C10E8D12EE12CF12C00E010E0FD
:103810000E94AE932BAF3CAF4DAF5EAF6FAF219622
:103820007FAF219722968FAF229723969FAF239742
:10383000AB8CBC8CCD8CDE8CEF8CF8A009A11AA1CE
:103840009501A601B701C8010E94289359016A0198
:103850007B01E82F192F02E00E9483940E2F0E9413
:10386000BA9469017A01162F272EF82FE92F322EEC
:103870008D2C942EAF2CB62E072F582EB92FA0E0EA
:103880000E94E1945CF4A1E00E94C394322E832E46
:10389000942EA52EB62E072F582EB92F232D382D56
:1038A000492D5A2D6B2D702F852D9B2F01E00E94E5
:1038B0009C942E962FAF2E972D963FAF2D9749A70C
:1038C0005AA76BA77CA78DA79EA7522E432E4BA36A
:1038D0005CA36DA37EA38FA398A7B22D9601A70129
:1038E000612F722D8F2F9E2FA0E00E94E1944CF447
:1038F000A3E00E94C39469017A01162FB72FF82F15
:10390000E92F9601A701612F7B2F8F2F9E2F02E0B9
:103910000E949C942FA738AB49AB5AAB6BAB7CABE6
:103920008DAB9EAB19014A01B62FA72F24968FAFFE
:103930002497F92F2B893C894D895E896F89788D71
:10394000898D9A8D24323A4F4F4F5F4F6F4F7F4F83
:103950008F4F9F4F0CF08CC02B8D3C8D4D8D5E8D0D
:103960006F8D78A189A19AA12455324F4F4F5F4F97
:103970006F4F7F4F8F4F9F4F59016A017B018C0121
:103980000E94289319014A01B62FA72FFC0103E0DA
:103990000E94839451016401EB2EFA2E8F010E9444
:1039A000CF9459016A017B018C012E962FAD2E9781
:1039B0002D963FAD2D9749A55AA56BA57CA58DA544
:1039C0009EA50E94BA94522E432E4BA35CA36DA3D6
:1039D0007EA38FA398A79101A4016B2F7A2FCF010B
:1039E00002E00E94839451016401EB2EFA2E8F01B4
:1039F0000E94CF9402E00E9483940E2F0E94CF94E5
:103A0000F22E032F142FD52EE62EB72FF82FE92FE5
:103A1000A0E00E94E1945CF4A1E00E94C394F22E25
:103A2000032F142FD52EE62EB72FF82FE92F2F2D89
:103A3000302F412F5D2D6E2D7B2F8F2F9E2F01E07C
:103A40000E949C9459016A017B018C012FA538A921
:103A500049A95AA96BA97CA98DA99EA90E94BA94CB
:103A600019014A01B62FA72F24968FAF2497F92F5B
:103A70002B813C814D815E816F8178858F8598890E
:103A8000A52CB42CCBA0DCA0EDA0FEA00FA118A506
:103A90000E94CF942B833C834D835E836F83788712
:103AA0008F87988B29853A854B855C856D857E85CA
:103AB00089899A8951016401EB2EFA2E24960FAD63
:103AC00024971F2F0E94CF9429873A874B875C87C2
:103AD0006D877E87898B9A8B2B893C894D895E897E
:103AE0006F89788D898D9A8DABACBCACCDACDEACDA
:103AF000EFAC2196FFAC219722960FAD229723962B
:103B00001FAD23970E94CF942056304F4F4F5F4FE9
:103B10006F4F7F4F8F4F9F4F243D304341055105DD
:103B2000610571058105910521F018F02FEF621AEA
:103B3000720A6FA978AD89AD9AADAB01BC0180E086
:103B400090E0DC0124964FAF249725965FAF259730
:103B500026966FAF269727967FAF279728968FAF29
:103B6000289729969FAF29972A96AFAF2A972B9629
:103B7000BFAF2B97A984BA84CB84DC84ED84FE8408
:103B800009891A899A01AB0160E070E080E090E059
:103B90000E942893F22E032F142FD52EE62EB72F36
:103BA000F82FE92FA0E00E94E19484F4215031091C
:103BB000404E5F4F6F4F7F4F8F4F9F4FF22E032F1F
:103BC000142FD52EE62EB72FF82FE92F2F2D302FBB
:103BD000412F5D2D6E2D7B2F8F2F9E2F05E10E9493
:103BE0009C94AB80BC80CD80DE80EF80F8840F8514
:103BF00018890E94CF94F22E032F142FD52EE62E73
:103C0000B72FF82FE92FA0E00E94E19484F421500F
:103C100030484F4F5F4F6F4F7F4F8F4F9F4FF22E68
:103C2000032F142FD52EE62EB72FF82FE92F2F2D87
:103C3000302F412F5D2D6E2D7B2F8F2F9E2F0FE06C
:103C40000E949C9469017A018B018A8399832901DE
:103C50001A014B015C01285E334041095109610999
:103C6000710981099109283D304D41405105610597
:103C700071058105910521F018F0BFEF6B1A7B0AE1
:103C80000E94CA66672859F09601A701B8018A8187
:103C900099810E943C9429011A014B015C01920117
:103CA000A101B401C5010E94BD8F20E030E048ECC5
:103CB00052E40E94248FC35BDF4F0FB6F894DEBF3F
:103CC0000FBECDBFDF91CF911F910F91FF90EF906D
:103CD000DF90CF90BF90AF909F908F907F906F902C
:103CE0005F904F903F902F9008954F925F926F9208
:103CF0007F928F929F92AF92BF92CF92DF92EF927C
:103D0000FF922B013C0169017A0123EC35EF4CE86D
:103D100051E4C701B6010E94A5914B015C0128EB5B
:103D20003EE143E753E4C701B6010E945A8E9B016E
:103D3000AC01C501B4010E94248F0E94918F4B01F8
:103D40005C0120E030E048EC52E4C301B2010E9483
:103D5000248F21E835E943EC50E40E94A591A501A8
:103D600094010E94A5914B015C0123E333E948E8EB
:103D700053E4C701B6010E945A8E9B01AC01C501F4
:103D8000B4010E94248F23E333EB48E553E40E94FF
:103D9000A591FF90EF90DF90CF90BF90AF909F9054
:103DA0008F907F906F905F904F9008954F925F92A9
:103DB0006F927F928F929F92AF92BF92CF92DF923B
:103DC000EF92FF9269017A010E94279120E030E092
:103DD00040E050E40E94598E22E93CE54EED5EE35E
:103DE0000E94248F4B015C0123EC35EF4CE851E439
:103DF000C701B6010E94A5912B013C0128EB3EE1D1
:103E000043E753E4C701B6010E945A8E9B01AC01FF
:103E1000C301B2010E94248F9B01AC01C501B40112
:103E20000E945A8E6B017C0128EB3EE143E753E48C
:103E30000E94A5914B015C01A701960163EC75EF0F
:103E40008CE891E40E94598E9B01AC01C501B4013C
:103E50000E94248FFF90EF90DF90CF90BF90AF90A3
:103E60009F908F907F906F905F904F9008954F92AA
:103E70005F926F927F928F929F92AF92BF92CF92FA
:103E8000DF92EF92FF922B013C0169017A0123EC52
:103E900035EF4CE851E4C701B6010E94A5914B01F2
:103EA0005C0128EB3EE143E753E4C701B6010E9401
:103EB0005A8E9B01AC01C501B4010E94248F0E945F
:103EC000918F4B015C0120E030E048EC52E4C301EB
:103ED000B2010E94248FA50194010E94A59120E0C7
:103EE00030E040E251E40E94598E24EE38E34EE087
:103EF0005FE30E94A5919B01AC01C701B6010E943E
:103F00005A8EFF90EF90DF90CF90BF90AF909F9030
:103F10008F907F906F905F904F90089580E80E94FF
:103F2000C86681110DC08EEF0E94D266811108C053
:103F30006BE17EE480E090E00E9444660C94CA66E7
:103F40000E94CA668091DC2F9091DD2FA091DE2F18
:103F5000B091DF2F0196A11DB11D8093DC2F9093AE
:103F6000DD2FA093DE2FB093DF2F0895FC01DC013D
:103F700082E020E041E39D91292798E0322F330F22
:103F800027FF03C0232F242701C0232F9150B1F70F
:103F9000815089F781E090E03281231711F080E0B1
:103FA00090E00895DF92EF92FF920F931F93CF93CB
:103FB000DF930E948E1F80E80E94C86681116DC049
:103FC0008AEF0E94D266811168C08FE00E94D2669B
:103FD000811163C065E375E080E090E00E94446673
:103FE00081E80E94C866811158C00E94E366C82F0C
:103FF0000E94E3660E94E366D82F0E94E3660E9457
:10400000E366182F0E94E3660E94ED66082F80E8A1
:104010000E94C866811141C08CEF0E94D266811156
:104020003CC089EC0E94D266811137C065E375E01F
:1040300080E090E00E94446681E80E94C8660E9489
:10404000E366E82E0E94E366D82E0E94E3660E9493
:10405000E366F82E0E94ED661F92DF921F92EF92A8
:104060001F920F931F921F931F92DF931F92CF9364
:104070001F928F931F92FF928EE294E09F938F93F3
:104080000E9460990E94CA668DB79EB742960FB68D
:10409000F8949EBF0FBE8DBF17C00E94CA66809164
:1040A000DC2F9091DD2FA091DE2FB091DF2F0196B4
:1040B000A11DB11D8093DC2F9093DD2FA093DE2FE7
:1040C000B093DF2F0E948E1F20E030E040E050E0F0
:1040D00060E070E080E090E0DF91CF911F910F9160
:1040E000FF90EF90DF900895EF92FF920F931F9350
:1040F000CF93DF9300D01F92CDB7DEB78C0180E85D
:104100000E94C866811154C00115110551F085EE59
:104110000E94D26681114CC061E077E980E090E0B6
:1041200009C083EE0E94D266811142C069E97AEB30
:1041300081E090E00E94446681E80E94C866811197
:1041400037C00E94E366F82E89830E94E366E82E5A
:104150008A830E94ED668B830E94CA66CE01019617
:104160000E94B61F892B21F16E2D70E07F296C7F94
:1041700080E090E0012B69F00E94C18F20E030E0E8
:104180004AEF5AE30E94A59120E030E040EC50E471
:104190000CC00E94C18F22E538EB4FE25BE30E9426
:1041A000A59126E636E64BE352E40E94598E1BC0E9
:1041B0000E94CA668091DC2F9091DD2FA091DE2FA6
:1041C000B091DF2F0196A11DB11D8093DC2F90933C
:1041D000DD2FA093DE2FB093DF2F0E948E1F60EFA4
:1041E0007FEF89E794E40F900F900F90DF91CF91CC
:1041F0001F910F91FF90EF9008950F931F93CF930E
:10420000DF93729A8091660283FF08C08EE40E9459
:104210006666811167C0C0E5D0E00AC0C0E5D0E0A5
:1042200087EE93E00E94290A21972097C9F7EECFE5
:1042300087EE93E00E94290A21972097C9F78FE41F
:104240000E9466660E94E366082F0F730E94E36671
:10425000182F0E94E366D82F0E94ED66C82F0E9497
:10426000CA668091660283FF7298602F70E0762F95
:104270006627610F711D80E090E00E94C18F20E1F0
:1042800034E048EC5BE30E94A5916093BE277093F5
:10429000BF278093C0279093C1276D2F70E0762FA2
:1042A00066276C0F711D769567957695679580E00A
:1042B00090E00E94C18F24EA3CEF44E25CE30E945C
:1042C000A59120E030E040E252E40E94598E6093D4
:1042D0009F347093A0348093A1349093A23480E0F3
:1042E00090E002C081E090E0DF91CF911F910F91AB
:1042F00008957298729A8EE40E94666680EA0E941F
:10430000D26680E00E94D26680E00E94D2668FE48E
:104310000E9466660E94E3668EE40E94666680E8FC
:104320000E94D26680E00E94D26680E00E94D2663F
:104330000E94CA6680E090E0089582EC9FE09F931F
:104340008F930E947299809181020F900F90882321
:1043500061F01F928F938FEB9FE09F938F930E944A
:1043600072990F900F900F900F9008958AE99FE037
:104370009F938F930E94729982E79FE09F938F9300
:104380000E9472998BE49FE09F938F930E94729991
:1043900080E19FE09F938F930E94729984ED9EE04D
:1043A0009F938F930E94729982EA9EE09F938F93CE
:1043B0000E94729986E69EE09F938F930E94729965
:1043C00080E49EE09F938F930E9472998AE09EE022
:1043D0009F938F930E9472998091CA2B9091CB2BBF
:1043E000827091702DB73EB72E5E3F4F0FB6F89496
:1043F0003EBF0FBE2DBF892B41F08AED9DE09F93FC
:104400008F930E9472990F900F908EEA9DE09F9378
:104410008F930E94729982E79DE09F938F930E94F1
:10442000729989E49DE09F938F930E9472998DE128
:104430009DE09F938F930E9472998EEE9CE09F93D4
:104440008F930E9472998CEB9CE09F938F930E94B4
:1044500072998BE89CE09F938F930E94729981E5FB
:104460009CE09F938F930E9472998BE19CE09F93B5
:104470008F930E9472998BEE9BE09F938F930E9483
:1044800072998FEB9BE09F938F930E94729980E9C2
:104490009BE09F938F930E94729987E59BE09F9387
:1044A0008F930E9472998EE19BE09F938F930E945D
:1044B000729987EE9AE09F938F930E94729989EB8D
:1044C0009AE09F938F930E9472998DB79EB78096C2
:1044D0000FB6F8949EBF0FBE8DBF85E89AE09F93FC
:1044E0008F930E94729984E59AE09F938F930E9424
:1044F000729985E29AE09F938F930E94729986EF5A
:1045000099E09F938F930E9472998FEC99E09F930B
:104510008F930E94729989E999E09F938F930E94EB
:10452000729983E699E09F938F930E9472998DE22E
:1045300099E09F938F930E94729984E099E09F93F2
:104540008F930E9472998CEC98E09F938F930E94B6
:10455000729981EA98E09F938F930E9472992DB788
:104560003EB72A5E3F4F0FB6F8943EBF0FBE2DBF39
:1045700008958DE594E00C9496994F925F926F9216
:104580007F928F929F92AF92BF92CF92DF92EF92E3
:10459000FF92CF93DF93CDB7DEB728970FB6F8948D
:1045A000DEBF0FBECDBF8091D02F9091D12FA091B3
:1045B000D22FB091D32F89839A83AB83BC83409051
:1045C000D02F5090D12F6090D22F7090D32F809108
:1045D000D02F9091D12FA091D22FB091D32F8D8336
:1045E0009E83AF83B8876091D02F7091D12F809137
:1045F000D22F9091D32F2CE3822E912CA12CB12C71
:10460000A50194010E94A9927F936F9330E1C32E7C
:104610003EE0D32EE12CF12C6D817E818F81988537
:10462000A70196010E94A992A50194010E94A99256
:104630003F932F9340E8842E41E5942EAA24A3941F
:10464000B12CC301B201A50194010E94A992A70156
:1046500096010E94A9923F932F9369817A818B8161
:104660009C81A50194010E94A9923F932F938BE70F
:1046700098E09F938F930E9472990FB6F894DEBFD3
:104680000FBECDBF28960FB6F894DEBF0FBECDBFCC
:10469000DF91CF91FF90EF90DF90CF90BF90AF90E0
:1046A0009F908F907F906F905F904F900895E4E679
:1046B000FDE3808191818234924479F0E456FD4398
:1046C000FF93EF938DE598E09F938F930E947299EB
:1046D0000F900F900F900F9008953A96E53F81E468
:1046E000F80738F30895CF93DF93EC018C9A0E947A
:1046F000A50C9F938F937F936F9381E598E09F9391
:104700008F930E9472990F900F900F900F900F90BF
:104710000F90209719F00E94C00D08C08FE498E018
:104720009F938F930E9472990F900F9081E00E9447
:10473000560C209186023091870240918802509158
:1047400089020E94A5919F938F937F936F9383E437
:1047500098E09F938F930E9472990F900F900F9003
:104760000F900F900F90209719F00E94C00D08C075
:1047700081E498E09F938F930E9472990F900F901D
:1047800082E00E94560C2091820230918302409177
:104790008402509185020E94A5919F938F937F93ED
:1047A0006F9385E398E09F938F930E9472990F9087
:1047B0000F900F900F900F900F90209719F00E947C
:1047C000C00D08C083E398E09F938F930E94729975
:1047D0000F900F9083E00E94560C9F938F937F93CE
:1047E0006F9384E298E09F938F930E9472998C98C4
:1047F0000F900F900F900F900F900F90209719F03F
:104800000E94C00D08C082E298E09F938F930E949F
:1048100072990F900F908091CA2B87FF83C021E07F
:1048200042E161E080ED0E942A689F938F937F931D
:104830006F9385E198E09F938F930E9472990F90F8
:104840000F900F900F900F900F90209719F00E94EB
:10485000C00D08C083E198E09F938F930E947299E6
:104860000F900F9021E042E162E080ED0E942A6803
:104870009F938F937F936F9386E098E09F938F939E
:104880000E9472990F900F900F900F900F900F90C1
:10489000209719F00E94C00D08C084E098E09F9313
:1048A0008F930E9472990F900F9021E042E163E094
:1048B00080ED0E942A689F938F937F936F9387EF79
:1048C00097E09F938F930E9472990F900F900F9093
:1048D0000F900F900F90CD2B19F00E94C00D08C0C3
:1048E00085EF97E09F938F930E9472990F900F909E
:1048F00021E042E164E080ED0E942A689F938F935B
:104900007F936F9388EE97E09F938F930E947299A5
:104910000F900F900F900F900F900F90DF91CF910D
:104920000C94C00DCD2BD1F3DF91CF9108950F934F
:104930001F93CF93DF93882389F049E050E06FEF16
:1049400070E083E994E30E94B49849E050E06EE09F
:1049500070E083E994E30E94E49A13C0C3E9D4E3CE
:1049600003EE17E089911F928F931F930F930E947C
:1049700072990F900F900F900F9084E3CB39D80766
:1049800089F7DF91CF911F910F910C94C00D88236F
:1049900011F0299A089529980895882311F02A9AE8
:1049A00008952A980895882311F02B9A08952B983A
:1049B0000895CF92DF92EF92FF92CF93DF936B0136
:1049C0007C0160FF11C08AE994E09F938F9387ED8B
:1049D0009FE09F938F930E9472990F900F900F907A
:1049E0000F9081E090E002C080E090E0C1FE09C03D
:1049F000EC0121964FE959E06FE974E00E9425121D
:104A0000CE01C2FE09C0EC0121964FE959E067EAE8
:104A100074E00E942512CE01C3FE09C0EC0121966C
:104A20004FE959E06FEA74E00E942512CE01C4FEFE
:104A300009C0EC0121964FE959E06AE176E00E9455
:104A40002512CE01C5FE09C0EC0121964FE959E0BF
:104A500063EB74E00E942512CE01C6FE09C0EC0192
:104A600021964FE959E067EB74E00E942512CE01D0
:104A7000C7FE09C0EC0121964FE959E06DEB74E0E7
:104A80000E942512CE01D0FE09C0EC0121964FE90B
:104A900059E065EC74E00E942512CE01D1FE09C0F8
:104AA000EC0121964FE959E06DEC74E00E9425126B
:104AB000CE01D2FE09C0EC0121964FE959E061ED2B
:104AC00074E00E942512CE012091CA2B3091CB2B8D
:104AD00024703270232B59F0D3FE09C0EC012196CB
:104AE0004FE959E067ED74E00E942512CE01209154
:104AF000CA2B23FF0BC0D4FE09C0EC0121964FE95D
:104B000059E06CED74E00E942512CE012091CA2B71
:104B100024FF0BC0D5FE09C0EC0121964FE959E0F6
:104B200062EE74E00E942512CE01D6FE09C0EC01AF
:104B300021964FE959E06AEE74E00E942512CE01F9
:104B4000D7FE09C0EC0121964FE959E065EF74E00A
:104B50000E942512CE01E0FE0CC04FE959E066E04C
:104B600075E0DF91CF91FF90EF90DF90CF900C94A4
:104B70002512CD28CE28CF2841F48EED97E09F93C3
:104B80008F930E9472990F900F90DF91CF91FF90B9
:104B9000EF90DF90CF900895CF92DF92EF92FF9247
:104BA000CF93DF93EC01C12CD12C7601209709F42F
:104BB000A3C069ED77E0CE010E949398892B11F490
:104BC0006894C0F861ED77E0CE010E949398892B3C
:104BD00011F46894C1F869EC77E0CE010E949398D3
:104BE000892B11F46894C2F865EC77E0CE010E943D
:104BF0009398892B11F46894C3F862EC77E0CE01A6
:104C00000E949398892B11F46894C4F86EEB77E0B6
:104C1000CE010E949398892B11F46894C5F868EB33
:104C200077E0CE010E949398892B11F46894C6F81E
:104C300060EB77E0CE010E949398892B11F4689481
:104C4000C7F868EA77E0CE010E949398892B11F4A7
:104C50006894D0F864EA77E0CE010E949398892B9B
:104C600011F46894D1F86EE977E0CE010E94939830
:104C7000892B11F46894D2F869E977E0CE010E949B
:104C80009398892B11F46894D3F863E977E0CE0107
:104C90000E949398892B11F46894D4F86BE877E01C
:104CA000CE010E949398892B11F46894D5F860E89E
:104CB00077E0CE010E949398892B11F46894D6F87E
:104CC0006FE677E0CE010E949398892B11F46894E7
:104CD000D7F86AE677E0CE010E949398892B11F409
:104CE0006894E0F860917F027091800280E090E02B
:104CF0000E94A798EC015ACFC701B601DF91CF916E
:104D0000FF90EF90DF90CF900895AF92BF92CF9237
:104D1000DF92EF92FF920F931F93CF93DF93F22EC8
:104D2000032F142FE52ED62EA72EB82EC92E2170B4
:104D300030E040E050E060E070E080E090E0A0E033
:104D40000E94E19489F0EBE0F5E0FF93EF93E7ED4B
:104D5000FFE0FF93EF930E9472990F900F900F90D6
:104D60000F90E1E0F0E002C0E0E0F0E08091CA2BBB
:104D700080FF17C02F2D247030E040E050E060E04D
:104D800070E080E090E0A0E00E94E19451F0EF013B
:104D900021964FE959E06FE075E0CF010E9425129E
:104DA000FE012F2D227030E040E050E060E070E026
:104DB00080E090E0A0E00E94E19451F0EF012196A4
:104DC0004FE959E063E175E0CF010E942512FE0131
:104DD0002F2D287030E040E050E060E070E080E08F
:104DE00090E0A0E00E94E19451F0EF0121964FE99C
:104DF00059E06BE275E0CF010E942512FE012F2DD4
:104E0000207130E040E050E060E070E080E090E051
:104E1000A0E00E94E19451F0EF0121964FE959E0A2
:104E200066E175E0CF010E942512FE012F2D207250
:104E300030E040E050E060E070E080E090E0A0E032
:104E40000E94E19451F0EF0121964FE959E069E1A8
:104E500075E0CF010E942512FE012F2D207430E055
:104E600040E050E060E070E080E090E0A0E00E9470
:104E7000E19451F0EF0121964FE959E06FE175E0BF
:104E8000CF010E942512FE012F2D207830E040E056
:104E900050E060E070E080E090E0A0E00E94E194EB
:104EA00051F0EF0121964FE959E065E275E0CF013D
:104EB0000E942512FE0120E0302F317040E050E0CA
:104EC00060E070E080E090E0A0E00E94E19451F0AA
:104ED000EF0121964FE959E068E275E0CF010E94A9
:104EE0002512FE0120E0302F327040E050E060E0FB
:104EF00070E080E090E0A0E00E94E19451F0EF01CA
:104F000021964FE959E06DE275E0CF010E9425122C
:104F1000FE0120E0302F347040E050E060E070E0AF
:104F200080E090E0A0E00E94E19451F0EF01219632
:104F30004FE959E064E375E0CF010E942512FE01BC
:104F400020E0302F387040E050E060E070E080E01A
:104F500090E0A0E00E94E19451F0EF0121964FE92A
:104F600059E067E375E0CF010E942512FE0120E0C1
:104F7000302F307140E050E060E070E080E090E081
:104F8000A0E00E94E19451F0EF0121964FE959E031
:104F90006CE375E0CF010E942512FE0120E0302F66
:104FA000307240E050E060E070E080E090E0A0E02F
:104FB0000E94E19451F0EF0121964FE959E063E43A
:104FC00075E0CF010E942512FE0120E030E040E0B4
:104FD00050E06D2D647070E080E090E0A0E00E94F1
:104FE000E19451F0EF0121964FE959E06AE475E050
:104FF000CF010E942512FE018091CA2B81FF17C0AC
:1050000020E0302F307440E050E060E070E080E05D
:1050100090E0A0E00E94E19451F0EF0121964FE969
:1050200059E06EE475E0CF010E942512FE018091E7
:10503000CA2B9091CB2B90FF17C020E030E040E0CE
:105040005E2D507160E070E080E090E0A0E00E9492
:10505000E19451F0EF0121964FE959E061E575E0E7
:10506000CF010E942512FE018091CA2B9091CB2B7B
:1050700090FF17C020E030E040E05E2D507260E00D
:1050800070E080E090E0A0E00E94E19451F0EF0138
:1050900021964FE959E064E575E0CF010E942512A1
:1050A000FE018091CA2B9091CB2B90FF17C020E07E
:1050B00030E040E05E2D507460E070E080E090E011
:1050C000A0E00E94E19451F0EF0121964FE959E0F0
:1050D0006AE575E0CF010E942512FE0120E0302F25
:1050E000307840E050E060E070E080E090E0A0E0E8
:1050F0000E94E19451F0EF0121964FE959E065E6F5
:1051000075E0CF010E942512FE0120E030E0412F22
:10511000417050E060E070E080E090E0A0E00E942C
:10512000E19451F0EF0121964FE959E06AE675E00C
:10513000CF010E942512FE0120E030E0412F427095
:1051400050E060E070E080E090E0A0E00E94E19438
:1051500051F0EF0121964FE959E06DE675E0CF017E
:105160000E942512FE0120E030E0412F447050E003
:1051700060E070E080E090E0A0E00E94E19451F0F7
:10518000EF0121964FE959E060E775E0CF010E94F9
:105190002512FE018091CA2B87FF17C020E030E066
:1051A000412F487050E060E070E080E090E0A0E0C7
:1051B0000E94E19451F0EF0121964FE959E063E735
:1051C00075E0CF010E942512FE018091CA2B87FF56
:1051D00017C020E030E0412F407150E060E070E007
:1051E00080E090E0A0E00E94E19451F0EF01219670
:1051F0004FE959E067E775E0CF010E942512FE01F3
:105200008091CA2B87FF17C020E030E0412F407209
:1052100050E060E070E080E090E0A0E00E94E19467
:1052200051F0EF0121964FE959E06BE775E0CF01AE
:105230000E942512FE018091CA2B87FF17C020E033
:1052400030E0412F407450E060E070E080E090E09A
:10525000A0E00E94E19451F0EF0121964FE959E05E
:105260006FE775E0CF010E942512FE018091CA2BE5
:1052700082FF17C020E030E0412F407850E060E02E
:1052800070E080E090E0A0E00E94E19451F0EF0136
:1052900021964FE959E06DEA76E0CF010E94251290
:1052A000FE018091CA2B82FF17C020E030E040E071
:1052B0005E2D517060E070E080E090E0A0E00E9420
:1052C000E19451F0EF0121964FE959E063E875E070
:1052D000CF010E942512FE018091CA2B9091CB2B09
:1052E00090FF17C020E030E040E05E2D527060E09B
:1052F00070E080E090E0A0E00E94E19451F0EF01C6
:1053000021964FE959E066E875E0CF010E94251229
:10531000FE018091CA2B9091CB2B90FF17C020E00B
:1053200030E040E05E2D547060E070E080E090E09E
:10533000A0E00E94E19451F0EF0121964FE959E07D
:105340006EE875E0CF010E942512FE018091CA2B04
:105350009091CB2B91FF1EC020E030E040E05E2D0D
:10536000587060E070E080E090E0A0E00E94E1947E
:1053700089F04FE959E067E975E0CF01DF91CF91FE
:105380001F910F91FF90EF90DF90CF90BF90AF9063
:105390000C9425122F2D302F412F5E2D6D2D7A2D3F
:1053A0008B2D9C2DA0E00E94E19441F485E697E0CE
:1053B0009F938F930E9472990F900F90DF91CF91DE
:1053C0001F910F91FF90EF90DF90CF90BF90AF9023
:1053D00008958F929F92BF92DF92EF920F931F9347
:1053E000CF93DF93EC014B01FB01108260E677E085
:1053F0000E949398892B61F58091CA2B7DE4D72E6A
:10540000E0E8EE2E82FD02C004E001C004E810E0F6
:10541000B12C81FF02C060ECE62E26E04AE250E0AB
:105420006BE270E089E290E00E946B6381E090E0C3
:105430000E944E0D882311F05DE5D52E8091CA2B78
:105440009091CB2B90FD16E091FF07C0186005C02E
:10545000D12CE12C00E010E0B12C6EE577E0CE011C
:105460000E949398892B61F481E0F401808360911C
:105470007F027091800280E090E00E94A798EC018A
:105480006CE577E0CE010E949398892B61F48FEF51
:10549000F401808360917F027091800280E090E04F
:1054A0000E94A798EC01209709F424C168E577E0F1
:1054B000CE010E949398892B19F4FD2DF160DF2E07
:1054C00064E577E0CE010E949398892B19F48D2D25
:1054D0008460D82E61E577E0CE010E949398892BF5
:1054E00019F4ED2DE260DE2E6FE477E0CE010E942C
:1054F0009398892B19F4FD2DF860DF2E6CE477E08A
:10550000CE010E949398892B19F48D2D8061D82E9D
:1055100066E477E0CE010E949398892B19F4ED2D73
:10552000E062DE2E60E477E0CE010E949398892B42
:1055300019F4FD2DF064DF2E6DE377E0CE010E94BB
:105540009398892B19F48D2D8068D82E68E377E025
:10555000CE010E949398892B19F4EE2DE160EE2E76
:1055600061E377E0CE010E949398892B19F4FE2D18
:10557000F260EF2E6EE277E0CE010E949398892BC5
:1055800019F48E2D8460E82E69E277E0CE010E9446
:105590009398892B19F4EE2DE860EE2E62E277E005
:1055A000CE010E949398892B19F4FE2DF061EF2E05
:1055B0006BE177E0CE010E949398892B19F48E2D30
:1055C0008062E82E67E177E0CE010E949398892BF4
:1055D00019F4EB2DE460BE2E64E177E0CE010E9469
:1055E0009398892B19F4FE2DF064EF2E6FE077E08D
:1055F000CE010E949398892B19F48E2D8068E82E95
:105600006CE077E0CE010E949398892B09F4016049
:1056100069E077E0CE010E949398892B09F402603B
:1056200066E077E0CE010E949398892B09F404602C
:1056300062E077E0CE010E949398892B09F408601C
:105640006EEF76E0CE010E949398892B09F40061F9
:105650006AEF76E0CE010E949398892B09F40062EC
:1056600066EF76E0CE010E949398892B09F40064DE
:1056700064EF76E0CE010E949398892B09F40068CC
:1056800061EF76E0CE010E949398892B09F41160B6
:1056900069EE76E0CE010E949398892B09F412609E
:1056A00060EE76E0CE010E949398892B09F4146095
:1056B00067ED76E0CE010E949398892B09F418607B
:1056C00064ED76E0CE010E949398892B09F4106175
:1056D0006EEC76E0CE010E949398892B09F410625B
:1056E00063EC76E0CE010E949398892B09F0D2CE2C
:1056F0001064D0CE2D2D3E2DA8016B2D70E080E0E2
:1057000090E0DF91CF911F910F91EF90DF90BF90CC
:105710009F908F9008955F926F927F928F929F9249
:10572000AF92BF92CF92DF92EF92FF920F931F93AF
:10573000CF93DF93782ECDEADBE100E010E0FDEBC4
:10574000EF2EF6E0FF2E8170582E872D8270682E86
:10575000A8EACA2EA6E0DA2EB0EBAB2EB6E0BB2E3E
:105760008EEA882E86E0982E772051F01F930F93B3
:10577000FF92EF920E9472990F900F900F900F90EE
:105780005520A1F089858F9388858F93BF92AF9222
:105790000E9472990F900F900F900F906620C1F0A9
:1057A0009F928F920E9472990F900F90662081F0C5
:1057B000DF92CF920E947299288139814A815B8160
:1057C0006C817D818E819F810E9485260F900F9034
:1057D0000E94C00D0F5F1F4F2A960430110521F65D
:1057E000DF91CF911F910F91FF90EF90DF90CF90BD
:1057F000BF90AF909F908F907F906F905F90089533
:1058000083EA96E09F938F930E9472998091BA27C2
:105810009091BB27A091BC27B091BD270F900F900E
:10582000813027EA92072EE1A207B10519F485E934
:1058300096E01DC0823026EA92072EE1A207B1054C
:1058400019F488E896E013C0823027EA92072EE127
:10585000A207B10519F48AE796E009C0823028EA68
:1058600092072EE1A207B10549F48CE696E09F93DA
:105870008F930E9472990F900F900895BF93AF93EA
:105880009F938F9386E696E09F938F930E947299E1
:105890000F900F900F900F900F900F90089586E546
:1058A00096E09F938F930E9472990E94B9220E9462
:1058B000002C0E94C00D84E99BE19F938F938EE49E
:1058C00096E09F938F930E9472996091600270910D
:1058D0006102809162029091630228EE33E040E021
:1058E00050E00E94A9925F934F933F932F938EE3D2
:1058F00096E09F938F930E94729985E396E09F9321
:105900008F930E9472990E944D128091CA2B2DB7DD
:105910003EB7225F3F4F0FB6F8943EBF0FBE2DBF7C
:1059200080FF05C041E061E081E00E94F71381E360
:1059300096E09F938F930E94729980E00E94972433
:105940000E94BD22809165021F928F9388E296E0AB
:105950009F938F930E94729980913D0A1F928F931B
:105960008FE196E09F938F930E94729980919102AC
:105970008F93809190028F9380918F028F9380916B
:105980008E028F9381E196E09F938F930E9472998C
:105990001F9280E48F9389EF95E09F938F930E94ED
:1059A00072998091A4341F928F938091A3341F9297
:1059B0008F9386EE95E09F938F930E9472998091CA
:1059C00064021F928F938DED95E09F938F930E94B9
:1059D00072998091660290916702A0916802B091DD
:1059E00069022DB73EB7225E3F4F0FB6F8943EBF17
:1059F0000FBE2DBF96FF03C080EA95E002C083EA88
:105A000095E09F938F9383ED95E09F938F930E94F2
:105A1000729983E00E948B2B0F900F900F900F9044
:105A20001D9B03C080EA95E002C083EA95E09F9346
:105A30008F9387EC95E09F938F930E9472998DEBE3
:105A400095E09F938F930E947299809166020F90C8
:105A50000F900F900F900F900F9081FF09C087EB70
:105A600095E09F938F930E9472990F900F9013C0AF
:105A700080FF03C080EA95E002C083EA95E09F932F
:105A80008F9383EB95E09F938F930E9472990F9071
:105A90000F900F900F908091660290916702A091F5
:105AA0006802B091690297FF03C080EA95E002C0E6
:105AB00083EA95E09F938F938AEA95E09F938F9373
:105AC0000E94729983EA95E09F938F930E94729946
:105AD0006091410A7091420A8091430A9091440A70
:105AE0000E94D9240E94C00D0F900F900F900F902C
:105AF0000F900F90779903C080EA95E002C083EA87
:105B000095E09F938F938AE995E09F938F930E94EE
:105B100072990E942F0A0E940A0D9F938F937F9380
:105B20006F938CE895E09F938F930E9472990E94E7
:105B3000B90C9F938F937F936F938EE795E09F931C
:105B40008F930E94729981E090E00E94732380916C
:105B5000793490917A34A0917B34B0917C34BF93A6
:105B6000AF939F938F9380E795E09F938F930E94CD
:105B7000729980918E348F9380918D348F93809120
:105B80008C348F9380918B348F938CE595E09F9329
:105B90008F930E94729980917D3490917E34A09170
:105BA0007F34B0918034BF93AF939F938F938EE4F3
:105BB00095E09F938F930E9472998DB79EB78296BE
:105BC0000FB6F8949EBF0FBE8DBF809192348F9315
:105BD000809191348F93809190348F9380918F3402
:105BE0008F938AE395E09F938F930E94729961E06F
:105BF00070E080E090E00E94C90D61E070E081E01B
:105C000090E00E94C90D0F900F900F900F900F9091
:105C10000F90299B03C080EA95E002C083EA95E0DB
:105C20009F938F9382E395E09F938F930E94729945
:105C30000F900F900F900F902A9B03C080EA95E081
:105C400002C083EA95E09F938F938AE295E09F9349
:105C50008F930E9472990F900F900F900F9008955C
:105C6000F894E0E0F0E081E2809357008491E2E074
:105C7000F0E041E2409357004491E4E0F0E091E22B
:105C800090935700E49190E0A0E0B0E0DC01992708
:105C9000882750E060E070E0762F652F542F44276E
:105CA000840F951FA61FB71F8E0F911DA11DB11D3B
:105CB0008093BA279093BB27A093BC27B093BD27AE
:105CC00078940895CF93DF93CDB7DEB761970FB681
:105CD000F894DEBF0FBECDBF48E250E062E270E054
:105CE0008DEA9BE10E94C69A2091AD1B3091AE1BBC
:105CF0004091AF1B5091B01B6091B11B7091B21BD2
:105D00008091B31B9091B41BAFEF0E94E19409F016
:105D10005DC08DE48093AD1B80E88093AE1B84E072
:105D20008093AF1B1092B01B1092B11B1092B21B4C
:105D30001092B31B1092B41B8CE390E09093B61BAF
:105D40008093B51B1092B71B1092B81B1092B91B11
:105D50001092BA1B1092BB1B1092BC1B1092BD1B61
:105D60001092BE1B1092C01B1092BF1B1092C11B41
:105D70001092C21B1092C31B1092C41B1092C51B21
:105D80001092C61B1092C71B1092C81B1092CA1B00
:105D90001092C91B1092CB1B1092CC1B1092CD1BE2
:105DA0001092CE1B1092CF1B1092D01B1092D11BC1
:105DB0001092D21B1092D41B1092D31B48E250E0D9
:105DC00062E270E08DEA9BE10E94E49A44E050E0D8
:105DD0006EE170E0CE010B960E94C69A8B859C8581
:105DE000AD85BE858F3F2FEF9207A207B207A9F4BA
:105DF0008AE090E4A0E0B0E08093660290936702AE
:105E0000A0936802B093690244E050E06EE170E054
:105E100086E692E00E94E49A08C08093660290931E
:105E20006702A0936802B093690280916602909124
:105E30006702A0916802B0916902A2FF02C02A9A8B
:105E400003C080E00E94CD2444E050E06AE570E0A9
:105E5000CE010B960E94C69A8B859C85AD85BE852A
:105E60008F3F2FEF9207A207B20789F41092410AE1
:105E70001092420A1092430A1092440A44E050E001
:105E80006AE570E081E49AE00E94E49A08C0809399
:105E9000410A9093420AA093430AB093440A49E00E
:105EA00050E06EE070E083E994E30E94C69A0E949D
:105EB000010F44E050E06EE470E0CE010B960E94CA
:105EC000C69A8B859C85AD85BE8544E050E06EE426
:105ED00070E08F3F9F4FAF4FBF4F29F486E892E0AD
:105EE0000E94E49A04C086E892E00E94C69A44E0C8
:105EF00050E06AE470E0CE010B960E94C69A8B8552
:105F00009C85AD85BE8544E050E06AE470E08F3F3B
:105F10009F4FAF4FBF4F29F482E892E00E94E49A6E
:105F200004C082E892E00E94C69A44E050E062E534
:105F300070E0CE010B960E94C69A8B859C85AD853C
:105F4000BE8544E050E062E570E08F3F9F4FAF4F69
:105F5000BF4F29F48AE892E00E94E49A04C08AE8DC
:105F600092E00E94C69A41E050E06DE170E0CE01FF
:105F700041960E94C69A898941E050E06DE170E047
:105F80008F3F29F48DE39AE00E94E49A04C08DE3E8
:105F90009AE00E94C69A41E050E06CE170E0CE01C8
:105FA00041960E94C69A898941E050E06CE170E018
:105FB0008F3F29F485E692E00E94E49A04C085E6CA
:105FC00092E00E94C69A41E050E06BE170E0CE01A1
:105FD00041960E94C69A898941E050E06BE170E0E9
:105FE0008F3F29F484E692E00E94E49A04C084E69C
:105FF00092E00E94C69A4AE050E064E070E0CE0170
:1060000001960E94C69A89814AE050E064E070E0FF
:106010008F3F29F484E99BE10E94E49A04C084E95B
:106020009BE10E94C69A44E050E066E570E0CE0134
:106030000B960E94C69A8B859C85AD85BE8544E0F3
:1060400050E066E570E08F3F9F4FAF4FBF4F29F4A0
:106050008EE892E00E94E49A04C08EE892E00E94EA
:10606000C69A44E050E067E170E0CE010B960E94D2
:10607000C69A8B859C85AD85BE8544E050E067E17E
:1060800070E08F3F9F4FAF4FBF4F29F480E692E003
:106090000E94E49A04C080E692E00E94C69A42E020
:1060A00050E062E070E0CE010F960E94C69A8F85A4
:1060B000988942E050E062E070E08F3F910529F45A
:1060C0008EE092E00E94E49A04C08EE092E00E948A
:1060D000C69A42E050E060E070E0CE010F960E9468
:1060E000C69A8F85988942E050E060E070E08F3F6B
:1060F000910529F48CE092E00E94E49A04C08CE0BF
:1061000092E00E94C69A61960FB6F894DEBF0FBE69
:10611000CDBFDF91CF910895CF92DF92EF92FF92A2
:1061200060917F027091800280E090E00E94A798C9
:1061300067EA75E00E94BB98892B09F03FC18DE4A6
:106140008093AD1B80E88093AE1B84E08093AF1BEF
:106150001092B01B1092B11B1092B21B1092B31B85
:106160001092B41B8CE390E09093B61B8093B51B08
:106170001092B71B1092B81B1092B91B1092BA1B49
:106180001092BB1B1092BC1B1092BD1B1092BE1B29
:106190001092C01B1092BF1B1092C11B1092C21B09
:1061A0001092C31B1092C41B1092C51B1092C61BE9
:1061B0001092C71B1092C81B1092CA1B1092C91BC9
:1061C0001092CB1B1092CC1B1092CD1B1092CE1BA9
:1061D0001092CF1B1092D01B1092D11B1092D21B89
:1061E0001092D41B1092D31B48E250E062E270E0A0
:1061F0008DEA9BE10E94E49A8AE090E4A0E0B0E09E
:106200008093660290936702A0936802B09369023C
:1062100044E050E06EE170E086E692E00E94E49A8D
:106220001092410A1092420A1092430A1092440AB4
:1062300044E050E06AE570E081E49AE00E94E49A6C
:1062400042E2C42EDD24DA944CECE42E4BE3F42E2F
:10625000C0928602D0928702E0928802F092890270
:1062600044E050E06EE470E086E892E00E94E49A38
:10627000C0928202D0928302E0928402F092850260
:1062800044E050E06AE470E082E892E00E94E49A20
:1062900087ED94E3AFEEBCE380938A0290938B0288
:1062A000A0938C02B0938D0244E050E062E570E070
:1062B0008AE892E00E94E49A8AE999E9A9E1B0E4C7
:1062C00080938E0290938F02A0939002B0939102DC
:1062D00044E050E066E570E08EE892E00E94E49AC7
:1062E00010923D0A80E00E94E67041E050E06DE1CE
:1062F00070E08DE39AE00E94E49A8AE1809365025F
:106300000E948D6F41E050E06CE170E085E692E024
:106310000E94E49A8FE08093640241E050E06BE1D8
:1063200070E084E692E00E94E49A8AE0E4E9FBE10E
:10633000DF011D928A95E9F74AE050E064E070E0E1
:10634000CF010E94E49A80EA96E8A1E0B0E0809351
:10635000600290936102A0936202B093630244E0F2
:1063600050E067E170E080E692E00E94E49A81E00C
:1063700090E090930F0280930E0242E050E062E0C2
:1063800070E08EE092E00E94E49A85E090E09093C5
:106390000D0280930C0242E050E060E070E08CE07F
:1063A00092E00E94E49A81E00E94972480E090E0CD
:1063B000FF90EF90DF90CF900C94150FFF90EF902F
:1063C000DF90CF9008950E94EB6C6C9A6B9A6A9A5A
:1063D0006F9A729A749A739A779A809880B3897F29
:1063E00080BB8398849887E080937E00549A0E94B3
:1063F000302E0E94622E81E00E94C20B80E090E06D
:106400000E94150F6091600270916102809162029A
:10641000909163020E9451660E94B90C6093CC2F48
:106420007093CD2F8093CE2F9093CF2F80916602C3
:1064300086FD239A219A229A239A0E949D0A1D9BE7
:1064400005C010923F0A10923E0A089581E090E044
:1064500090933F0A80933E0A08950F931F93CF9322
:10646000DF939DE8899FE0011124CA54D34E4091E7
:10647000410A5091420A6091430A7091440A41FDD9
:1064800008C08091660280FD04C081FF89C01D9B09
:1064900087C0CE0104969F938F938EEA95E09F93D9
:1064A0008F930E946099FE01ED57FF4F80810F90FE
:1064B0000F900F900F90088119812A813B818823CA
:1064C00009F440C04091D02F5091D12F6091D22F2C
:1064D0007091D32F401B510B620B730B7F936F9303
:1064E0005F934F93389691819F9390819F933297BA
:1064F00091819F9390819F93339790811F929F9357
:10650000319790811F929F93339690811F929F9312
:10651000319790811F929F93CC57DF4F98811F92A4
:106520009F931F928F9384EB95E09F938F930E948C
:1065300060998DB79EB746960FB6F8949EBF0FBE72
:106540008DBF1CC08091D02F9091D12FA091D22FC0
:10655000B091D32F801B910BA20BB30BBF93AF93C2
:106560009F938F938BEF95E09F938F930E946099F9
:106570000F900F900F900F900F900F900E94C00DF2
:1065800080918102882361F01F928F9383EE91E0C6
:106590009F938F930E9472990F900F900F900F907E
:1065A000DF91CF911F910F9108958091B31C8823A3
:1065B00041F08091B41C90E00E942D320E948B0B20
:1065C000F4CF0895CF93DF93EC0188819981823DC8
:1065D0002EE0920749F08A3D2EE09207D1F1892BF7
:1065E00091F582ED9EE02CC0623189F5299A609187
:1065F0000C0270910D027695762F66277795679538
:1066000083E59AE00E946F5D4091410A5091420AF1
:106610006091430A7091440A60FF10C080910D029E
:106620008F9380910C028F938CE790E19F938F93CF
:106630000E9472990F900F900F900F908AED9EE03C
:106640009983888304C01982188283E00FC081E097
:106650000DC083E59AE00E94965D892BC1F383E526
:106660009AE00E94795D0E94D532BBCFDF91CF9135
:1066700008952F923F924F925F926F927F928F92E6
:106680009F92AF92BF92CF92DF92EF92FF920F93C1
:106690001F93CF93DF93CDB7DEB72B970FB6F89448
:1066A000DEBF0FBECDBF9B878A874A01FC01808178
:1066B0009181892B11F00C94924760917F02709127
:1066C0008002CA010E94A79860E870E0C4010E949D
:1066D000DA98009759F460915E3D70915F3D8AE0D1
:1066E00090E00E942E9981E00C94974781309105AB
:1066F00061F4F401B0801B2D110F110B012F412EFD
:10670000512E612E712EA12EBCC082309105B9F49C
:10671000F4018081992787FD9095982F8827218102
:10672000820F911D27FD9A95B82E192F092F000F62
:10673000000B402E502E602E702EA02EA2C0833053
:106740009105B1F5F4012081922F990F990B392F02
:10675000492F592F692F792F892F00E10E948394A7
:1067600019012A013B01B82FA92F2181922F990FDE
:10677000990B392F492F592F692F792F892F08E02D
:106780000E94839459016A017B018C019101A2014D
:10679000B3018B2F9A2F0E94BA94A2801A2D110F49
:1067A000110BB12EC12ED12EE12EF12E012F55C08D
:1067B00004970CF45DC0F4012081922F990F990B7E
:1067C000392F492F592F692F792F892F08E10E94DE
:1067D000839419012A013B01B82FA92F2181922FFF
:1067E000990F990B392F492F592F692F792F892FFD
:1067F00000E10E94839459016A017B018C0191019F
:10680000A201B3018B2F9A2F0E94BA94A3801A2D54
:10681000110F110BB12EC12ED12EE12EF12E012F11
:106820000E94BA9419012A013B01B82FA92F228195
:10683000922F990F990B392F492F592F692F792FA3
:10684000892F08E00E94839459016A017B018C0121
:106850009101A201B3018B2F9A2F0E94BA94B22EFC
:10686000132F042F452E562E672E782EA92E09C0E1
:10687000EAE0BE2E10E000E0412C512C612C712C7E
:10688000A12C0E94C00D2B2D312F402F542D652D92
:10689000762D872D9A2D2537F3E63F07FDE64F0726
:1068A0005105610571058105910511F40C947A4239
:1068B0002537E3E63E07EDE64E0751056105710514
:1068C0008105910511F008F0C0C12337F2E73F07B9
:1068D00041055105610571058105910511F40C947F
:1068E0000D452337E2E73E07410551056105710576
:1068F0008105910511F008F0BFC02536F4E63F0789
:1069000041055105610571058105910509F4F9C736
:106910002536E4E63E07410551056105710581050F
:10692000910511F008F043C0A6E70E94E19411F42C
:106930000C94033F0E94E19409F070F4A8E60E94D1
:10694000E19411F40C94D23CA5E70E94E19411F477
:106950000C94ED3E0C9490472B2D312F402F542D4D
:10696000652D762D872D9A2D2436F1E63F074105BA
:106970005105610571058105910511F40C943545AA
:106980002537E2E63E0741055105610571058105A0
:10699000910509F44DC52A3336424105510561057B
:1069A00071058105910509F44CC30C9490472B2D7A
:1069B000312F402F542D652D762D872D9A2D273779
:1069C000EFE63E0741055105610571058105910519
:1069D00011F40C94E0422737FFE63F0741055105CB
:1069E000610571058105910509F0C8F42436E9E6D1
:1069F0003E0741055105610571058105910511F4B9
:106A00000C94C63E25363E4641055105610571058B
:106A10008105910511F40C9414430C9490472B2D8F
:106A2000312F402F542D652D762D872D9A2D25360B
:106A3000E2E73E07410551056105710581059105B4
:106A400011F40C94DE432936F2E73F074105510566
:106A5000610571058105910511F40C94BC44233343
:106A6000314741055105610571058105910511F019
:106A70000C9490470C9435452B2D312F402F542DDD
:106A8000652D762D872D9A2D2236F5E63F07F4E603
:106A90004F075105610571058105910509F431C75D
:106AA0002236E5E63E07E4E64E075105610571052D
:106AB0008105910511F008F05DC02133F4E63F0730
:106AC000F1E64F075105610571058105910509F44E
:106AD000CCC22133E4E63E07E1E64E0751056105ED
:106AE00071058105910509F0C0F42337F3E73F07ED
:106AF00041055105610571058105910511F40C945D
:106B00002145283734474105510561057105810547
:106B1000910509F496C20C9490472B2D312F402FEC
:106B2000542D652D762D872D9A2D2837F4E63F07B5
:106B3000F1E64F075105610571058105910509F4DD
:106B400090C22C36E5E73E07E2E64E0751056105A7
:106B500071058105910509F46BC42336344641461D
:106B60005105610571058105910511F00C9490475F
:106B70000C9435452B2D312F402F542D652D762D1E
:106B8000872D9A2D2D36E5E73E07E8E64E0751059D
:106B9000610571058105910511F40C944B452D3665
:106BA000F5E73F07F8E64F075105610571058105D7
:106BB000910509F0E0F42237E2E73E07E5E64E07EB
:106BC0005105610571058105910511F40C942B4265
:106BD00023363D46484651056105710581059105FD
:106BE00011F00C9490470E9453180C9492472B2D4F
:106BF000312F402F542D652D762D872D9A2D24363B
:106C0000E3E63E07ECE64E07510561057105810597
:106C1000910511F40C948E412736FFE63F07FCE600
:106C20004F075105610571058105910511F40C941B
:106C3000914123363243494651056105710581056D
:106C4000910511F00C94904730C22B2D312F402F1D
:106C5000542D652D762D872D9A2D2037FCE63F0784
:106C6000F5E64F07F8E65F076105710581059105B7
:106C700009F498C62037ECE63E07E5E64E07E8E65D
:106C80005E07610571058105910511F008F0E6C008
:106C90002437F8E73F07F4E74F0751056105710511
:106CA0008105910511F40C946F3F2437E8E73E0706
:106CB000E4E74E075105610571058105910511F065
:106CC00008F05FC02033F1E33F07F1E74F075105BC
:106CD000610571058105910511F40C942B42203357
:106CE000E1E33E07E1E74E075105610571058105C6
:106CF000910509F0C0F42133F2E63F07F0E74F07B2
:106D00005105610571058105910509F4A6C222337B
:106D1000324640475105610571058105910509F429
:106D2000F1C20C9490472B2D312F402F542D652DFF
:106D3000762D872D9A2D2037F5E63F07F2E74F078E
:106D40005105610571058105910511F40C94DE432F
:106D50002C36E4E73E074E075105610571058105B4
:106D6000910511F40C94B946213331434147510543
:106D7000610571058105910511F00C9490470C9403
:106D80007A422B2D312F402F542D652D762D872DB6
:106D90009A2D2B36ECE63E07E5E74E07E2E65E0766
:106DA000610571058105910509F442C32B36FCE6A6
:106DB0003F07F5E74F07F2E65F07610571058105BB
:106DC000910509F0E0F42437E4E63E07E7E74E07D3
:106DD0005105610571058105910511F40C94074772
:106DE00024373F464F46524661057105810591059E
:106DF00011F00C9490470C9400000C9492472B2DAA
:106E0000312F402F542D652D762D872D9A2D2E361E
:106E1000E1E63E07E8E64E07E3E65E076105710539
:106E20008105910511F40C94433F2633F9E63F07A1
:106E3000F5E74F07F5E65F076105710581059105E7
:106E400009F4B4C529363C464146534661057105EF
:106E50008105910511F00C94904791C32B2D312F92
:106E6000402F542D652D762D872D9A2D2437F3E74D
:106E70003F07F5E64F07F2E75F07610571058105FA
:106E8000910511F40C948E432437E3E73E07E5E6C1
:106E90004E07E2E75E07610571058105910511F076
:106EA00008F064C02337F5E63F07F2E74F07F0E745
:106EB0005F07610571058105910511F40C94FB458F
:106EC0002337E5E63E07E2E74E07E0E75E076105A8
:106ED00071058105910509F0D0F42136FDE63F07E3
:106EE000F5E74F07F8E65F07610571058105910534
:106EF00011F40C94FE422237374740475047610552
:106F000071058105910509F462C20C9490472B2DFF
:106F1000312F402F542D652D762D872D9A2D243617
:106F2000FDE63F07F3E64F07F2E75F0761057105EE
:106F30008105910509F445C62136ECE63E07E5E6F4
:106F40004E07E2E75E07610571058105910509F4C9
:106F50004AC52337324747475047610571058105C8
:106F6000910511F00C9490470C9491432B2D312FE7
:106F7000402F542D652D762D872D9A2D2437E2E74D
:106F80003E07E1E64E07E5E75E076105710581050D
:106F9000910509F471C62437F2E73F07F1E64F0780
:106FA000F5E75F07610571058105910509F0C8F4F2
:106FB0002437E3E73E07E5E64E07E4E75E076105B1
:106FC00071058105910509F4B5C727373047484752
:106FD0005447610571058105910509F42AC70C9490
:106FE00090472B2D312F402F542D652D762D872D39
:106FF0009A2D2F36ECE63E07EFE54E07E6E75E07F3
:10700000610571058105910509F486C52C36F1E607
:107010003F07F4E74F07F8E75F0761057105810552
:10702000910511F40C948346223737464047554763
:10703000610571058105910511F00C9490470C9440
:10704000694183E0809381341092833410928234BA
:1070500041E854E362E182E492E00E94F05A0C9429
:1070600092470E94DB170C94924721E042E161E0D5
:1070700080ED0E942A6821E042E161E080ED0E94FB
:107080002A6821E042E161E080ED0E942A6821E067
:1070900042E161E080ED0E942A6821E042E161E086
:1070A00080ED0E942A680C94924760917F02709153
:1070B000800280E090E00E94A79867E076E00E945E
:1070C000BB98892B09F0C5C060917F027091800246
:1070D00080E090E00E94A7985C01009709F497C0B7
:1070E00060EF73E00E94BB98892BE1F488EE93E097
:1070F000A0E0B0E08093600290936102A0936202EE
:10710000B093630268EE73E080E090E00E94516605
:1071100044E050E067E170E080E692E00E94E49A8B
:107120000C9492476DE076E0C5010E94BB98892BD4
:10713000E1F480E197E2A0E0B0E0809360029093F8
:107140006102A0936202B093630260E177E280E0A3
:1071500090E00E94516644E050E067E170E080E614
:1071600092E00E94E49A0C94924760E176E0C501B7
:107170000E94BB98892BE1F480EA96E8A1E0B0E098
:107180008093600290936102A0936202B0936302C5
:1071900060EA76E881E090E00E94516644E050E0C9
:1071A00067E170E080E692E00E94E49A0C949247D6
:1071B00064E176E0C5010E94BB98892BE1F480E888
:1071C0009AE1A6E0B0E08093600290936102A09300
:1071D0006202B093630260E87AE186E090E00E9488
:1071E000516644E050E067E170E080E692E00E9482
:1071F000E49A0C94924782E693E09F938F930E94C7
:1072000072990E94C00D0F900F900C94924760915C
:10721000600270916102809162029091630228EE97
:1072200033E040E050E00E94A9925F934F933F9378
:107230002F938EE593E09F938F930E9472990E9403
:10724000C00D0F900F900F900F900F900F900C9417
:1072500092470E944D120C94924760917F02709168
:10726000800280E090E00E94A7988C0160EA75E0BF
:107270000E94BB98892BA1F48091660290916702CD
:10728000A0916802B0916902A26080936602909317
:107290006702A0936802B0936902299A0C949247FE
:1072A00063EA75E0C8010E94BB98892BB1F4809114
:1072B000660290916702A0916802B0916902AD7F69
:1072C0008093660290936702A0936802B09369026C
:1072D00080E00E94C7240C949247299B03C080EA57
:1072E00095E002C083EA95E09F938F9386E593E053
:1072F0009F938F930E9472990F900F900F900F9011
:107300000C94924760917F027091800280E090E03F
:107310000E94A7988C0160EA75E00E94BB98892BB7
:10732000E1F48091660290916702A0916802B091A9
:107330006902A4608093660290936702A09368023A
:10734000B09369022A9A44E050E06EE170E086E66C
:1073500092E00E94E49A0C94924763EA75E0C801B7
:107360000E94BB98892BF1F480916602909167028C
:10737000A0916802B0916902AB7F809366029093FE
:107380006702A0936802B093690280E00E94CD2456
:1073900044E050E06EE170E086E692E00E94E49AFC
:1073A0000C9492472A9B03C080EA95E002C083EACE
:1073B00095E09F938F938EE493E09F938F930E9429
:1073C00072990F900F900F900F900C9492476091CC
:1073D0007F027091800280E090E00E94A7988C016B
:1073E00060EA75E00E94BB98892B19F477980C9499
:1073F000924763EA75E0C8010E94BB98892B19F493
:10740000779A0C949247779903C080EA95E002C07E
:1074100083EA95E09F938F9384E195E09F938F9308
:107420000E9472990F900F900F900F900C949247BA
:1074300060917F027091800280E090E00E94A798A6
:107440008C0168E176E00E94BB98892BD1F4809191
:10745000B31C1F928F938091B51C1F928F938091C4
:10746000B41C1F928F931F9284E18F9384E293E068
:107470009F938F930E9472990FB6F894DEBF0FBE50
:10748000CDBF6DE176E0C8010E94BB98892B19F44D
:107490000E94D53270C065E276E0C8010E94BB98B8
:1074A000892B09F047C060917F027091800280E0D3
:1074B00090E00E94A798009709F45DC00E949597FC
:1074C0008531910570F590930F0280930E0242E092
:1074D00050E062E070E08EE092E00E94E49A6091F9
:1074E0007F027091800280E090E00E94A798009750
:1074F00009F441C00E94959790930D0280930C026D
:1075000042E050E060E070E08CE092E00E94E49A9B
:1075100060917F027091800280E090E00E94A798C5
:107520002AC082E193E09F938F930E9472990F90FB
:107530000F9021C080910F028F9380910E028F9344
:1075400089E093E09F938F930E9472990E94C00DEF
:1075500080910D028F9380910C028F938AEF92E0BD
:107560009F938F930E9472990E94C00D0FB6F8945A
:10757000DEBF0FBECDBF0E94C00D0C94924760913C
:107580007F027091800280E090E00E94A7988C01B9
:107590006AE675E00E94BB98892B09F077C060917C
:1075A0007F027091800280E090E00E94A7988C0199
:1075B000009711F40C94924763E276E00E94BB9826
:1075C000892BB1F482E29FEFACECBBE3809386029F
:1075D00090938702A0938802B093890244E050E020
:1075E0006EE470E086E892E00E94E49A0C94924780
:1075F00069E276E0C8010E94BB98892BB1F482E26F
:107600009FEFACECBAE38093860290938702A0933D
:107610008802B093890244E050E06EE470E086E8AE
:1076200092E00E94E49A0C949247C8010E949197BC
:107630002B013C0120E030E0A9010E94208F88232B
:10764000D9F081E00E94560C9B01AC01C301B2014C
:107650000E94248F60938602709387028093880231
:107660009093890244E050E06EE470E086E892E096
:107670000E94E49A0C9492478DEE92E09F938F9330
:107680000E9472990F900F900C9492476DE675E0EE
:10769000C8010E94BB98892B09F077C060917F02D6
:1076A0007091800280E090E00E94A7988C01009782
:1076B00011F40C94924763E276E00E94BB98892B08
:1076C000B1F482E29FEFACECBBE380938202909333
:1076D0008302A0938402B093850244E050E06AE400
:1076E00070E082E892E00E94E49A0C94924769E28A
:1076F00076E0C8010E94BB98892BB1F482E29FEF2B
:10770000ACECBAE38093820290938302A09384024C
:10771000B093850244E050E06AE470E082E892E0D1
:107720000E94E49A0C949247C8010E9491972B0101
:107730003C0120E030E0A9010E94208F8823D9F08D
:1077400082E00E94560C9B01AC01C301B2010E9471
:10775000248F6093820270938302809384029093BB
:10776000850244E050E06AE470E082E892E00E9422
:10777000E49A0C94924780EE92E09F938F930E943C
:1077800072990F900F900C94924765E675E0C801CE
:107790000E94BB98892B09F073C060917F027091A1
:1077A000800280E090E00E94A7988C01009711F47D
:1077B0000C94924763E276E00E94BB98892BB1F467
:1077C00087ED94E3AFEEBCE380938A0290938B0243
:1077D000A0938C02B0938D0244E050E062E570E02B
:1077E0008AE892E00E94E49A0C94924769E276E07B
:1077F000C8010E94BB98892B51F481ED92E09F93C0
:107800008F930E9472990F900F900C949247C80129
:107810000E9491972B013C0120E030E0A9010E94D9
:10782000208F882319F180E00E94560C4B015C01E7
:1078300021EE3AE744E95EE3C301B2010E94598EAA
:10784000A50194010E94248F60938A0270938B0299
:1078500080938C0290938D0244E050E062E570E0EA
:107860008AE892E00E94E49A0C94924784EC92E0B9
:107870009F938F930E9472990F900F900C94924750
:107880000E94A50C9F938F937F936F938DEB92E053
:107890009F938F930E94729982E00E94560C2091D0
:1078A00082023091830240918402509185020E94AD
:1078B000A591162F072FF82EE92E81E00E94560C75
:1078C000EF92FF920F931F932091860230918702CF
:1078D00040918802509189020E94A5919F938F93B5
:1078E0007F936F9381EB92E09F938F930E947299A5
:1078F0000E94C00D0FB6F894DEBF0FBECDBF0C9432
:10790000924760917F027091800280E090E00E9437
:10791000A798009711F10E94CC258090410A909081
:10792000420AA090430AB090440A681579058A0576
:107930009B0539F16093410A7093420A8093430A90
:107940009093440A44E050E06AE570E081E49AE0F4
:107950000E94E49A8DE095E002C086E095E09F9356
:107960008F930E9472996091410A7091420A8091AE
:10797000430A9091440A0E94D9240E94C00D0F909E
:107980000F908BEF94E09F938F930E9472996FEF0B
:107990007FEFCB010E94D9240E94C00D0F900F9061
:1079A0000C9492470E94B6210C949247F401848172
:1079B000843329F440E061E080E00E94F713809175
:1079C0008102882311F40C9492471F928F9388EFC1
:1079D00094E09F938F930E9472990F900F900F9055
:1079E0000F900C949247F4018481893709F080C08C
:1079F00060917F027091800280E090E00E94A798E1
:107A00008C0160EA75E00E94BB98892B51F480914B
:107A1000660290916702A0916802B0916902906439
:107A200010C063EA75E0C8010E94BB98892BD1F4AD
:107A30008091660290916702A0916802B0916902FC
:107A40009F7B8093660290936702A0936802B09335
:107A5000690244E050E06EE170E086E692E00E9448
:107A6000E49A46C06EE276E0C8010E94BB98892B7A
:107A700021F58091AC1B8F938091AB1B8F938091EC
:107A8000AA1B8F938091A91B8F938091A81B8F9322
:107A90008091A71B8F938091A61B8F938091A51B2C
:107AA0008F9386E892E09F938F930E9472990FB60E
:107AB000F894DEBF0FBECDBF1BC0809166029091CF
:107AC0006702A0916802B091690296FF03C080EA44
:107AD00095E002C083EA95E09F938F9382E892E05D
:107AE0009F938F930E9472990F900F900F900F9019
:107AF00080918102882311F40C9492471F928F93F6
:107B000085EF94E09F938F930E9472990F900F904E
:107B10000F900F900C949247F40184818737E9F518
:107B200060917F027091800280E090E00E94A798AF
:107B30000097D9F00E9491972B013C0120E030E0A2
:107B4000A9010E94208F882381F040928E025092DA
:107B50008F02609290027092910244E050E066E5DC
:107B600070E08EE892E00E94E49A809191028F93F7
:107B7000809190028F9380918F028F9380918E02DB
:107B80008F9384E792E09F938F930E9472990F9056
:107B90000F900F900F900F900F908091810288238B
:107BA00011F40C9492471F928F9382EF94E09F936D
:107BB0008F930E9472990F900F900F900F900C94DA
:107BC000924760917F027091800280E090E00E9475
:107BD000A7988C0160EA75E00E94BB98409066020D
:107BE000509067026090680270906902892B19F4C6
:107BF000689457F809C063EA75E0C8010E94BB9811
:107C0000892B99F4E89457F84092660250926702E3
:107C1000609268027092690244E050E06EE170E0A8
:107C200086E692E00E94E49A13C057FE03C080EA01
:107C300095E002C083EA95E09F938F9380E792E0FE
:107C40009F938F930E9472990F900F900F900F90B7
:107C500080918102882311F40C9492471F928F9394
:107C60008FEE94E09F938F930E9472990F900F90E4
:107C70000F900F900C94924760917F027091800258
:107C800080E090E00E94A7985C0164E376E00E94A7
:107C9000BB98892B11F489E108C068E376E0C5013F
:107CA0000E94BB98892B49F480E18093C400109214
:107CB000C50082E08093C00055C06CE376E0C5014A
:107CC0000E94BB98892B11F488E0EFCF61E476E045
:107CD000C5010E94BB98892B39F066E476E0C501A6
:107CE0000E94BB98892B11F483E0DFCF8091C40000
:107CF000893141F48BE692E09F938F930E947299B1
:107D00000F900F908091C400803141F486E692E09C
:107D10009F938F930E9472990F900F908091C4004F
:107D2000883041F480E692E09F938F930E9472998D
:107D30000F900F908091C400833041F48AE592E067
:107D40009F938F930E9472990F900F908091C4001F
:107D5000883041F484E592E09F938F930E9472995A
:107D60000F900F9080918102882311F40C94924718
:107D70001F928F938CEE94E09F938F930E94729941
:107D80000F900F900F900F900C94924760917F028C
:107D90007091800280E090E00E94A79863E276E014
:107DA0000E94BB98892B11F481E001C080E00E9401
:107DB000972480918102882311F40C9492471F929A
:107DC0008F9389EE94E09F938F930E9472990F9006
:107DD0000F900F900F900C9492470E94BD228091BB
:107DE0008102882311F40C9492471F928F9386EEA0
:107DF00094E09F938F930E9472990F900F900F9031
:107E00000F900C9492470E94B9228091810288239E
:107E100011F40C9492471F928F9383EE94E09F93FA
:107E20008F930E9472990F900F900F900F900C9467
:107E3000924760917F027091800280E090E00E9402
:107E4000A7980E949597803170F480933D0A0E9414
:107E5000E67041E050E06DE170E08DE39AE00E9451
:107E6000E49A0C94924780913D0A1F928F938AE482
:107E700092E09F938F930E9472990F900F900F90B2
:107E80000F900C94924760917F027091800280E085
:107E900090E00E94A7980E94959795EF980F9031D7
:107EA00070F4809365020E948D6F41E050E06CE1B8
:107EB00070E085E692E00E94E49A0C9492478091EB
:107EC00065021F928F9381E492E09F938F930E94AB
:107ED00072990F900F900F900F900C9492476091B1
:107EE0007F027091800280E090E00E94A798009746
:107EF00089F04AE050E0BC0184E99BE10E94CB9804
:107F00004AE050E064E070E084E99BE10E94E49A7A
:107F10000C94924784E99BE19F938F938BE496E0C6
:107F20009F938F930E9460990F900F900F900F90E6
:107F30000C94924760917F027091800280E090E003
:107F40000E94A7985C0160EF73E00E94BB98892BA8
:107F5000D9F4219A8091660290916702A0916802FB
:107F6000B091690280618093660290936702A0934A
:107F70006802B093690244E050E06EE170E086E68A
:107F800092E00E94E49ACEC76EE675E0C5010E94B9
:107F9000BB98892BD9F4229A80916602909167024E
:107FA000A0916802B091690280628093660290930A
:107FB0006702A0936802B093690244E050E06EE16A
:107FC00070E086E692E00E94E49AACC762ED73E04E
:107FD000C5010E94BB98892BD9F4239A809166022F
:107FE00090916702A0916802B091690280648093C9
:107FF000660290936702A0936802B093690244E01E
:1080000050E06EE170E086E692E00E94E49A8AC752
:1080100061E175E0C5010E94BB98892BD9F4239AD0
:108020008091660290916702A0916802B091690206
:1080300080688093660290936702A0936802B09371
:10804000690244E050E06EE170E086E692E00E9452
:10805000E49A68C768EE79E0C5010E94BB98892B55
:1080600071F581E08093E52F8DEA9BE19093E72FF6
:108070008093E62F1092E92F1092E82F80916602EC
:1080800090916702A0916802B0916902916080931B
:10809000660290936702A0936802B093690244E07D
:1080A00050E06EE170E086E692E00E94E49A45EED0
:1080B0005FE262E182E492E00E94F05A33C769EF26
:1080C00073E0C5010E94BB98892B11F5EDEDFBE132
:1080D000119211922BE1ED3FF207D1F780916602E8
:1080E00090916702A0916802B091690292608093BA
:1080F000660290936702A0936802B093690244E01D
:1081000050E06EE170E086E692E00E94E49A0AC7D1
:1081100063EA75E0C5010E94BB98409166025091E8
:1081200067026091680270916902892BC1F44F70F7
:108130005C7F40936602509367026093680270937D
:1081400069022B9A44E050E06EE170E086E692E02E
:108150000E94E49A80918A340E94A26FE3C644FF91
:1081600003C080EA95E002C083EA95E09F938F9375
:1081700086E392E09F938F930E94729980916602AA
:108180000F900F900F900F9085FF03C080EA95E04D
:1081900002C083EA95E09F938F938BE292E09F93D6
:1081A0008F930E947299809166020F900F900F90AA
:1081B0000F9086FF03C080EA95E002C083EA95E055
:1081C0009F938F9380E292E09F938F930E94729986
:1081D000809166020F900F900F900F9087FF03C061
:1081E00080EA95E002C083EA95E09F938F9385E152
:1081F00092E09F938F930E94729980916602909172
:108200006702A0916802B09169020F900F900F90E1
:108210000F9090FF03C080EA95E002C083EA95E0EA
:108220009F938F938AE092E09F938F930E9472991D
:108230008091660290916702A0916802B0916902F4
:108240000F900F900F900F9091FF03C080EA95E080
:1082500002C083EA95E09F938F938FEF91E09F9305
:108260008F930E9472998091660290916702A0910B
:108270006802B09169020F900F900F900F9091FFDC
:1082800051C683E596E00E9496996DEDA62E6BE1AE
:10829000B62E0BE010E07BE5872E76E0972EF501F9
:1082A00080819181F2E0AF0EB11C9F938F931F9359
:1082B0000F939F928F920E9460990F5F1F4F0F90B4
:1082C0000F900F900F900F900F900B31110539F711
:1082D00029C68FED94E09F938F930E9472998091AD
:1082E00081020F900F90882361F01F928F938CED85
:1082F00094E09F938F930E9472990F900F900F902C
:108300000F90F89428E088E190E00FB6F894A895D3
:10831000809360000FBE20936000FFCF0E94DB6758
:1083200001C660917F027091800280E090E00E941F
:10833000A7988C0160EA75E00E94BB98892BE9F44C
:108340000E948E6E8091660290916702A0916802F1
:10835000B09169028D7F816080936602909367027D
:10836000A0936802B093690244E050E06EE170E0CF
:1083700086E692E00E94E49AD5C563EA75E0C801FA
:108380000E94BB98892BE1F40E94466E80916602A0
:1083900090916702A0916802B09169028C7F8093EE
:1083A000660290936702A0936802B093690244E06A
:1083B00050E06EE170E086E692E00E94E49AB2C579
:1083C00066E676E0C8010E94BB98892BE9F40E941A
:1083D000466E8091660290916702A0916802B0910A
:1083E00069028E7F82608093660290936702A093F9
:1083F0006802B093690244E050E06EE170E086E606
:1084000092E00E94E49A8EC58091660281FF0FC0BF
:1084100086E696E09F938F938BEF91E09F938F93E7
:108420000E9472990F900F900F900F907BC580FF64
:1084300003C080EA95E002C083EA95E09F938F93A2
:1084400087EF91E09F938F930E9472990F900F9006
:108450000F900F9067C58091E32F8F938091E22F4B
:108460008F938091E12F8F938091E02F8F93809154
:10847000DF2F8F938091DE2F8F938091DD2F8F934D
:108480008091DC2F8F938091DB2F8F938091DA2F57
:108490008F938091D92F8F938091D82F8F93809134
:1084A000D72F8F938091D62F8F938091D52F8F9335
:1084B0008091D42F8F9380EB94E09F938F930E94B1
:1084C00072990E94C00D809181020FB6F894DEBFB0
:1084D0000FBECDBF882309F425C51F928F938DEA67
:1084E00094E09F938F930E9472990F900F900F903A
:1084F0000F9018C5F89481E090E029E0FC012093EA
:108500005700C895E02C80E090E0FC0120935700D4
:10851000C895F02C7894F89483E090E0FC012093C7
:108520005700C895002D82E090E0FC012093570091
:10853000C895102D78948091BD278F938091BC278A
:108540008F938091BB278F938091BA278F9323EAD3
:1085500034E03F932F930E9472991F92EF921F92E3
:10856000FF921F920F931F921F938CE794E09F93AB
:108570008F930E9472990E945723809166001F92E8
:108580008F9380E794E09F938F930E9472990E944B
:10859000C00D809181020FB6F894DEBF0FBECDBF33
:1085A000882309F4BFC41F928F938DE694E09F93B4
:1085B0008F930E9472990F900F900F900F90B2C4FA
:1085C00060E070E080E090E00E94C90D60E070E043
:1085D00081E090E00E94C90D80918102882309F416
:1085E000A1C41F928F938AE694E09F938F930E9479
:1085F00072990F900F900F900F9094C40E94792160
:108600000E94C00D80918102882309F48BC41F92BF
:108610008F9387E694E09F938F930E9472990F90B7
:108620000F900F900F907EC460917F027091800236
:1086300080E090E00E94A7986DE176E00E94BB98F0
:10864000892B31F5F89482E89AE00E94DD5B5C01A9
:10865000009769F0C5010F960E94E15EB50184E0C4
:1086600092E00E94975BC5010E94855CF0CF82E892
:108670009AE00E946A5C892B29F082E89AE00E94C5
:10868000165CF5CF82E89AE00E94D95B789434C0FA
:1086900082E89AE00E94DD5B5C010BE616E0A11423
:1086A000B10451F1F50186811F928F9380851F924D
:1086B0008F9385811F928F9381851F928F938781DE
:1086C0001F928F9384811F928F9383811F928F9328
:1086D00082811F928F9382851F928F931F930F9396
:1086E0000E946099C5010E94855C5C010FB6F894F8
:1086F000DEBF0FBECDBFD3CF80918102882309F4A6
:1087000011C41F928F9384E694E09F938F930E94ED
:1087100072990F900F900F900F9004C40E948C30AC
:1087200001C460917F027091800280E090E00E941D
:10873000A7988C016AEA76E00E94BB98892BD1F455
:108740008091660290916702A0916802B0916902DF
:10875000977F8093660290936702A0936802B0931C
:10876000690244E050E06EE170E086E692E00E942B
:10877000E49AD8C369E276E0C8010E94BB98892BCD
:10878000D1F48091660290916702A0916802B09145
:10879000690298608093660290936702A0936802D2
:1087A000B093690244E050E06EE170E086E692E04A
:1087B0000E94E49AB7C30E942F0AB4C360917F025B
:1087C0007091800280E090E00E94A798FC012081D7
:1087D0002332B1F44AE050E060E070E001960E947C
:1087E00049951B0160917F027091800280E090E0CA
:1087F0000E94A798F4E02F1631040CF094C002C038
:10880000212C312C009709F48EC01982BE016F5FB4
:108810007F4F0E94E92929013A014B01B82FA92F66
:108820008AE0829DF001839DF00D1124E355F44E02
:1088300020812A8331813B8382818C8393819D8334
:1088400024812E8335813F8386818887978199870C
:108850009201A301B4018B2F9A2FAA80BB80CC80F8
:10886000DD80EE80FF80088519850E94D89409F488
:108870005DC08981882351F18CF02A81422A3B8195
:10888000532A8C81682A9D81792A2E81822A3F81F0
:10889000932A8885B82B9985A92B18C040945094A9
:1088A0006094709480949094B095A0952A8142220F
:1088B0003B8153228C8168229D8179222E818222E4
:1088C0003F8193228885B8239985A92340825182CC
:1088D0006282738284829582B683A78348E250E0E5
:1088E00062E270E08DEA9BE10E94E49A8CE594E0FC
:1088F0009F938F930E9472998AE0829DF001839DDD
:10890000F00D1124E355F44E2081318142815381D1
:1089100064817581868197810E9485260E94C00DA1
:108920000F900F9003C082E00E948B2B80E594E0B3
:108930009F938F930E9472992FEF3FEF4FEF5FEF5E
:108940006FEF7FEF8FEF9FEF0E9485260E94C00D93
:10895000809181020F900F90882309F4E3C21F9247
:108960008F938DE494E09F938F930E9472990F9060
:108970000F900F900F90D6C260917F02709180028D
:1089800080E090E00E94A798FC0120812332A1F4AE
:108990004AE050E060E070E001960E9449958B014A
:1089A00060917F027091800280E090E00E94A79821
:1089B00004301105ECF402C000E010E00097C1F0B3
:1089C0004AE050E060E070E00E947D962AE0209F3F
:1089D000F001219FF00D1124E355F44E718760875B
:1089E00048E250E062E270E08DEA9BE10E94E49A86
:1089F00081E00E948B2B80918102882309F492C22E
:108A00001F928F938AE494E09F938F930E947299B0
:108A10000F900F900F900F9085C20E941A5F809167
:108A20008102882309F47EC21F928F9387E494E029
:108A30009F938F930E9472990F900F900F900F90B9
:108A400071C20E944F2C80918102882309F46AC26E
:108A50001F928F9384E494E09F938F930E94729966
:108A60000F900F900F900F905DC280E090E00E94F9
:108A7000732380918102882309F454C21F928F933B
:108A800081E494E09F938F930E9472990F900F90CE
:108A90000F900F9047C28091CA2B81FF2DC00E947A
:108AA000FD20892B49F58091C1278F938091C027A4
:108AB0008F938091BF278F938091BE278F9386E3FA
:108AC00094E09F938F930E9472998091A2348F9328
:108AD0008091A1348F938091A0348F9380919F34A3
:108AE0008F9389E294E09F938F930E9472990FB6BF
:108AF000F894DEBF0FBECDBF0E94C00D8091CA2B7F
:108B00009091CB2B90FF63C081E090E00E94742095
:108B10003B014C0180E090E00E9474201B012C017D
:108B20000E94D21F9F928F927F926F9288E194E071
:108B30009F938F930E9472995F924F923F922F92D0
:108B400088E094E09F938F930E947299222D332D99
:108B5000442D552D662D772D882D992D0E94751E3B
:108B60009F938F937F936F938DEF93E09F938F935A
:108B70000E947299222D332D442D552D662D772D6F
:108B8000882D992D0E94D61E9F938F937F936F936C
:108B90008FEE93E09F938F930E947299222D332D35
:108BA000442D552D662D772D882D992D0E94371F28
:108BB0009F938F937F936F938CED93E09F938F930D
:108BC0000E9472990FB6F894DEBF0FBECDBF0E940F
:108BD000C00D80918102882309F4A4C11F928F9354
:108BE00089ED93E09F938F930E9472990F900F905D
:108BF0000F900F9097C18091CA2B82FF2BC021E06C
:108C000048E061E083E00E946C158091B11C8F9375
:108C10008091B01C8F938091AF1C8F938091AE1C7C
:108C20008F938091AD1C8F938091AC1C8F9380911A
:108C3000AB1C8F938091AA1C8F9382EC93E09F933F
:108C40008F930E9472990E94C00D0FB6F894DEBFF8
:108C50000FBECDBF8091CA2B9091CB2B91FF41C00D
:108C60000E94C219B62EA72E982E892E20E030E041
:108C700048EC52E4D501F4016B2F7A2F8F2F9E2FF1
:108C80000E94A59120E836EE45EC57E40E94248F1F
:108C900021E03EED42E45EE30E9408929B01AC01BC
:108CA00060E070E080E89FE30E94598E2BE43AE395
:108CB0004DEB57E30E94248F9F938F937F936F9385
:108CC0008F929F92AF92BF9289EA93E09F938F9386
:108CD0000E9472990E94C00D0FB6F894DEBF0FBEBD
:108CE000CDBF80918102882309F41CC11F928F930C
:108CF00086EA93E09F938F930E9472990F900F9052
:108D00000F900F900FC160917F027091800280E000
:108D100090E00E94A7986FEA76E00E94BB98892BAA
:108D2000B1F460917F027091800280E090E00E9437
:108D3000A798009709F4F6C00E949597803108F033
:108D4000F1C090915201982B90935201EBC0809109
:108D500052018F701F928F938AEE91E09F938F93B1
:108D60000E9472990E94C00D0F900F900F900F906B
:108D7000D9C060917F027091800280E090E00E94F3
:108D8000A798009711F14AE050E060E070E00E947F
:108D90004995603198F4609364021F926F9389E95A
:108DA00093E09F938F930E94729941E050E06BE1B2
:108DB00070E084E692E00E94E49A11C0809164021F
:108DC0001F928F9380E993E006C0809164021F9206
:108DD0008F9387E893E09F938F930E9472990F90EF
:108DE0000F900F900F900E94C00D809181028823F8
:108DF00009F498C01F928F9384E893E09F938F9318
:108E00000E9472990F900F900F900F908BC06091FD
:108E10007F027091800280E090E00E94A7988C0110
:108E200060EA75E00E94BB98892BE1F40E94F76C20
:108E30008091660290916702A0916802B0916902E8
:108E400090618093660290936702A0936802B0934A
:108E5000690244E050E06EE170E086E692E00E9434
:108E6000E49A60C063EA75E0C8010E94BB98892B50
:108E700081F5F8940E94056D88E10FB6F89480930F
:108E80006000109260000FBE84B7877F84BF80911E
:108E900060008861809360001092600078948091F7
:108EA000660290916702A0916802B09169029F7E6C
:108EB0008093660290936702A0936802B093690260
:108EC00044E050E06EE170E086E692E00E94E49AB1
:108ED00029C064EB76E0C8010E94BB98409166020D
:108EE000509167026091680270916902892B21F4A8
:108EF00054FF18C0F894FFCF54FF03C080EA95E0F8
:108F000002C083EA95E09F938F9386EE91E09F9352
:108F10008F930E9472990F900F900F900F9002C044
:108F20000E949D21EA85FB851182108283E02B96A9
:108F30000FB6F894DEBF0FBECDBFDF91CF911F916A
:108F40000F91FF90EF90DF90CF90BF90AF909F90E8
:108F50008F907F906F905F904F903F902F900895EB
:108F6000CF93DF93EC0188819981009741F08C3C8D
:108F7000914109F48CC01982188283E093C00E9449
:108F8000E3318091660280FD05C081FF01C01D9B19
:108F90000E94466E809170008C7F8093700080915B
:108FA000B60080628093B6001092B20082E0809397
:108FB000B1008091B6008770E1F780917000816008
:108FC000809370006DE47AE080E090E00E94D56CC0
:108FD0000E94B92280E00E94972488EA90E19F9342
:108FE0008F930E9472990E944D128091CA2B0F900C
:108FF0000F9086FD0E9487678091CA2B9091CB2BA2
:1090000090FD0E948E1F8091CA2B87FF06C021E031
:109010004CE061E080ED0E942A6880913D0A0E9448
:10902000E670809165020E948D6F0E948A6F809326
:10903000720A809165020E948D6F80913D0A1F9295
:109040008F938091720A1F928F9389EB96E09F9382
:109050008F930E9460991092740A1092730A0F9075
:109060000F900F900F900F900F9086E592E09093E5
:109070009D3480939C3483E290E09093851280939A
:1090800084128CEC91E19983888381E00BC0633278
:10909000E1F749EF5FE260E070E083E79AE00E9469
:1090A0003933E3CFDF91CF9108950F931F93CF937F
:1090B000DF93EC018A0188819981009711F1813E4B
:1090C000914121F01982188283E020C06231E9F4D5
:1090D000A80162E170E083E79AE00E94393384E0FE
:1090E00080938134109283341092823410938534AB
:1090F0000093843441E854E362E182E492E00E9408
:10910000F05A81EE91E19983888381E0DF91CF91DC
:109110001F910F910895AF92BF92CF92DF92EF927D
:10912000FF920F931F93CF93DF93EC018B015A01B2
:109130008091410A9091420AA091430AB091440A59
:1091400081FD08C08091660280FD04C081FF55C08A
:109150001D9B53C0F801C384D484E584F684A4E63F
:10916000B0E0A70196010E941593672F782F892FF1
:10917000992724E630E040E050E00E94A9927F93D6
:109180006F93CD2CDE2CEF2CFF24DF92CF92F801D1
:1091900086811F928F9385811F928F9388818F7014
:1091A0001F928F9389811F928F93F50181811F9266
:1091B0008F9380811F928F932296DF93CF938BECB6
:1091C00096E09F938F930E94609980918102EDB702
:1091D000FEB774960FB6F894FEBF0FBEEDBF88239E
:1091E00061F01F928F9380EE91E09F938F930E9486
:1091F00072990F900F900F900F90DF91CF911F9168
:109200000F91FF90EF90DF90CF90BF90AF900895B7
:109210008436910514F19F938F938FE097E09F938D
:109220008F930E9460998091D42F9091D52FA09117
:10923000D62FB091D72F0196A11DB11D8093D42FA9
:109240009093D52FA093D62FB093D72F0F900F9038
:109250000F900F9081E090E0089580E090E00895F5
:109260002F923F924F925F926F927F928F929F9236
:10927000AF92BF92CF92DF92EF92FF920F931F9324
:10928000CF93DF93CDB7DEB7C859D1090FB6F894A5
:10929000DEBF0FBECDBFC057DF4F99838883C05953
:1092A000D0408A01633871F487E79AE0C856DF4FEF
:1092B0006883C859D0400E943359C856DF4F68812F
:1092C000C859D040C057DF4FA881B981C059D0409C
:1092D0002D913C912937B1E13B0709F4D8C340F403
:1092E0002115310581F02D3A3F4009F41AC40EC40E
:1092F0002B3841E1340709F4EAC32239314111F432
:109300000C94695603C448EF52E061E870E087E7C7
:109310009AE00E9419598DEA9FE0B0C3E3E0F0E0C3
:10932000EC0FFD1FE20FF31F1082C9010E940849D4
:10933000892B89F720E030E040E050E0C357DF4F51
:109340006881CD58D040627070E080E090E0A0E08D
:109350000E94E19409F097C6C557DF4F2881CB588A
:10936000D040287030E040E050E060E070E080E005
:1093700090E0A0E00E94E194A1F127E04AE250E0F1
:109380006BE270E089E290E00E946B6383E994E312
:109390000E94D965BC01882777FD8095982F0E948F
:1093A000C38F20E030E048EC52E40E94248F9F936A
:1093B0008F937F936F9383E497E09F938F931F9294
:1093C00087E78F93CE018E0D9F1D03969F938F93FA
:1093D0000E94C399E80EF91E0FB6F894DEBF0FBEC7
:1093E000CDBFC557DF4F2881CB58D040207130E02A
:1093F00040E050E060E070E080E090E0A0E00E949B
:10940000E194F1F126E04AE250E06BE270E089E29B
:1094100090E00E946B6381E090E00E944E0D80938B
:109420003C0A86E09CE10E94D965BC01882777FD53
:109430008095982F0E94C38F20E030E048EC52E4E2
:109440000E94248F9F938F937F936F938DE497E077
:109450009F938F931F9287E78F93C7010296E1E056
:10946000F0E0EC0FFD1F8E0F9F1F9F938F930E94C4
:10947000C399E80EF91E0FB6F894DEBF0FBECDBF3C
:10948000272D30E040E050E060E070E080E090E0C8
:10949000A0E00E94E19401F10E940A0D9F938F9336
:1094A0007F936F9388E597E09F938F931F9287E751
:1094B0008F93C701029641E050E04C0F5D1F840F6F
:1094C000951F9F938F930E94C399E80EF91E0FB6C4
:1094D000F894DEBF0FBECDBFC557DF4F2881CB58F4
:1094E000D040207430E040E050E060E070E080E088
:1094F00090E0A0E00E94E19431F18091CF2F8F9312
:109500008091CE2F8F938091CD2F8F938091CC2FF0
:109510008F9386E697E09F938F931F9287E78F93B1
:10952000C7010296A1E0B0E0AC0FBD1F8A0F9B1FE0
:109530009F938F930E94C399E80EF91E0FB6F8947B
:10954000DEBF0FBECDBFC557DF4F2881CB58D040FF
:10955000207830E040E050E060E070E080E090E0B3
:10956000A0E00E94E19441F1F894809179349091C7
:109570007A34A0917B34B0917C347894BF93AF93CC
:109580009F938F9384E797E09F938F931F9287E732
:109590008F93C701029621E030E02C0F3D1F820F10
:1095A000931F9F938F930E94C399E80EF91E0FB6E5
:1095B000F894DEBF0FBECDBF20E0C457DF4F388127
:1095C000CC58D040317040E050E060E070E080E086
:1095D00090E0A0E00E94E19409F067C520E0C45744
:1095E000DF4F3881CC58D040327040E050E060E02E
:1095F00070E080E090E0A0E00E94E19409F0C8C52E
:1096000020E0C457DF4F3881CC58D040347040E060
:1096100050E060E070E080E090E0A0E00E94E19423
:1096200009F0E7C520E0C457DF4F3881CC58D0405F
:10963000387040E050E060E070E080E090E0A0E052
:109640000E94E19409F004C620E0C457DF4F38813E
:10965000CC58D040307140E050E060E070E080E0F5
:1096600090E0A0E00E94E19409F065C620E0C457B4
:10967000DF4F3881CC58D040307240E050E060E09D
:1096800070E080E090E0A0E00E94E19409F083C6E1
:1096900020E030E040E050E0C357DF4F6881CD5814
:1096A000D040647070E080E090E0A0E00E94E1941F
:1096B00009F09FC620E0CB56DF4F3881C559D04016
:1096C00040E050E060E070E080E090E0A0E00E94C8
:1096D000E19409F0FBC620E0CA56DF4F3881C65935
:1096E000D04040E050E060E070E080E090E0A0E03A
:1096F0000E94E19409F018C7502F5170D52E20E038
:1097000030E0452F50E060E070E080E090E0A0E0C5
:109710000E94E19409F036C720E030E0402F42700B
:1097200050E060E070E080E090E0A0E00E94E19412
:1097300009F05BC720E030E0C657DF4F4881CA58C8
:10974000D04050E060E070E080E090E0A0E00E9457
:10975000E19409F07DC720E030E0402F487050E0F0
:1097600060E070E080E090E0A0E00E94E19409F009
:1097700099C720E030E0402F407150E060E070E099
:1097800080E090E0A0E00E94E19409F0BBC720E0F7
:1097900030E0402F407250E060E070E080E090E008
:1097A000A0E00E94E19409F0DDC720E030E0402F06
:1097B000407450E060E070E080E090E0A0E00E9443
:1097C000E19411F00C94E353F02FF078AF2E20E0E9
:1097D00030E04F2F50E060E070E080E090E0A0E0EB
:1097E0000E94E19411F00C941654212F2170B22E96
:1097F00020E030E040E05B2D60E070E080E090E051
:10980000A0E00E94E19411F00C94235420E030E099
:109810004A2D50E060E070E080E090E0A0E00E941F
:10982000E19411F00C94315420E030E040E05B2DE5
:1098300060E070E080E090E0A0E00E94E19411F030
:109840000C94665420E030E040E0512F527060E00C
:1098500070E080E090E0A0E00E94E19411F00C94B0
:109860009B5420E030E040E0512F547060E070E005
:1098700080E090E0A0E00E94E19411F00C94CE54BE
:1098800020E030E040E0512F507160E070E080E077
:1098900090E0A0E00E94E19411F00C94015520E0CA
:1098A00030E040E0512F507260E070E080E090E0E6
:1098B000A0E00E94E19411F00C94405520E030E0CB
:1098C00040E0512F507460E070E080E090E0A0E054
:1098D0000E94E19411F00C947F5520E030E040E0CC
:1098E000512F587060E070E080E090E0A0E00E94AE
:1098F000E19411F00C94BE5520E030E040E05C2D86
:1099000060E070E080E090E0A0E00E94E19411F05F
:109910000C94EF5520E030E04D2D50E060E070E019
:1099200080E090E0A0E00E94E19411F00C942B56AE
:10993000C557DF4F2881CB58D040C457DF4F3881FF
:10994000CC58D040A801C357DF4F6881CD58D040D4
:10995000CE56DF4F7881C259D040CD56DF4F888137
:10996000C359D040CC56DF4F9881C459D040A0E0B5
:109970000E94E19411F00C9436568091640280614B
:10998000898380916B0A8A83FE01EE0DFF1D13828D
:109990008091410A9091420AA091430AB091440AF1
:1099A00087010D5F1F4F80FF0CC01F930F9384E052
:1099B00099E09F938F930E9460990F900F900F9062
:1099C0000F90B801CE0101960E94626280916602FA
:1099D00082FF0AC029E730E3A801BE016F5F7F4F15
:1099E0008FE692E00E94F7668091410A9091420AC8
:1099F000A091430AB091440A82FD73980E948E6E32
:109A000087E79AE00E94355980916602909167023B
:109A1000A0916802B091690290FF40C03FEFE31A45
:109A2000F30A0E948A6FD82E89E10E94A26F4091AA
:109A3000660250916702609168027091690250FF5E
:109A400029C0739880916B0A8F5F80936B0A8A8319
:109A5000B7016F5F7F4FCE0101960E94626287E778
:109A60009AE00E94355940E050E065E88091881204
:109A7000909189120E94F05A89E791E1C057DF4F17
:109A8000A881B981C059D0408D939C933CC0E12CF2
:109A9000F12CCDCF8D2D0E94A26F739A80913E0A3A
:109AA00090913F0A892B11F00E94466E80916B0ABB
:109AB0008F5F80936B0A8091410A9091420AA09136
:109AC000430AB091440A82FF26CC739A24CC83E6E1
:109AD0009AE00E94965D892BB1F00E948E6E809173
:109AE000660287FD2B9860E470E083E69AE00E94AE
:109AF0006F5D82E991E1C057DF4FE881F981C0597C
:109B0000D0409183808381E00C947C56C057DF4F16
:109B1000A881B981C059D0401D921C9283E00C9459
:109B20007C56623181F7C0906602D0906702E09067
:109B30006802F0906902D1FCEECBF801808181309F
:109B400091F50180F281E02D2081C557DF4F2883F8
:109B5000CB58D0403181C457DF4F3883CC58D040E8
:109B6000028113814481C357DF4F4883CD58D040D1
:109B70005581CE56DF4F5883C259D0408681CD568D
:109B8000DF4F8883C359D0409781CC56DF4F9883ED
:109B9000C459D04020843184C257DF4F19821882C3
:109BA000CE58D0406AC08230E9F4A381B481C25754
:109BB000DF4FB983A883CE58D040212C312CB1E09F
:109BC000C557DF4FB883CB58D040C457DF4F1882FA
:109BD000CC58D04000E010E8C357DF4F1882CD5872
:109BE000D0403CC08330F9F0843009F094CB212C74
:109BF000312CC257DF4F19821882CE58D040E5E091
:109C0000C557DF4FE883CB58D040C457DF4F188289
:109C1000CC58D04000E010E0F2E0C357DF4FF883AB
:109C2000CD58D0401BC0212C312CC257DF4F198298
:109C30001882CE58D04025E0C557DF4F2883CB5837
:109C4000D040C457DF4F1882CC58D04000E010E01D
:109C500031E0C357DF4F3883CD58D040CE56DF4F69
:109C60001882C259D040CD56DF4F1882C359D04018
:109C7000CC56DF4F1882C459D0408090CC2F9090A2
:109C8000CD2FA090CE2FB090CF2F40908E0250902D
:109C90008F0260909002709091022DEC3CEC4CE4AD
:109CA0005EE3C301B2010E945A8E9B01AC01C50163
:109CB000B4010E94E69087FD0BC0E894E0F8C092E2
:109CC0006602D0926702E0926802F09269024AC08E
:109CD000A3019201C501B4010E94208F87FF42C0F9
:109CE0008091D82F9091D92FA091DA2FB091DB2FAE
:109CF0000196A11DB11D8093D82F9093D92FA093C9
:109D0000DA2FB093DB2FE0FC06CB6894E0F8C0922A
:109D10006602D0926702E0926802F092690245E41E
:109D2000C557DF4F4883CB58D04050E2C457DF4F70
:109D30005883CC58D04000E010E084E0C357DF4F98
:109D40008883CD58D040CE56DF4F1882C259D040BC
:109D5000CD56DF4F1882C359D040CC56DF4F188202
:109D6000C459D040902F9470C657DF4F9883CA587B
:109D7000D04020E030E0492F50E060E070E080E02B
:109D800090E0A0E00E94E19409F08C9AC557DF4F63
:109D9000A881CB58D040A0727A2E2A2F30E040E024
:109DA00050E060E070E080E090E0A0E00E94E1948C
:109DB00011F00E940A0DC457DF4FB881CC58D04033
:109DC000B074CB56DF4FB883C559D04020E03B2F4D
:109DD00040E050E060E070E080E090E0A0E00E94B1
:109DE000E19411F00E94FD20C457DF4FE881CC5868
:109DF000D040E078CA56DF4FE883C659D04020E013
:109E00003E2F40E050E060E070E080E090E0A0E0B5
:109E10000E94E19451F00E94A50C609386347093E7
:109E200087348093883490938934C557DF4F2881D5
:109E3000CB58D040217030E040E050E060E070E06E
:109E400080E090E0A0E00E94E194F1F084E99BE1E1
:109E50009F938F9383E297E09F938F931F9287E75F
:109E60008F93CE0103969F938F930E94C3996C01A9
:109E70000E9408490FB6F894DEBF0FBECDBF892BF4
:109E800009F049CA760102C0E12CF12CC557DF4F19
:109E90002881CB58D040227030E040E050E060E0B4
:109EA00070E080E090E0A0E00E94E194D1F1C70171
:109EB00002966BE277E041E050E04C0F5D1F840FAB
:109EC000951F0E94C49853E0E50EF11C43E9A42EAF
:109ED00044E3B42E52E0C52E54E0D52E67E7962E0B
:109EE000D5018D915D011F928F93DF92CF921F92CA
:109EF0009F92C7010296E1E0F0E0EC0FFD1F8E0F8C
:109F00009F1F9F938F930E94C399E80EF91E0FB66F
:109F1000F894DEBF0FBECDBF3BE9A31634E3B30612
:109F2000F9F6C557DF4F2881CB58D040247030E078
:109F300040E050E060E070E080E090E0A0E00E944F
:109F4000E19409F447C0C70102966FE277E041E06F
:109F500050E04C0F5D1F840F951F0E94C49854E081
:109F6000E50EF11C4E018AE7880E911C80E1D401B8
:109F70001D928A95E9F728E0A40168E980EB0E9428
:109F8000B0135401B8E0AB0EB11C22E0C22E24E0A5
:109F9000D22E37E7632EF40181914F011F928F93E8
:109FA000DF92CF921F926F92C701029621E030E0BC
:109FB0002C0F3D1F820F931F9F938F930E94C39975
:109FC000E80EF91E0FB6F894DEBF0FBECDBF8A149F
:109FD0009B0409F7512F5078C52E20E030E040E077
:109FE00060E070E080E090E0A0E00E94E194E1F4A5
:109FF00080913E0A90913F0A9F938F9384E397E06C
:10A000009F938F931F9287E78F93CE018E0D9F1D95
:10A0100003969F938F930E94C399E80EF91E0FB683
:10A02000F894DEBF0FBECDBF20E030E040E050E04E
:10A03000C357DF4F6881CD58D040617070E080E039
:10A0400090E0A0E00E94E19409F474C9E3E0F0E03C
:10A05000EC0FFD1FEE0DFF1D80E28083ECEFFFE2B1
:10A06000808197012F5F3F4F7901882309F456C9FA
:10A070008081A1E0B0E0AC0FBD1FAE0DBF1D1296F8
:10A080008C933196EDCFCE018E0D9F1D6BE377E063
:10A0900003960E94C49897E0E90EF11CC7010E9444
:10A0A0000849892B09F037C957C92114310409F42B
:10A0B00095CAF8944090793450907A3460907B340B
:10A0C00070907C3478948091FE1B9091FF1BA0913E
:10A0D000001CB091011CA3019201281B390B4A0BF3
:10A0E0005B0BCA01B9010E94C18F4B015C01B10138
:10A0F00080E090E00E94C18F9B01AC01C501B401DA
:10A100000E94248FB82ED92E9F938F937F936F93A5
:10A110008FE797E09F938F931F9287E78F939E011E
:10A120002E0D3F1D2D5F3F4F3F932F93C856DF4F9E
:10A130006883C859D040C956DF4F7883C759D0408B
:10A140000E94C399E80EF91EC856DF4F6881C859AE
:10A15000D040C956DF4F7881C759D040862F972FFE
:10A16000AB2DBD2D80938B3490938C34A0938D3484
:10A17000B0938E344092FE1B5092FF1B6092001CE5
:10A180007092011C0FB6F894DEBF0FBECDBF26CA79
:10A190002114310409F434CAF8948091D51B9091AC
:10A1A000D61BA091D71BB091D81B78949F938F9307
:10A1B00080916D028F9380916C028F938CE897E071
:10A1C0009F938F931F9287E78F93C7010296A1E019
:10A1D000B0E0AC0FBD1F8A0F9B1F9F938F930E940F
:10A1E000C399E80EF91E0FB6F894DEBF0FBECDBFBF
:10A1F00007CAF89480917D3490917E34A0917F3489
:10A20000B09180347894BF93AF939F938F938CE9F0
:10A2100097E09F938F931F9287E78F93C7010296D2
:10A2200021E030E02C0F3D1F820F931F9F938F93EF
:10A230000E94C399E80EF91EC7010E9408490FB693
:10A24000F894DEBF0FBECDBF892B09F064C8EAC900
:10A250002114310409F4F8C9F89440907D345090E9
:10A260007E3460907F347090803478948091021CAA
:10A270009091031CA091041CB091051CA3019201B4
:10A28000281B390B4A0B5B0BCA01B9010E94C18F15
:10A290004B015C01B10180E090E00E94C18F9B0105
:10A2A000AC01C501B4010E94248FB82ED92E9F9312
:10A2B0008F937F936F9387EA97E09F938F931F927B
:10A2C00087E78F939E012E0D3F1D2D5F3F4F3F93DC
:10A2D0002F93C856DF4F6883C859D040C956DF4F07
:10A2E0007883C759D0400E94C399E80EF91EC8561A
:10A2F000DF4F6881C859D040C956DF4F7881C759B0
:10A30000D040862F972FAB2DBD2D80938F34909307
:10A310009034A0939134B09392344092021C5092A6
:10A32000031C6092041C7092051C0FB6F894DEBFEB
:10A330000FBECDBF89C9232809F498C9F89480912C
:10A34000D91B9091DA1BA091DB1BB091DC1B789498
:10A350009F938F9380916B028F9380916A028F936A
:10A3600084EB97E09F938F931F9287E78F93C701AA
:10A370000296A1E0B0E0AC0FBD1F8A0F9B1F9F9318
:10A380008F930E94C399E80EF91E0FB6F894DEBFB2
:10A390000FBECDBF6BC98091D02F9091D12FA091CE
:10A3A000D22FB091D32FBF93AF939F938F9384EC11
:10A3B00097E09F938F931F9287E78F93C701029631
:10A3C00021E030E02C0F3D1F820F931F9F938F934E
:10A3D0000E94C399E80EF91EC7010E9408490FB6F2
:10A3E000F894DEBF0FBECDBF892B11F00C948B49C2
:10A3F0004FC98091DB2F8F938091DA2F8F938091BB
:10A40000D92F8F938091D82F8F938091D72F8F93AF
:10A410008091D62F8F938091D52F8F938091D42FB9
:10A420008F938FEC97E09F938F931F9297E7D92E8E
:10A43000DF92C7010296A1E0B0E0AC0FBD1F8A0F0A
:10A440009B1F9F938F930E94C399E80EF91EC7012B
:10A450000E9408490FB6F894DEBF0FBECDBF892B0E
:10A4600011F00C948B498091CA2B9091CB2B90FFCB
:10A4700021C98091DF2F8F938091DE2F8F93809160
:10A48000DD2F8F938091DC2F8F9383EF97E09F9345
:10A490008F931F92DF92C701029621E030E02C0FCC
:10A4A0003D1F820F931F9F938F930E94C399E80EC5
:10A4B000F91EC7010E9408490FB6F894DEBF0FBE0F
:10A4C000CDBF892B11F00C948B49F4C88091C12722
:10A4D0008F938091C0278F938091BF278F93809116
:10A4E000BE278F9385E098E09F938F931F9287E715
:10A4F0008F93C7010296A1E0B0E0AC0FBD1F8A0F99
:10A500009B1F9F938F930E94C399E80EF91EC7016A
:10A510000E9408490FB6F894DEBF0FBECDBF892B4D
:10A5200011F00C948B49D7C8809189348F93809116
:10A5300088348F93809187348F93809186348F9362
:10A5400080E198E09F938F931F9287E78F93C701D5
:10A55000029621E030E02C0F3D1F820F931F9F9346
:10A560008F930E94C399E80EF91EC7010E94084903
:10A570000FB6F894DEBF0FBECDBF892B11F00C943F
:10A580008B49BAC881E00E94560C20918602309116
:10A59000870240918802509189020E94A5919F9361
:10A5A0008F937F936F938DE198E09F938F931F928A
:10A5B00087E78F93C7010296A1E0B0E0AC0FBD1F03
:10A5C0008A0F9B1F9F938F930E94C399E80EF91ED9
:10A5D000C7010E9408490FB6F894DEBF0FBECDBF79
:10A5E000892B11F00C948B4997C882E00E94560C7D
:10A5F0002091820230918302409184025091850221
:10A600000E94A5919F938F937F936F938AE298E026
:10A610009F938F931F9287E78F93C701029621E044
:10A6200030E02C0F3D1F820F931F9F938F930E944A
:10A63000C399E80EF91EC7010E9408490FB6F894A5
:10A64000DEBF0FBECDBF892B11F00C948B4972C8B1
:10A6500083E00E94560C9F938F937F936F9387E3C1
:10A6600098E09F938F931F9287E78F93C70102967D
:10A67000A1E0B0E0AC0FBD1F8A0F9B1F9F938F938B
:10A680000E94C399E80EF91E8C98C7010E940849E0
:10A690000FB6F894DEBF0FBECDBF892B11F00C941E
:10A6A0008B4959C88091CA2B87FF63C821E042E1DA
:10A6B00061E080ED0E942A689F938F937F936F9350
:10A6C00084E498E09F938F931F9287E78F93C7014D
:10A6D000029621E030E02C0F3D1F820F931F9F93C5
:10A6E0008F930E94C399E80EF91EC7010E94084982
:10A6F0000FB6F894DEBF0FBECDBF892B11F00C94BE
:10A700008B4937C88091CA2B87FF41C821E042E1BD
:10A7100062E080ED0E942A689F938F937F936F93EE
:10A7200082E598E09F938F931F9287E78F93C701ED
:10A730000296A1E0B0E0AC0FBD1F8A0F9B1F9F9354
:10A740008F930E94C399E80EF91EC7010E94084921
:10A750000FB6F894DEBF0FBECDBF892B11F00C945D
:10A760008B4915C88091CA2B87FF1FC821E042E1A1
:10A7700063E080ED0E942A689F938F937F936F938D
:10A7800080E698E09F938F931F9287E78F93C7018E
:10A79000029621E030E02C0F3D1F820F931F9F9304
:10A7A0008F930E94C399E80EF91EC7010E940849C1
:10A7B0000FB6F894DEBF0FBECDBF892B11F00C94FD
:10A7C0008B490C94D54B8091CA2B87FD02C00C9409
:10A7D000E44B21E042E164E080ED0E942A689F930F
:10A7E0008F937F936F938EE698E09F938F931F9242
:10A7F00087E78F93C7010296A1E0B0E0AC0FBD1FC1
:10A800008A0F9B1F9F938F930E94C399E80EF91E96
:10A81000C7010E9408490FB6F894DEBF0FBECDBF36
:10A82000892B11F00C948B490C94E44B8091CA2B2A
:10A8300082FD02C00C94F54B46E061E083E00E948B
:10A840006C150C94F54B8091CA2B82FD02C00C94C0
:10A85000064C21E046E061E083E00E946C150C9418
:10A86000064C8091CA2B82FD02C00C94144C80913E
:10A87000AD1C8F938091AC1C8F938091AB1C8F93F8
:10A880008091AA1C8F938CE798E09F938F931F92DF
:10A8900087E78F93C701029641E050E04C0F5D1FA0
:10A8A000840F951F9F938F930E94C399E80EF91E02
:10A8B000C7010E9408490FB6F894DEBF0FBECDBF96
:10A8C000892B11F00C948B490C94144C8091CA2B59
:10A8D00082FD02C00C94224C8091B11C8F93809118
:10A8E000B01C8F938091AF1C8F938091AE1C8F937F
:10A8F00084E898E09F938F931F9287E78F93C70117
:10A900000296E1E0F0E0EC0FFD1F8E0F9F1F9F937A
:10A910008F930E94C399E80EF91EC7010E9408494F
:10A920000FB6F894DEBF0FBECDBF892B11F00C948B
:10A930008B490C94224C8091CA2B9091CB2B90FD8B
:10A9400002C00C94314C80E090E00E9474209F93F0
:10A950008F937F936F938FE898E09F938F931F92CD
:10A9600087E78F93C701029641E050E04C0F5D1FCF
:10A97000840F951F9F938F930E94C399E80EF91E31
:10A98000C7010E9408490FB6F894DEBF0FBECDBFC5
:10A99000892B11F00C948B490C94314C8091CA2B6B
:10A9A0009091CB2B90FD02C00C94404C81E090E044
:10A9B0000E9474209F938F937F936F938FE998E009
:10A9C0009F938F931F9287E78F93C7010296E1E0D1
:10A9D000F0E0EC0FFD1F8E0F9F1F9F938F930E943F
:10A9E000C399E80EF91EC7010E9408490FB6F894F2
:10A9F000DEBF0FBECDBF892B11F00C948B490C9498
:10AA0000404C8091CA2B9091CB2B90FD02C00C94AE
:10AA10004F4C81E090E00E9474204B015C0180E08B
:10AA200090E00E9474209B01AC01C501B4010E941A
:10AA3000751E9F938F937F936F9380EB98E09F9306
:10AA40008F931F9287E78F93C701029641E050E0F2
:10AA50004C0F5D1F840F951F9F938F930E94C39986
:10AA6000E80EF91EC7010E9408490FB6F894DEBF30
:10AA70000FBECDBF892B11F00C948B490C944F4C19
:10AA80008091CA2B9091CB2B90FD02C00C945E4C10
:10AA900081E090E00E9474204B015C0180E090E036
:10AAA0000E9474209B01AC01C501B4010E94D61E16
:10AAB0009F938F937F936F938BEB98E09F938F93EC
:10AAC0001F9287E78F93C7010296E1E0F0E0EC0F59
:10AAD000FD1F8E0F9F1F9F938F930E94C399E80EB7
:10AAE000F91EC7010E9408490FB6F894DEBF0FBED9
:10AAF000CDBF892B11F00C948B490C945E4C809146
:10AB0000CA2B9091CB2B90FD02C00C946D4C81E030
:10AB100090E00E9474204B015C0180E090E00E9474
:10AB200074209B01AC01C501B4010E94371F9F93A3
:10AB30008F937F936F9389EC98E09F938F931F92ED
:10AB400087E78F93C701029641E050E04C0F5D1FED
:10AB5000840F951F9F938F930E94C399E80EF91E4F
:10AB6000C7010E9408490FB6F894DEBF0FBECDBFE3
:10AB7000892B11F00C948B490C946D4C8091CA2B4D
:10AB80009091CB2B91FD02C00C947C4C0E94C21979
:10AB90009F938F937F936F938CED98E09F938F9308
:10ABA0001F9287E78F93C7010296E1E0F0E0EC0F78
:10ABB000FD1F8E0F9F1F9F938F930E94C399E80ED6
:10ABC000F91EC7010E9408490FB6F894DEBF0FBEF8
:10ABD000CDBF892B11F00C948B490C947C4CC2573F
:10ABE000DF4FA881B981CE58D04016968C91169728
:10ABF0001F928F9315968C9115971F928F93139692
:10AC00008C9113971F928F9312968C911F928F9312
:10AC10008DEE98E09F938F931F9287E78F93C701E4
:10AC20000296E1E0F0E0EC0FFD1F8E0F9F1F9F9357
:10AC30008F930E94C399E80EF91EC7010E9408492C
:10AC40000FB6F894DEBF0FBECDBF892B11F00C9468
:10AC50008B490C948A4C779A8091410A9091420AD0
:10AC6000A091430AB091440A92FD749A8091410ADE
:10AC70009091420AA091430AB091440A82FD0CC00F
:10AC80008091660280FD08C081FD02C00C94BD4C1D
:10AC90001D9902C00C94BD4C40E050E060E070E0B3
:10ACA000CE0101960E94A40A2091B31C30E080914D
:10ACB0000E0290910F022817390710F40C94BD4C26
:10ACC00040E050E062E180E192E00E94F05A0C9492
:10ACD000BD4C83E69AE00E94965D892B11F40C949A
:10ACE000834D0E94466E8091660287FD02C00C94DF
:10ACF0008B492B9A0C948B49C856DF4F0FB6F894AA
:10AD0000DEBF0FBECDBFDF91CF911F910F91FF909E
:10AD1000EF90DF90CF90BF90AF909F908F907F90FB
:10AD20006F905F904F903F902F9008950C945C59D6
:10AD30006F927F928F929F92AF92BF92CF92DF924B
:10AD4000EF92FF920F931F93CF93DF93CDB7DEB7B0
:10AD500060970FB6F894DEBF0FBECDBF5B010E94B7
:10AD60008A6FE82FF0E0EE0FFF1FE953F44E808169
:10AD700091810196918380838091410A9091420A4A
:10AD8000A091430AB091440A81FD7498C090660274
:10AD9000D0906702E0906802F09069020E94B6616C
:10ADA0008C01FC018081982F92959F70913099F4CD
:10ADB0008F7051F48091AB1B9091AC1B01969093D6
:10ADC000AC1B8093AB1B38C1B50183EA94E30E94AE
:10ADD000D258892B51F08091A91B9091AA1B019602
:10ADE0009093AA1B8093A91B27C1D701C6012EE00F
:10ADF000B695A795979587952A95D1F7F82FF17075
:10AE00006F2E82E89AE00E94DD5B4C01009709F406
:10AE100048C0B501C40102960E94D258892BE9F1BD
:10AE2000940147E65AE060E074E6C4010F960E9480
:10AE30005D5EF8019181F4018481981321C08285BF
:10AE40008F5F82878091A71B9091A81B019690939A
:10AE5000A81B8093A71B84E00E94D362F401208585
:10AE600030E02817390708F07BC184E00E94D362E4
:10AE7000F4018087F80180818F70F4018187DCC044
:10AE8000F401128684E00E94D362F4018087F80105
:10AE900080818F70F401818764C1C4010E94855C48
:10AEA000B4CF84E092E00E94725B4C01009709F4F9
:10AEB000C3C0B501C40102960E94C958F80181813E
:10AEC0008150F401848380E091E0A0E0B0E08387CA
:10AED0009487A587B687128684E00E94D362F40126
:10AEE0008087F80180818F70F4018187B40182E846
:10AEF0009AE00E943D5C940147E65AE060E074E607
:10AF0000C4010F960E945D5E77247394F8018181DD
:10AF1000F4018483F80180818F70F401878384E0D9
:10AF20000E94D362F401858383E00E94D362F4011E
:10AF3000868387818F3009F0712CF801C180F4017C
:10AF40008481C81AD12CE12CF12C76E0CC0CDD1CCC
:10AF5000EE1CFF1C7A95D1F72385348545855685EF
:10AF6000A0ECB0E00E941593BB27A92F982F872F44
:10AF7000C80ED91EEA1EFB1EC386D486E586F68659
:10AF8000A501B401C8010E94A40A2091B31C30E0BD
:10AF900080910E0290910F022817390738F040E097
:10AFA00050E062E180E192E00E94F05A80910E024E
:10AFB00090910F02029708F44BC08091CA2B86FF34
:10AFC0002AC00E947967C80105960E944567F8016A
:10AFD00081811F928F93F40186811F928F938581C7
:10AFE0001F928F9385E199E09F938F931F9280E149
:10AFF0008F93CE0101967C01FF928F930E94C3999B
:10B0000082E00E945F67C7010E9445670FB6F8940F
:10B01000DEBF0FBECDBF8091660290916702A09106
:10B020006802B091690297FD50C080910E02909124
:10B030000F02029708F47EC08091410A9091420A63
:10B04000A091430AB091440A81FF8DC0749A8BC0CD
:10B050008091660290916702A0916802B0916902A6
:10B0600096FFABCF662009F4A8CFF8012081322FDC
:10B070003F70832F90E00297F4F08FEF830F207FD3
:10B08000822B808387E79AE00E9496568091A51BC9
:10B090009091A61B01969093A61B8093A51B80916F
:10B0A000410A9091420AA091430AB091440A96FF46
:10B0B00084CF739882CF8091AB1B9091AC1B01968B
:10B0C0009093AC1B8093AB1B78CF84E99BE12091DC
:10B0D000941B222309F4A9CF9F938F9388E299E0D0
:10B0E0009F938F93CE0101967C01FF928F930E94D4
:10B0F000009A6C01B701C80102960E94E5980F9072
:10B100000F900F900F900F900F90009709F48DCF34
:10B1100096012F5F3F4F280F391FA9012F5F3F4F27
:10B12000FA0180818032C9F362E18AE192E00E94F3
:10B13000F05A7BCF772009F47FCF82E08093E52F10
:10B140001092E72F1092E62F9092E92F8092E82F2D
:10B1500045EE5FE262E182E492E00E94F05A6CCF39
:10B16000612C712CD3CE60960FB6F894DEBF0FBE63
:10B17000CDBFDF91CF911F910F91FF90EF90DF90A6
:10B18000CF90BF90AF909F908F907F906F900895D9
:10B190000895FB012081FC012083FB012181FC013A
:10B1A00021830895FC019081DB018C91981309C0E3
:10B1B00081E090E0318111962C91321721F080E0EE
:10B1C000089580E090E00895BC0183EA94E30C9434
:10B1D000C958DC011996ED91FC911A970280F38110
:10B1E000E02D309709F0099408950F931F93CF93A2
:10B1F000DF9300D0CDB7DEB78C0188E10E94E66214
:10B20000BC01CE0101960E94C958D8011996ED9152
:10B21000FC911A970190F081E02DBE016F5F7F4F86
:10B22000C80109950F900F90DF91CF911F910F9159
:10B230000895EF92FF920F931F93CF93DF93EC014A
:10B240008B017A0142E153E00E944259FA86E98675
:10B2500066E173E0C801DF91CF911F910F91FF90DC
:10B26000EF900C949B590C945A59CF93DF93EC01B7
:10B2700063EA74E388E10E94DC62CE01DF91CF9142
:10B280000C945C59EF92FF920F931F93CF93DF932F
:10B29000EC018B017A010E947759F886EF826AE10E
:10B2A00073E0C801DF91CF911F910F91FF90EF9054
:10B2B0000C949B590C947F590C940474DC011796E0
:10B2C000ED91FC9118970190F081E02D0994DC013B
:10B2D0001796ED91FC9118970280F381E02D30973D
:10B2E00009F00994089586E892E10C94D95BFC0179
:10B2F00073836283BC0186E892E10C943D5CBC01DF
:10B3000086E892E10C94225CCF93DF93EC0186E80F
:10B3100092E10E94DD5B009749F0FC0122813381BC
:10B320002C173D0729F00E94855CF5CF80E090E066
:10B33000DF91CF9108950F931F93CF93DF938B01EC
:10B340000E948459EC01009731F01D830C83C801E1
:10B350000E9435768E83DF91CF911F910F910895D2
:10B360001F93CF93DF93EC01162FEC81FD81309773
:10B37000D1F0909389128093881282E08887CE0161
:10B3800006960995992787FD90950297029710F0E8
:10B39000133839F4BE01CE01DF91CF911F910C9487
:10B3A000DD5981E08887DF91CF911F910895FC01DD
:10B3B000208520FD0C94B0590895CF92DF92EF9232
:10B3C000FF920F931F93CF93DF93EC016B01E090FB
:10B3D0008812F090891200918A1210918B12F80154
:10B3E000EC17FD0739F0309709F44AC00190F0815D
:10B3F000E02DF6CF209709F443C08885882309F112
:10B4000018860115110561F0C017D10729F0AE01AA
:10B4100067E8C8010E94D759F80100811181F1CF76
:10B42000EC81FD81309769F0CC15DD0551F0D093AA
:10B430008912C093881240E050E063E8CE0106967E
:10B440000995E0918A12F0918B12CE17DF0769F40B
:10B450008881998190938B1280938A120DC080818C
:10B4600091818C179D0721F0FC013097C1F704C032
:10B470008881998191838083F0928912E092881269
:10B48000DF91CF911F910F91FF90EF90DF90CF90C0
:10B4900008951F93CF93DF9310929412C0918A1254
:10B4A000D0918B1211E0209779F08985882341F0A3
:10B4B0001887198640E050E062E8CE010E94B0593A
:10B4C0000990D881C02DEFCFDF91CF911F910895C2
:10B4D0008091371391E0980F9093371308956091FE
:10B4E0008812709189120C94DD598AE88093371381
:10B4F000109235131092361310928B1210928A12FA
:10B5000010928912109288120895809194128111DC
:10B510000E94495A70913613772309F451C0E09183
:10B5200035132E2F30E085E0E89FF0011124EB5613
:10B53000FD4E60816093931241815281509392122B
:10B5400040939112838194819093901280938F12F3
:10B550002F5F3F4F2F713327209335137150709316
:10B560003613009731F580918A1290918B12909347
:10B570008E1280938D1280918D1290918E12892B54
:10B58000F9F08091941281110E94495A40919112D0
:10B59000509192126091931280918D1290918E121F
:10B5A0000E94D759E0918D12F0918E128081918185
:10B5B000DECF613819F421E0FC0120870E94D759C1
:10B5C000809194122091361390E0820F911D08957E
:10B5D000809194122091361390E0820F911D08956E
:10B5E000209136132032B9F0E0913513E20FEF715C
:10B5F000E0938C1235E0E39FF0011124EB56FD4EF1
:10B60000608352834183948383832F5F2093361317
:10B6100080E090E0089581E090E00895CF93DF937B
:10B62000C0918812D09189120E94D759D093891263
:10B63000C0938812DF91CF910895AB0130918A12A7
:10B6400020918B12E32FF22FE817F907B1F0309712
:10B6500021F00190F081E02DF7CF009771F0FC010F
:10B660003083218390938B1280938A1221E020876C
:10B670001782168261E80C940E5B0895009749F0DA
:10B68000FC0120852150223020F421E021872093E5
:10B690009412089521E030E0FC018085811102C000
:10B6A00020E030E0C9010895CF93DF93EC014A8197
:10B6B0005B8160E070E08C819D810E94B4982A815A
:10B6C0003B8188819981289FA001299F500D389F37
:10B6D000500D112460E070E08E819F81DF91CF9149
:10B6E0000C94B498FC018281938120E030E028170B
:10B6F0003907D1F0A481B581A20FB31F4C9141113C
:10B7000010C081E08C9380819181289FA001299FA6
:10B71000500D389F500D112486819781840F951FFD
:10B7200008952F5F3F4FE3CF80E090E00895FC0144
:10B73000268137814281538180E090E0841795070C
:10B74000C9F02617370781F4A481B581A80FB91F66
:10B750002C91121614F421502C930480F581E02DC5
:10B76000E80FF91F80810895A081B1812A0F3B1F46
:10B770000196E4CF8FEF0895FC01868197816817C9
:10B780007907A0F0A081B18142815381A49F9001EB
:10B79000A59F300DB49F300D1124280F391F81E073
:10B7A00090E06217730720F080E0089580E090E059
:10B7B0000895FC01118210820895FC01808191811D
:10B7C0000895FB0120813181FC013183208308959C
:10B7D000DC01ED91FC91309731F0808191810097EF
:10B7E00029F0FC01FACF80E090E00895CF010895A0
:10B7F000DC01ED91FC9111973097A9F02081318106
:10B80000232B21F41D921C92CF010895A081B181B8
:10B810008D919C911197892B11F0FD01F7CF118229
:10B820001082CD01089580E090E00895DC01ED9153
:10B83000FC911197309721F0208131812D933C9319
:10B84000CF010895DC01ED91FC913097A9F0A0E0C3
:10B85000B0E020813181E617F70741F4109709F431
:10B86000DC012D933C93118210820895211531053E
:10B8700019F0DF01F901EDCF08950F931F93CF93D6
:10B88000DF938C01EB010E94225C19821882C801AF
:10B890000E94E85B009711F4F80101C0FC01D1831C
:10B8A000C083DF91CF911F910F9108950F931F9344
:10B8B000CF93DF93EC018B010E94225C88819981F8
:10B8C000F8019183808319830883DF91CF911F91C1
:10B8D0000F910895DC01ED91FC9180E090E03097AC
:10B8E00029F001960190F081E02DF9CF0895FB0138
:10B8F000309719F4BA010C94565C80819181DA0179
:10B900008D939C93518340830895009721F0FC010F
:10B9100080819181089580E090E0089580913A13AC
:10B9200090913B13892B29F41092391310923813FC
:10B9300008950E94916BE0913A13F0913B1322819C
:10B94000338140815181240F351F281B390B04801E
:10B95000F581E02D309769F04281538160817181DA
:10B96000460F571F481B590B4217530780F79A0180
:10B97000EECF280F391F30933913209338130895D1
:10B9800084E992E00C943E5BEF92FF920F931F9339
:10B99000CF93DF938C01FC0180819181009799F016
:10B9A0008A359105D9F0F8011182108283E068C0D0
:10B9B000868197818417950709F049C00480F58135
:10B9C000E02D3097A9F710923B1310923A138AE5B5
:10B9D00090E0F8019183808381E052C0673891F153
:10B9E0006238A9F7C0913A13D0913B13E12CF12CA6
:10B9F000209769F3CE010E94067A892BF1F0AE01FF
:10BA000068E88E819F810E94F05A892BA1F41F82E1
:10BA10001E828C819D81E114F10421F0F701958350
:10BA2000848304C090933B1380933A131D821C823D
:10BA30000E948E5CD7CF0E94C05C7E010C80DD81AD
:10BA4000C02DD6CFE0913A13F0913B13BACFF093CB
:10BA50003B13E0933A13A481B581109709F4B7CF53
:10BA600016968D919C9117978417950711F0FD01FB
:10BA7000F2CF14968D919C91159795838483EBCF8B
:10BA8000DF91CF911F910F91FF90EF900895CF9389
:10BA9000DF93EC010E94C05C8E819F8130913A134C
:10BAA00020913B13892B59F0E32FF22F309739F077
:10BAB000EC17FD0781F00480F581E02DF7CF809130
:10BAC0008812909189129F838E833C832D83D0931B
:10BAD0003B13C0933A13DF91CF910C948E5CCF93BC
:10BAE000DF93EC010E94E679CE01DF91CF910C94B7
:10BAF000475DCF93DF93EC010E94F279CE01DF9195
:10BB0000CF910C94475DCF93DF93EC010E94FC79B9
:10BB1000CE01DF91CF910C94475DFC0120813181F2
:10BB2000260F371F318320830C948E5C21E030E098
:10BB3000FC0186819781892B11F020E030E0C9015A
:10BB40000895FC012281338180819181820F931FAE
:10BB50000895FC0180819181089581E090E0209119
:10BB60003A1330913B13232B11F480E090E00895B9
:10BB700080913A1390913B13892B29F080913813CF
:10BB800090913913089580E090E00895CF93DF936A
:10BB9000EC01E0913A13F0913B138E179F0769F483
:10BBA0008C819D8190933B1380933A130DC08481C7
:10BBB00095818C179D0721F0FC013097C1F706C0D5
:10BBC0008C819D81958384830E948E5C1D821C8262
:10BBD0001F821E82DF91CF910895EF92FF920F9303
:10BBE0001F93CF93DF938C017A01FC0180819181B7
:10BBF000009741F08B34910501F1F8011182108218
:10BC000083E048C08DE393E10E94DD5BEC01209767
:10BC100051F06C817D81CE0102960E946F5D09908A
:10BC2000D881C02DF4CF81E080933C138BE490E069
:10BC3000F8019183808381E02DC06838E1F78DE3BE
:10BC400093E10E94DD5BEC01209781F3CE01029627
:10BC5000E816F906D9F4BE018DE393E10E94225C57
:10BC6000E0908812F09089128A859B8590938912C2
:10BC700080938812EC85FD85309719F08E859F851D
:10BC80000995F0928912E0928812D0CF0990D8815C
:10BC9000C02DDACFDF91CF911F910F91FF90EF90E0
:10BCA000089510923C138DE393E10E94D95B60E00C
:10BCB00070E08EE992E00C941D5B0F931F93CF937D
:10BCC000DF93EC0100918812109189121B870A877B
:10BCD0005D874C873F872E8780913C13882379F0BE
:10BCE0008EE992E09093891280938812CE01029699
:10BCF0000E946F5D109389120093881202C07D83A9
:10BD00006C83BE018DE393E10E94225CBE018DE352
:10BD100093E1DF91CF911F910F910C943D5C0F93B4
:10BD20001F93CF93DF93EC0180913C13882391F014
:10BD300000918812109189128EE992E090938912F5
:10BD400080938812CE0102960E94795D1093891229
:10BD500000938812BE018DE393E10E94225CBE0134
:10BD60008DE393E1DF91CF911F910F910C943D5C96
:10BD70000F931F93CF93DF93EC0180913C138823A3
:10BD800091F000918812109189128EE992E09093BF
:10BD9000891280938812CE0102960E94835D1093CF
:10BDA000891200938812BE018DE393E10E94225C08
:10BDB000BE018DE393E1DF91CF911F910F910C9420
:10BDC0003D5CCF93DF93EC0180913C13882329F0F5
:10BDD000CE0102960E94C65D04C01F821E82198693
:10BDE0001886BE018DE393E1DF91CF910C94225C24
:10BDF000CF93DF93EC0180913C13882331F0CE0187
:10BE00000296DF91CF910C94965D8DE393E10E94B1
:10BE1000DD5B009739F08C179D0739F0FC018081BC
:10BE20009181F7CF81E090E002C080E090E0DF9167
:10BE3000CF9108952F923F924F925F926F927F928F
:10BE40008F929F92AF92BF92CF92DF92EF92FF922A
:10BE50000F931F93CF93DF93CDB7DEB7E8970FB65D
:10BE6000F894DEBF0FBECDBFEAEDF6E3208131814D
:10BE700042815381E6EDF6E3508041803280238099
:10BE8000E2EDF6E38081898391819A83A281AB837D
:10BE90006380EEECF6E3B081BC8381818D83928177
:10BEA0009E83A381AF83EAECF6E3B081B8878181FA
:10BEB000898792819A87A381AB87E6ECF6E3B0810C
:10BEC000BC8781818D8792819E87A381AF87E2ECB9
:10BED000F6E3B081B88B8181898B92819A8BA381A3
:10BEE000AB8BEEEBF6E3B081BC8B81818D8B9281C5
:10BEF0009E8BA381AF8BEAEBF6E3B081B88F818193
:10BF0000898F92819A8FA381AB8FE6EBF6E3B081A4
:10BF1000BC8F81818D8F92819E8FA381AF8FE2EB49
:10BF2000F6E3B081B8A3818189A392819AA3A3810A
:10BF3000ABA3EEEAF6E3B081BCA381818DA392812D
:10BF40009EA3A381AFA3EAEAF6E3B081B8A78181FB
:10BF500089A792819AA7A381ABA7E6EAF6E3B0810D
:10BF6000BCA781818DA792819EA7A381AFA7E2EA9A
:10BF7000F6E3B081B8AB818189AB92819AAB7380D3
:10BF8000EEE9F6E3B080A18092808380EAE9F6E3EF
:10BF9000F080E180D280C380E6E9F6E3A081AFAB18
:10BFA000B181B8AF128103812BAB3CAB4DAB5EAB23
:10BFB0000E94BF6B5EA95F934DA94F933CA93F932D
:10BFC0002BA92F932F923F924F925F926F922B81CA
:10BFD0002F932A812F9329812F932F812F932E81A5
:10BFE0002F932D812F932C812F932B852F932A858F
:10BFF0002F9329852F9328852F932F852F932E8577
:10C000002F932D852F932C852F932B892F932A895E
:10C010002F9329892F9328892F932F892F932E8946
:10C020002F932D892F932C892F932B8D2F932A8D2E
:10C030002F93298D2F93288D2F932F8D2F932E8D16
:10C040002F932D8D2F932C8D2F932BA12F932AA1DE
:10C050002F9329A12F9328A12F932FA12F932EA1A6
:10C060002F932DA12F932CA12F932BA52F932AA58E
:10C070002F9329A52F9328A52F932FA52F932EA576
:10C080002F932DA52F932CA52F937F922AA92F9321
:10C0900029A92F9328A92F938F929F92AF92BF9295
:10C0A000CF92DF92EF92FF920F931F9328AD2F93C1
:10C0B0002FA92F939F938F937F936F93A4EAB4E359
:10C0C0008C911F928F93E3EAF4E380811F928F9308
:10C0D0008DE191E19F938F930E947299EAE0F7E3DB
:10C0E0002081318142815381E6E0F7E35080418035
:10C0F00032802380EAEFF6E3908081807280638053
:10C10000E6EFF6E38081898391819A83A281AB83F4
:10C11000B381BC83E2EFF6E380818D8391819E83BE
:10C12000A281AF83B381B887EEEEF6E38081898781
:10C1300091819A87A281AB87B381BC87EAEEF6E34F
:10C1400080818D8791819E87A281AF87B381B88BD3
:10C15000E6EEF6E38081898B91819A8BB280A38091
:10C16000E2EEF6E3F080E180D280C380EEEDF6E30C
:10C17000A081AB8BB181BC8B128103810FB6F89487
:10C18000DEBF0FBECDBF2BAB3CAB4DAB5EAB0E9459
:10C19000BF6B5EA95F934DA94F933CA93F932BA919
:10C1A0002F932F923F924F925F926F927F928F9236
:10C1B0009F922C812F932B812F932A812F9329815A
:10C1C0002F9328852F932F812F932E812F932D81AD
:10C1D0002F932C852F932B852F932A852F93298599
:10C1E0002F9328892F932F852F932E852F932D857D
:10C1F0002F93AF92BF922A892F9329892F93CF92A1
:10C20000DF92EF92FF920F931F932C892F932B892C
:10C210002F939F938F937F936F93A4EAB4E38C91B2
:10C220001F928F93E3EAF4E380811F928F938EEA4B
:10C2300090E19F938F930E9472990FB6F894DEBF9E
:10C240000FBECDBFE8960FB6F894DEBF0FBECDBFD0
:10C25000DF91CF911F910F91FF90EF90DF90CF90E2
:10C26000BF90AF909F908F907F906F905F904F9016
:10C270003F902F90089580E38093F3130895CF9318
:10C28000DF936091F31370E0C0E3D0E0C61BD70BDF
:10C290006F5B7C4EAE010E94AB98CE01DF91CF91D7
:10C2A0000895CF92DF92EF92FF920F931F93CF9357
:10C2B000DF937C01C090F613D090F7136091F313D5
:10C2C00070E0E601E096C61BD70BC138D105D8F463
:10C2D00000E310E0061B170B6F5B7C4EA8010E9469
:10C2E000AB9860913F13709140138091F41390913B
:10C2F000F513680F791FA601C701800F911F0E94D7
:10C30000AB98CE0102C080E090E0DF91CF911F9109
:10C310000F91FF90EF90DF90CF9008959091F313DD
:10C32000980F9093F31308954091F6135091F713DB
:10C330004817590798F02091F4133091F513280FFE
:10C34000391F3093F5132093F413481B590B509366
:10C35000F7134093F61381E090E0089580E090E0B9
:10C3600008959093F7138093F61308958091F41332
:10C370009091F5138F589C4E08958091F31390E09F
:10C380008F5B9C4E089581E090E020913F133091A7
:10C3900040132157334111F480E090E008950E944A
:10C3A000C361892B61F060913F13709140134091FC
:10C3B000F6135091F71381E793E10C94AB98209119
:10C3C000F4133091F51321153105B9F08091F6136E
:10C3D0009091F713C096E1E7F3E1AF014154534167
:10C3E0004817590734F4DF01A20FB31F4C91419352
:10C3F000F4CF1092F5131092F413089580913F1327
:10C400009091401308958091F6139091F713089539
:10C410009091F31380E3891B089520E38091F31337
:10C42000281B8091F6139091F713820F911D0895A8
:10C430001F93CF93DF93EC011091F313812F90E0C2
:10C440008C179D076CF00E940D628C0F9D1F813828
:10C45000910530F41C1B1093F31381E090E002C0AF
:10C4600080E090E0DF91CF911F910895CF93DF930B
:10C47000EDEAF4E31192119284E3ED3DF807D1F770
:10C48000C5EAD4E360E173E0CE010E94C958229668
:10C4900084E3CD3AD807B1F7DF91CF910895109298
:10C4A000F5131092F4131092F7131092F61380E321
:10C4B0008093F31381E793E19093401380933F13AC
:10C4C0000C943662EF92FF920F931F93CF93DF93FA
:10C4D00000D0CDB7DEB78C0169837A830E944F62AA
:10C4E0006981E62E7A81F72E81E8E816F10418F0CA
:10C4F00080E8E82EF12CA701B80180913F139091BC
:10C5000040130E94AB98F092F713E092F613C70124
:10C510000F900F90DF91CF911F910F91FF90EF90AF
:10C5200008950F931F93CF93DF938C01EB010E942B
:10C530004F621093401300933F13D093F713C093AF
:10C54000F613DF91CF911F910F91089520E3EDEA4B
:10C55000F4E3DC0101900D922A95E1F788E0E5EA29
:10C56000F4E3DB0101900D928A95E1F7089520E351
:10C57000FC01ADEAB4E301900D922A95E1F788E061
:10C58000FB01A5EAB4E301900D928A95E1F70895C5
:10C59000E82FF0E0EE0FFF1FE355FB4C7183608343
:10C5A00081E090E00895E82FF0E0EE0FFF1FE355E3
:10C5B000FB4C80819181089590E0880F991F8B58E2
:10C5C0009B4C0E94C95881E090E0089590E0880F4C
:10C5D000991F8B589B4C08958115910511F0019777
:10C5E000F1F70895E091E034F091E1349081809189
:10C5F000DF3489230895E091DD34F091DE348081C9
:10C600009091DF34892B8083E091E234F091E33420
:10C6100080819091DF34892B80830895E091DD340F
:10C62000F091DE3490818091DF348095892380837E
:10C63000E091E234F091E33490818091DF34809591
:10C640008923808308951F93CF93DF93E091DD3496
:10C65000F091DE3490818091DF348095892380834E
:10C66000E091E234F091E33480819091DF34892BC2
:10C6700080838FEB93E00E94EC621FB7F894E09107
:10C68000E234F091E33490818091DF348095892306
:10C69000808383E890E00E94EC62E091E034F091C6
:10C6A000E134D081C091DF341FBF78948BE393E0F5
:10C6B0000E94EC62E091E034F091E134908180914D
:10C6C000DF34982319F08D2F8C2301C081E0DF9196
:10C6D000CF911F9108955093E3344093E2347093C7
:10C6E000DE346093DD349093E1348093E03481E074
:10C6F00001C0880F2A95EAF78093DF340C942363F6
:10C70000CF93DF93C82FDFB7F894E091E234F09134
:10C71000E33480819091DF34892B808383E090E043
:10C720000E94EC62CC2351F0E091E234F091E334CA
:10C7300080819091DF3490959823908387E190E0F9
:10C740000E94EC62E091E034F091E13480819091BC
:10C75000DF34892309F4C0E089E590E00E94EC62AF
:10C76000E091E234F091E33480819091DF34909550
:10C7700098239083DFBF8BE390E00E94EC628C2FC4
:10C78000DF91CF910895CF93DF93C82FD8E08C2FFE
:10C7900081700E948063C6958111C068D150B9F73D
:10C7A0008C2FDF91CF9108958FEF0C94C363DF92AC
:10C7B000EF92FF920F931F93CF93DF93E82EEB013D
:10C7C0000E94236381112FC080EF0E94C363F12C6C
:10C7D00010E488EFD82ED10E81E00E948063082FEC
:10C7E00081E00E948063882319F0002361F01DC05E
:10C7F000011109C01E1528F0888180FF04C0E116D0
:10C8000011F0F12E01E0802F0E94806398819695AF
:10C8100001119068988311501D11DECF21961111DE
:10C82000D8CF8F2D03C08FEF01C08EEFDF91CF9156
:10C830001F910F91FF90EF90DF900895FF920F935B
:10C840001F93CF93DF93F82EEB010E942363209771
:10C8500069F085E50E94C3638E01085F1F4F8991CF
:10C860000E94C363C017D107D1F703C08CEC0E94AC
:10C87000C3638F2DDF91CF911F910F91FF900C9487
:10C88000C3630F931F93CF93DF93DB01EC9111965A
:10C890009C911197F0E0F92B803181F4BF016E7FFC
:10C8A000E3E0660F771FEA95E1F716969C911697DD
:10C8B000ECE0F0E0E91BF109E60FF71FF7FF07C016
:10C8C00091E0EA019883F195E195F10902C0EA014E
:10C8D0001882883279F414968C91982F907690363D
:10C8E00049F086FF02C0EE7F05C085FF02C0EC7FE5
:10C8F00001C0E87FCF0144E0969587954A95E1F71E
:10C90000D9018C93EF70E801E88380E0DF91CF914B
:10C910001F910F9108950F931F93CF93DF93EC0115
:10C920008B01B80188810E94D763888381508D3F35
:10C9300030F4F8018081883211F0803191F7DF9175
:10C94000CF911F910F910895CF93DF93EC010E9437
:10C950002363BE0184EB0E941E6481E00E94806319
:10C96000C82F0E94236381E0C11101C080E0DF91E4
:10C97000CF9108951F93CF93DF9300D0CDB7DEB74B
:10C98000182F69837A830E9423630E94F26269816F
:10C990007A81882341F084E40E941E64113029F0DA
:10C9A0000E94FB6202C082E001C080E00F900F9005
:10C9B000DF91CF911F9108954F925F926F927F9276
:10C9C0008F929F92AF92BF92CF92DF92EF92FF929F
:10C9D0000F931F93CF93DF93CDB7DEB729970FB691
:10C9E000F894DEBF0FBECDBF6C015B014A01890127
:10C9F0000E942363B6018EEB0E941E64CE01019655
:10CA00007C013E019AE0690E711C27010E94D463EB
:10CA1000F70181937F01E615F705C1F769E070E042
:10CA2000C2010E94777E811109C09401A501B20163
:10CA3000F60180810E94416480E001C083E0299674
:10CA40000FB6F894DEBF0FBECDBFDF91CF911F911F
:10CA50000F91FF90EF90DF90CF90BF90AF909F909D
:10CA60008F907F906F905F904F9008955F926F923C
:10CA70007F928F929F92AF92BF92CF92DF92EF926E
:10CA8000FF920F931F93CF93DF93CDB7DEB7299714
:10CA90000FB6F894DEBF0FBECDBF582E6B015A0102
:10CAA000890160E070E08EEB0E941E64CE01019669
:10CAB0007C014E019AE0890E911C37010E94D463DB
:10CAC000F70181937F01E815F905C1F769E070E08E
:10CAD000C3010E94777E811108C09501A601B301B0
:10CAE000852D0E94416480E001C083E029960FB645
:10CAF000F894DEBF0FBECDBFDF91CF911F910F9194
:10CB0000FF90EF90DF90CF90BF90AF909F908F906D
:10CB10007F906F905F9008950F931F93CF93DF9353
:10CB2000CDB7DEB728970FB6F894DEBF0FBECDBFE6
:10CB3000182F062F98E0ECE1F3E0DE01119601904A
:10CB40000D929A95E1F7242F332727FD309541E781
:10CB500052E0249FC001259F900D349F900D112419
:10CB600064E670E00E949592CB0144E6049F800D3C
:10CB7000911D1124FE013196AE01475F5F4F619117
:10CB800070E02617370711F4019603C0E417F50784
:10CB9000B1F7112319F091958195910928960FB657
:10CBA000F894DEBF0FBECDBFDF91CF911F910F91E3
:10CBB0000895EF92FF920F931F93CF93DF93CDB71A
:10CBC000DEB72B970FB6F894DEBF0FBECDBFF82EA1
:10CBD000E92E682F792F88E08F0D0E94BA64882390
:10CBE00019F084E391E243C066E471E48FE090E0E1
:10CBF0000E9444668E01075F1F4F9801AE01465F99
:10CC00005F4FBE01655F7F4F8F2D9E2D0E94DC64BC
:10CC10008111E7CF88E0ECE1F3E0DE0111960190AD
:10CC20000D928A95E1F7498521E732E0429FC001E4
:10CC3000439F900D112464E670E00E9495928A85CE
:10CC400094E6899F600D711D1124FE01319681913A
:10CC5000481303C06F5F7F4F03C0E017F107B9F7B8
:10CC60008B85882319F0719561957109CB012B96FD
:10CC70000FB6F894DEBF0FBECDBFDF91CF911F91ED
:10CC80000F91FF90EF900895DC01CB018115910584
:10CC9000A105B10529F081509040A040B040D9F7DE
:10CCA00008959B01AC011092B90060E072E18AE73F
:10CCB00090E00E94A99220513109410951095695ED
:10CCC0004795379527952093B800089594EA909357
:10CCD000BC0040EA56E861E070E09091BC0097FD2E
:10CCE0000BC0415051096109710941155105610598
:10CCF000710599F781E008959091B900987F983077
:10CD000011F09031B9F78093BB0084E88093BC00A8
:10CD100080EA96E8A1E0B0E02091BC0027FD08C0C1
:10CD20000197A109B1090097A105B105A9F7E2CFC3
:10CD30008091B900887F883111F08034D9F680E085
:10CD4000089524EA34E844E92093BC009091BC00A3
:10CD500097FFFCCF9091B900987F983011F09031F7
:10CD600099F78093BB003093BC009091BC0097FF73
:10CD7000FCCF9091B900987F903211F0983539F43A
:10CD80004093BC009091BC0094FDFCCFDDCF089592
:10CD90000C94666684E98093BC008091BC0084FD9D
:10CDA000FCCF08958093BB0084E88093BC00809101
:10CDB000BC0087FFFCCF9091B900987F81E098324A
:10CDC00009F480E0089584EC8093BC008091BC005D
:10CDD00087FFFCCF8091BB00089584E88093BC005E
:10CDE0008091BC0087FFFCCF8091BB000895E0E1FB
:10CDF000DC01FD91CD01F0933F01E150C9F7809135
:10CE00003C018F7D80933C0180913C01877F809322
:10CE10003C01FB0180E1919190933E018150D9F753
:10CE200080913C01806880933C0180913D0180FFAE
:10CE3000FCCF4051510980913C01806280933C01BC
:10CE400080913C01877F80933C01141615069CF469
:10CE5000FB0180E1919190933E018150D9F780913F
:10CE60003C01806880933C0180913D0180FFFCCFB4
:10CE700040515109EACFF90180E190913E0191932F
:10CE80008150D9F781E090E008950F931F93CF93DD
:10CE9000DF93EC018CE70E94A1668CE70E94D266CA
:10CEA0008E01005F1F4F89910E94D266C017D10783
:10CEB000D1F7DF91CF911F910F910C94CA66813009
:10CEC00019F440E050E002C040EC50E060E070E057
:10CED0008CE790E00C949913813019F44EE050E007
:10CEE00002C048E050E060E070E08CE790E00C9415
:10CEF000991341E050E060E070E08CE790E00E9420
:10CF000099136AE67AE080E090E00C94446648E386
:10CF100050E060E070E08CE790E00E94991349E3F4
:10CF200050E060E070E08CE790E00E94991344E1EB
:10CF300050E060E070E08CE790E00E94991348E7D1
:10CF400050E060E070E08CE790E00E9499134EE5BD
:10CF500050E060E070E08CE790E00E9499134DE6AD
:10CF600050E060E070E08CE790E00E9499136CE183
:10CF70007AE186E090E00E9444664CE050E060E098
:10CF800070E08CE790E00E94991341E050E060E08F
:10CF900070E08CE790E00E94991346E050E060E07A
:10CFA00070E08CE790E00E9499136AE67AE080E0F6
:10CFB00090E00C944466CF93DF93CDB7DEB7A29791
:10CFC0000FB6F894DEBF0FBECDBF81E1ECEBF9E008
:10CFD000DE01529601900D928A95E1F781E1EDEC28
:10CFE000F9E0DE01119601900D928A95E1F70E9419
:10CFF0008767CE0142960E94456782E00E945F6784
:10D000006AE67AE080E090E00E944466CE010196F4
:10D010000E94456760E17EEA88E290E00E944466F3
:10D0200080E00E946C6760E17EEA88E290E00E9406
:10D0300044664EE050E060E070E08CE790E00E94D3
:10D040009913A2960FB6F894DEBF0FBECDBFDF9145
:10D05000CF910895CF92DF92EF92FF920F931F939B
:10D06000CF93DF9300D01F92CDB7DEB7F82E042FF9
:10D07000122F213031F0223031F0243031F02830BD
:10D0800031F090E005C091E003C092E001C093E070
:10D090000C3059F00E3011F4946007C0003111F4D7
:10D0A000986003C0023109F49C60613059F062302D
:10D0B00011F4906207C0633011F4906403C06430CF
:10D0C00009F490669068692F70E023E030E0AE01CB
:10D0D0004F5F5F4F8F2D90E00E94B01369E07AE1BF
:10D0E00080E090E00E9444668F2D8160F82E0E94BF
:10D0F00066660E94E36689830E94E3668A83023142
:10D1000019F40E94E3668B830E94E36687FDF1CFEA
:10D110000E94ED660E94CA6669E07AE180E090E0D4
:10D120000E9444668F2D0E9466660E94E366898392
:10D130000E94E3668A83023119F40E94ED668B83B4
:10D140000E94ED660E94CA6639812A81023149F542
:10D15000832F90E0A0E0B0E04B817727662731FF76
:10D160000EC030E0322F2227620F731F811D911DE8
:10D17000640F711D811D911D8C6F9F6F0BC030E07E
:10D18000322F2227620F731F811D911D640F711DA5
:10D19000811D911D0E94C38F20E83FEF4FEF57E4A0
:10D1A00020C0632F70E0762F6627620F711D8827DD
:10D1B00077FD8095982F0E94C38F0C3029F420E0D2
:10D1C00030EE4FEF54E40DC00E3029F420E038EF7C
:10D1D0004FEF55E406C0003131F420E03EEF4FEF51
:10D1E00056E40E94248F2FE632E143E050E40E948F
:10D1F000A5916B017C01612F70E080E090E00E94BE
:10D20000C38F9B01AC01C701B6010E94248F0F9010
:10D210000F900F90DF91CF911F910F91FF90EF90A2
:10D22000DF90CF900895E6E4F1E080812081908145
:10D230003081829586958695837022952F70822BFA
:10D24000832B92959F70892B08950F931F93CF93F3
:10D25000DF9300D0CDB7DEB746E06CE080E00E94FF
:10D26000556C89E18093C4001092C50082E08093E0
:10D27000C00080E00E94E26C0E94816B84B784B79A
:10D2800084B784B784B7E4E6FDE322E432E4318373
:10D2900020833A968DB79EB70A97E817F907B8F337
:10D2A0008EED99E09F938F938AE692E19F938F93FF
:10D2B0000E9472990E94BA7A0E94755A60E070E0EA
:10D2C00084E992E00E941D5B0E94515EE09124037C
:10D2D000F091250309950E94136990E00E94F67A67
:10D2E000CE0101960E94B66A0F900F900F900F909A
:10D2F000882341F08AE492E19F938F930E94729970
:10D300000F900F90CE0101960E94E4580E94C46ACB
:10D310008C010E94C06AAE014F5F5F4FB8010E944E
:10D32000AC6F0E94306A0E948D6F0E94C86A0E9492
:10D33000E6708DE392E19F938F930E9472998A81A8
:10D340001F928F9309E312E11F930F930E9472992A
:10D3500089811F928F931F930F930E94729987E385
:10D3600092E19F938F930E9472990E94FA7AE091C2
:10D370006103F09162030995E0915303F091540326
:10D380000995E0913A03F0913B0309950E94ED70F5
:10D39000182F0E948A6F1F921F931F928F93809164
:10D3A00060038F9380915F038F93809152038F93DB
:10D3B000809151038F938CE192E19F938F930E9410
:10D3C0007299E0916B03F0916C030FB6F894DEBF95
:10D3D0000FBECDBF309791F00995BC0180E890E079
:10D3E0000E9481927F936F9389E092E19F938F9344
:10D3F0000E9472990F900F900F900F9087E092E12A
:10D400009F938F930E94729960E070E08AEE92E0A1
:10D410000E941D5B8EEF92E00E94CA798FEF91E12E
:10D420009F938F930E9472990F900F900F900F907F
:10D430000F900F90DF91CF911F910F9108957F93DF
:10D440006F939F938F9389EF91E19F938F930E94A6
:10D4500072990F900F900F900F900F900F9008956A
:10D460001F93CF93DF93CDB7DEB7A0970FB6F89495
:10D47000DEBF0FBECDBF83E690E00E94DE9A182F7C
:10D48000282F35EF380F303108F0982F9095291755
:10D4900009F461C085E892E19F938F930E9472998D
:10D4A000EAECF2E10F900F90DE01119684918D93DA
:10D4B000319682E1E23DF807C9F7F89448E050E080
:10D4C0006FE770E0CE0101960E94E49AECEBF2E186
:10D4D000DE01119684918D93319682E1EA3CF80742
:10D4E000C9F74EE050E061E770E0CE0101960E947E
:10D4F000E49AE2EBF2E1DE01119684918D9331968C
:10D5000082E1EC3BF807C9F74AE050E067E670E0DB
:10D51000CE0101960E94E49A6DEC7BEA81E690E0F0
:10D520000E94FC9A60E070E08FE590E00E94FC9A17
:10D5300060E08EE590E00E94EE9A60E070E085E6A3
:10D5400090E00E94FC9A1AE16AE175EE83E690E0B1
:10D550000E94FC9A7894812FA0960FB6F894DEBFB3
:10D560000FBECDBFDF91CF911F910895F89442E097
:10D5700050E06FE770E00E94C69A789480E00895CA
:10D5800081E690E00C94DE9A8FE590E00C94DE9AB0
:10D590008EE590E00C94D69A4091F2345091F33499
:10D5A0006091F4347091F53490E0A0E0B0E0480F61
:10D5B000591F6A1F7B1F4093F2345093F3346093DA
:10D5C000F4347093F5344091EE345091EF3460911F
:10D5D000F0347091F134480F591F6A1F7B1F40933C
:10D5E000EE345093EF346093F0347093F134209123
:10D5F00092362223A1F04091EA345091EB346091AD
:10D60000EC347091ED34480F591F6A1F7B1F409313
:10D61000EA345093EB346093EC347093ED34089516
:10D620001F920F920FB60F9211240BB60F922F93E9
:10D630003F934F935F936F937F938F939F93AF939A
:10D64000BF93EF93FF938091FA139091FB13019690
:10D650009093FB138093FA138091F9138F5F80935B
:10D66000F9138038A9F41092F9138091F234909153
:10D67000F334A091F434B091F5340196A11DB11D9D
:10D680008093F2349093F334A093F434B093F53450
:10D69000809192368823E1F08091F8138F5F809318
:10D6A000F8138038A9F41092F8138091EA3490911D
:10D6B000EB34A091EC34B091ED340196A11DB11D75
:10D6C0008093EA349093EB34A093EC34B093ED3430
:10D6D0000E94AD5D892B11F00E94C05CFF91EF911B
:10D6E000BF91AF919F918F917F916F915F914F917A
:10D6F0003F912F910F900BBE0F900FBE0F901F9078
:10D700001895F8941092B60016BC83EF87BD82E09E
:10D7100084BD94E095BD95B395BB80936E007894DD
:10D7200008958091FA139091FB132091FA13309190
:10D73000FB1382179307A9F70895009751F022E38E
:10D7400030E000002150310921153105D1F7019752
:10D75000F4CF08950F931F93CF93DF93EC010E94B2
:10D76000916B8C010E94916B801B910B8C179D0714
:10D77000C8F3DF91CF911F910F91089508950F93F2
:10D780001F936091F2347091F3348091F43490914E
:10D79000F5340091F2341091F3342091F434309147
:10D7A000F534601771078207930759F71F910F919E
:10D7B00008951F920F920FB60F9211241092C0027B
:10D7C0000F900FBE0F901F9018951F920F920FB6DB
:10D7D0000F9211240BB60F922F933F934F935F93A9
:10D7E0006F937F938F939F93AF93BF93EF93FF9329
:10D7F000E091B602F091B7028081E091C102F09110
:10D80000C202309709F00995FF91EF91BF91AF9156
:10D810009F918F917F916F915F914F913F912F9148
:10D820000F900BBE0F900FBE0F901F9018951F9278
:10D830000F920FB60F9211241092CD020F900FBECF
:10D840000F901F9018951F920F920FB60F921124F0
:10D850000BB60F922F933F934F935F936F937F93EA
:10D860008F939F93AF93BF93EF93FF93E091C30286
:10D87000F091C4028081E091CE02F091CF02309706
:10D8800009F00995FF91EF91BF91AF919F918F9111
:10D890007F916F915F914F913F912F910F900BBEB0
:10D8A0000F900FBE0F901F9018959DE0899FF0017B
:10D8B0001124EA54FD4FA281B3811C92A481B58149
:10D8C0006C93A681B78188ED8C93A085B1854C932C
:10D8D00012861486138608959DE0899FF001112415
:10D8E000EA54FD4F81E08287A081B1816C933A9622
:10D8F00080818111FDCF08951F93CF93DF93182F5F
:10D90000EB01FE018491882339F0FE016491812F9F
:10D910000E946C6C2196F5CFDF91CF911F910895F5
:10D920001F93CF93DF93182FEB018881882369F031
:10D930008A3021F46DE0812F0E946C6C69916D300A
:10D94000A1F3812F0E946C6CF0CFDF91CF911F91DA
:10D950000895CF93DF93CDB7DEB79E01285F3F4F89
:10D960004E815F8160E470E08CEF93E10E942F9A1A
:10D970006CEF73E18D810E94906CDF91CF910895DF
:10D98000CF93C82F8A3031F46DE080913C140E940F
:10D990006C6C02C08D3029F06C2F80913C140E9479
:10D9A0006C6C80E090E0CF9108959DE0899FF0013C
:10D9B0001124EA54FD4F748763870895682F80E02F
:10D9C0000C946C6C80933C1488EA92E090935F3DD9
:10D9D00080935E3D089584B7877F84BF88E10FB64A
:10D9E000F89480936000109260000FBE08952FE0BD
:10D9F00088E190E00FB6F894A895809360000FBE80
:10DA0000209360000895A895089588E10FB6F894D2
:10DA100080936000109260000FBE0895F89428E093
:10DA200088E190E00FB6F894A895809360000FBE4F
:10DA300020936000FFCF8091FD348091FD3490E011
:10DA4000089540E06FE181E491E00C948272E9E393
:10DA5000F1E0808180818D7F80838DE090E001976F
:10DA6000F1F723E040E06FE182E491E00E948C72E4
:10DA700083E090E00197F1F708959091390191FDCD
:10DA80000AC0282F803108F02FE040E06FE085E4E5
:10DA900091E00C948C7208958091390181FD0EC043
:10DAA00040E06FE181E491E00E948272282F2F7E96
:10DAB00081E090E0213021F080E0089580E090E066
:10DAC00008958091390181FD10C040E06FE181E44B
:10DAD00091E00E9482728F3131F0982F9F7E915099
:10DAE00081E0923018F480E0089581E008950E946A
:10DAF000616D8823E1F30895CF93DF93C82F0E94CF
:10DB0000776D0E94216DD82FC81789F1C83019F49C
:10DB10000E94276D25C0C93121F4863189F429E09E
:10DB200005C0C63169F4893159F426E040E06FE15F
:10DB300082E491E00E948C72E3E0F0E03197F1F72B
:10DB40002C2F40E06FE182E491E00E948C72D8308B
:10DB500019F4E9E6F1E002C0E3E0F0E03197F1F713
:10DB60000E94216D8C1719F083E490E002C080E4DC
:10DB700090E0DF91CF9108950E94776D10929236D8
:10DB80000E94276D809139018260809339018091D4
:10DB900015378823D9F18091940090919500409198
:10DBA00026375091273784179507A0F48091F236D5
:10DBB0009091F336A091F436B091F5368C57914E92
:10DBC000AF4FBF4F8093F2369093F336A093F43665
:10DBD000B093F5362091940030919500241B350BBD
:10DBE0008091F2369091F336A091F436B091F536EB
:10DBF000820F931FA11DB11D8093F2369093F336CF
:10DC0000A093F436B093F5361092153780911737FC
:10DC10008823D9F1809194009091950040912A3702
:10DC200050912B3784179507A0F48091FA36909184
:10DC3000FB36A091FC36B091FD368C57914EAF4F1C
:10DC4000BF4F8093FA369093FB36A093FC36B09387
:10DC5000FD362091940030919500241B350B809166
:10DC6000FA369091FB36A091FC36B091FD36820FCA
:10DC7000931FA11DB11D8093FA369093FB36A0939C
:10DC8000FC36B093FD361092173708958091923686
:10DC9000882381F08091C014811104C00E94616DBD
:10DCA000811106C081E08093BE1481E090E0089568
:10DCB0000E94BC6D80E090E0089580919400909166
:10DCC000950090932B3780932A3721E020931737C4
:10DCD0008091390181FD08C08091390181FD1AC010
:10DCE00086E10E947C6D16C020939136809194004D
:10DCF000909195009093273780932637209315377E
:10DD0000809139018D7F8093390180919136811105
:10DD1000FCCFE2CF81E080939236089580919236D5
:10DD200081110AC08091C014882321F081E0809382
:10DD3000BF1402C00E945D6E81E090E008951F93C1
:10DD4000CF93DF931F92CDB7DEB78FB789838091D2
:10DD5000C014811126C0F89480919236882351F026
:10DD60008091390181FD1BC00E94616D8823B9F04B
:10DD700080E003C00E948E6E81E02091470191E017
:10DD80002E3008F090E0192F119581110E94466EF7
:10DD9000107429F089818FBF81E090E004C08981EF
:10DDA0008FBF80E090E00F90DF91CF911F91089599
:10DDB0008091BF14882321F00E945D6E1092BF14E1
:10DDC0008091BE14882321F00E94BC6D1092BE1475
:10DDD0001092C01408950F931F93AB0121E020937C
:10DDE000C0140091D6361091D7362091D836309194
:10DDF000D9360F5F1F4F2F4F3F4F0093D6361093EA
:10DE0000D7362093D8363093D93622E0260F27FF15
:10DE10000CC080918F3690919036019690939036F9
:10DE200080938F360FEF1FEF07C0BC018DE394E1A5
:10DE30000E94AB9800E010E00E94D86EC8011F91CC
:10DE40000F9108958093C21408950E94216D82302D
:10DE500011F0823111F480E0089581E00895089571
:10DE60008FEF80934E0122E044E060EF8CE691E07A
:10DE70000E948C7225E041E06EE08CE290E00E940E
:10DE80008C7280E880936F018091460180936D01D0
:10DE900021E045E060E284E491E00C948C728DEF27
:10DEA00093E00197F1F70E94787210920635109274
:10DEB000883510920A361092053510920435E9E340
:10DEC000F1E080818E7F808380818D7F80838DE0F3
:10DED00090E00197F1F780818160808323E040E04A
:10DEE0006FE182E491E00E948C728DEF93E00197E4
:10DEF000F1F780915D0180915E010E94306F60E0DA
:10DF000070E080ED92E00E941D5B0E945D6E81E0FA
:10DF100090E008958091C1140895CF93DF931F92EC
:10DF2000CDB7DEB789830E94776D89818093C11454
:10DF3000282F40E06FE188E491E00F90DF91CF91CE
:10DF40000C948C720E948D6F8091390181FD03C009
:10DF500086E00C947C6D0895FA01809362019093A1
:10DF6000630160936001709361013097C1F080811B
:10DF700080936B01818180936A0182818093690122
:10DF80008381809368018481809367018581809378
:10DF9000660186818093650187818093640108957D
:10DFA00080ED92E00E943E5B81E08093FD348091A1
:10DFB000FE349091FF3401969093FF348093FE34A9
:10DFC00081E090E008958091053592E8899FF00105
:10DFD0001124EA5FFA4C10828F5F833018F480932B
:10DFE000053502C010920535E091053582E8E89FBD
:10DFF000F0011124EA5FFA4C808181110C94D06FFA
:10E000001092FD3408951F93CF93DF93209105352F
:10E0100012E8129F90011124D901AA5FBA4C4C91C9
:10E02000411103C00E94E36F93C05091390151FD2B
:10E030008FC050919236552309F48AC047FF16C00D
:10E040000E94E36F8091C6369091C736A091C83682
:10E05000B091C9360196A11DB11D8093C63690932B
:10E06000C736A093C836B093C93672C04330B0F4F7
:10E070000E94E36F8091C2369091C336A091C4365E
:10E08000B091C5360196A11DB11D8093C236909303
:10E09000C336A093C436B093C5365AC050E0EA01E7
:10E0A00022976C177D07B0F40E94E36F8091BE3613
:10E0B0009091BF36A091C036B091C1360196A11D96
:10E0C000B11D8093BE369093BF36A093C036B093F7
:10E0D000C1363EC0B901695F7A4C0E94AB98E091AD
:10E0E00005351E9FF0011124EA57FA4C8081809378
:10E0F000F6340E94E36F809147018093F73490914A
:10E10000FC34992311F0891710F48093FC3460914A
:10E11000F73470E084E00E94C8626091F63470E0E9
:10E1200083E00E94C8624091DA365091DB366091FC
:10E13000DC367091DD364F5F5F4F6F4F7F4F4093FE
:10E14000DA365093DB366093DC367093DD3602C0EE
:10E15000C0E0D0E0CE01DF91CF911F910895CF9321
:10E16000DF93EC01888199810097E9F08730954031
:10E1700021F01982188283E026C06238C1F410921F
:10E18000FD340E944F620E94B66160E870E00E9418
:10E190000370181619066CF40E94B161E0916503D2
:10E1A000F0916603099587E095E09983888381E083
:10E1B0000AC08091FA349091FB3401969093FB341D
:10E1C0008093FA34F0CFDF91CF91089591E090934E
:10E1D000C0140E943D6D0C94D86E8091390181FD70
:10E1E00006C040E06FE085E491E00C94827280E12B
:10E1F00008950F931F93CF93DF93182F21E020935F
:10E20000C014009192368091390181FF16C080912F
:10E210009400909195009093273780932637209310
:10E22000153720939136809139018D7F8093390184
:10E23000809191368111FCCF00E00E94776D809132
:10E240009236882309F43FC0809117378823D9F18B
:10E250008091940090919500E0912A37F0912B37AE
:10E260008E179F07A0F44091FA365091FB366091CB
:10E27000FC367091FD364C57514E6F4F7F4F409397
:10E28000FA365093FB366093FC367093FD3620913E
:10E290009400309195002E1B3F0B4091FA3650911F
:10E2A000FB366091FC367091FD36420F531F611DA5
:10E2B000711D4093FA365093FB366093FC36709391
:10E2C000FD36109217378091390181FD03C089E135
:10E2D0000E947C6D86E00E94D362892B51F00E94DF
:10E2E000ED70C82F86E00E94D36281500E943D6D80
:10E2F00002C0C0E0D0E020919400309195003093AE
:10E3000029372093283781E080931637F89480913D
:10E310003901826080933901809139018D7F80932A
:10E32000390162E0610F8DE394E10E94BB72789441
:10E3300020918C3630918D362F5F3F4F30938D3644
:10E3400020938C360E94776D45E060EE82E491E088
:10E350000E948272182F86E00E94D362892B19F0E6
:10E360008C2F0E943D6D002319F00E945D6E02C04B
:10E370000E94BC6D809116378823D9F1809194005A
:10E3800090919500E0912837F09129378E179F07DB
:10E39000A0F44091F6365091F7366091F8367091BE
:10E3A000F9364C57514E6F4F7F4F4093F63650938E
:10E3B000F7366093F8367093F936209194003091D7
:10E3C00095002E1B3F0B4091F6365091F736609129
:10E3D000F8367091F936420F531F611D711D40933D
:10E3E000F6365093F7366093F8367093F9361092FC
:10E3F000163780919236882361F0209194003091F5
:10E40000950030932B3720932A3781E0809317377C
:10E4100007C023E040E06FE182E491E00E948C724B
:10E420000E94D86E1130E9F01330A9F48091CE36F5
:10E430009091CF36A091D036B091D1360196A11DE2
:10E44000B11D8093CE369093CF36A093D036B09343
:10E45000D13612E009C0153031F0173029F411E03F
:10E4600003C010E001C013E0812F90E0DF91CF9155
:10E470001F910F910895CF93DF93EB010E94EB6EF4
:10E48000009729F4CE010E94F970009751F0209175
:10E490008F36309190362F5F3F4F309390362093D8
:10E4A0008F36DF91CF910895CF93DF93809192368D
:10E4B000811104C00E948E6ED1E001C0D0E00E94A4
:10E4C000216D863111F0813119F4C091470109C0E5
:10E4D00040E06FE186E491E00E948272C82FCC0F89
:10E4E000C80FD1110E94466E8C2FDF91CF910895F5
:10E4F0001092C4141092C314EFE6F0E080818062A1
:10E5000080830895FC018081862390E002C0959568
:10E5100087954A95E2F70895F894FC015081362FCB
:10E5200030955323042E01C0220F0A94EAF72623C4
:10E53000522B50837894089540917B01FC014193C4
:10E54000A0E8B1E050E8540F9D012F5F3F4F6C9160
:10E550006193521711F0D901F7CF4150E42FF0E049
:10E56000E058FE4F2181FC01E058FF4F2083319697
:10E5700021E02083089560938001E1E8F1E0615893
:10E580009F012F5F3F4FDC014D91CD01408362170A
:10E5900011F0F901F5CF08951F920F920FB60F9267
:10E5A00011240BB60F922F933F934F935F936F936A
:10E5B0007F938F939F93AF93BF93EF93FF9380913C
:10E5C00047018093F7348091043522E8829FC0018F
:10E5D00011248A5F9A4C0E949C72809104358F5F4F
:10E5E000833018F48093043502C0109204350E94E1
:10E5F000D06FFF91EF91BF91AF919F918F917F91DC
:10E600006F915F914F913F912F910F900BBE0F90A3
:10E610000FBE0F901F9018951F920F920FB60F927A
:10E6200011240F900FBE0F901F9018951F920F92FC
:10E630000FB60F9211240F900FBE0F901F901895D8
:10E640001F920F920FB60F9211240F900FBE0F90D2
:10E650001F9018951F920F920FB60F9211241092CF
:10E6600091360F900FBE0F901F9018951F920F922A
:10E670000FB60F921124109291360F900FBE0F908B
:10E680001F9018951F920F920FB60F9211248F931F
:10E6900081E08093FD348F910F900FBE0F901F90FB
:10E6A00018951F920F920FB60F9211241092913667
:10E6B0000F900FBE0F901F9018951F920F920FB6DC
:10E6C0000F9211248F939F938091C3149091C4143F
:10E6D00001969093C4148093C3149F918F910F90CF
:10E6E0000FBE0F901F901895CF92DF92EF92FF927E
:10E6F0000F931F93CF93DF937C018B016A0185EC0D
:10E7000094E10E94DD5BEC01009751F0EC81FD810A
:10E71000309711F0C8010995CE010E94855CF3CFB6
:10E72000A601B801C701DF91CF911F910F91FF9012
:10E73000EF90DF90CF900C9467590F931F93CF9376
:10E74000DF9300D0CDB7DEB780919A3690919B369B
:10E75000A0919C36B0919D360196A11DB11D80936C
:10E760009A3690939B36A0939C36B0939D360E9428
:10E7700007768C0185EC94E10E94DD5B009779F0CF
:10E78000DC011296ED91FC911397309729F0898363
:10E790009A8309959A8189810E94855CEFCF011542
:10E7A000110549F0C8010F900F90DF91CF911F9193
:10E7B0000F910C945E590F900F90DF91CF911F91A4
:10E7C0000F9108950E94FA7A0E944F620E942E745F
:10E7D00081E593E090939536809394360E94057678
:10E7E0002FEF31E040E05EE160E074E082E090E035
:10E7F0000C94CE75BC0185EC94E10C943D5CBC019D
:10E8000085EC94E10C94225CCF93DF93EC01409172
:10E8100096365091973660919836709199364F5F41
:10E820005F4F6F4F7F4F409396365093973660936C
:10E830009836709399360E941A76009761F00E947C
:10E84000CF61E0915503F0915603BE0184E793E751
:10E85000099581E090E0DF91CF9108958BEC94E1F0
:10E860000C94D95B0F93CF93DF93EC017B836A8386
:10E8700018865F834E83BC018BEC94E10E943D5C63
:10E88000E091C714F091C814309749F04C815D8134
:10E8900001E020E030E068858A819B810995DF9165
:10E8A000CF910F910895BC018BEC94E10C94225C04
:10E8B0000F93DC0118961C921897E091C714F09101
:10E8C000C814309759F000E020E030E040E050E01C
:10E8D00060E012968D919C91139709950F91089580
:10E8E0000F93DC01AB0114962D913C91159781E0BB
:10E8F00018968C93189715967C936E931497E091C5
:10E90000C714F091C814309739F000E061E0129616
:10E910008D919C91139709950F9108950F93DC01A8
:10E92000E091C714F091C814309771F014964D918E
:10E930005C91159701E09A0118966C9118971296C0
:10E940008D919C91139709950F910895E091C914A9
:10E95000F091CA14309709F0099408959093CA145D
:10E960008093C91408959093C8148093C714089590
:10E970008BEC94E10C94DD5BEF92FF920F931F936D
:10E98000CF93DF938C01EB017A018BEC94E10E9431
:10E99000DD5B0097D9F0DC0112962D913C91139725
:10E9A0002C173D0781F41696ED91FC91179730973F
:10E9B00069F09701AE01B801DF91CF911F910F91DE
:10E9C000FF90EF9009940E94855CE3CFDF91CF9197
:10E9D0001F910F91FF90EF9008950895CF93DF93CB
:10E9E000CEEFD4E16881798120E030E04DE055E759
:10E9F00088EE94E10E945D5E0E94F87A68817981D8
:10EA00000E94819220E030E041E255E7BC0188EDB0
:10EA100094E1DF91CF910C945D5E8091FE14909112
:10EA2000FF142091FC143091FD14880F991F2817B2
:10EA3000390708F4C9019093FF148093FE140C94D5
:10EA4000EE74CF93DF930E944F620E94B661EC0197
:10EA5000198218820E94B87428813981009719F1AF
:10EA6000FC0140854423F9F0FC0142815381F90106
:10EA7000EE0FFF1FEE0FFF1FEC0FFD1F53834283AE
:10EA8000FC01448155812F5F3F4FF901EE0FFF1FBD
:10EA9000EE0FFF1FEC0FFD1F518340833983288346
:10EAA0000E94855CD9CFC901880F991F880F991FD3
:10EAB00002960E94B16188819981892B31F08DEC99
:10EAC00094E1DF91CF910C943559DF91CF91089566
:10EAD000AF92BF92CF92DF92EF92FF920F931F936C
:10EAE000CF93DF9300D0CDB7DEB76B010E94B66144
:10EAF000FC01008111811A8309830C30110518F47F
:10EB0000E12CF12C0DC01F930F938CEF99E09F9394
:10EB10008F930E9460990F900F900F900F9021C0DB
:10EB2000E016F106F1F00E94B661F701EE0FFF1F4B
:10EB3000EE0FFF1FE80FF91FA280B3800E94B6619D
:10EB4000FFEFEF1AFF0AF701EE0FFF1FEE0FFF1F97
:10EB5000E80FF91F40815181B501C6010E94BC74C4
:10EB6000DFCF0F900F90DF91CF911F910F91FF900A
:10EB7000EF90DF90CF90BF90AF9008950F9301304A
:10EB800059F48091F8149091F9149093FF148093A4
:10EB9000FE140F910C94EE740F910895EF92FF9272
:10EBA0000F931F93CF93DF938B01EA0179014EE31B
:10EBB00053E0BC018DEC94E10E9419591093F914B3
:10EBC0000093F814D093FB14C093FA14F092FD1440
:10EBD000E092FC148EEB95E7DF91CF911F910F919E
:10EBE000FF90EF900C94B37488EE94E10E94E15E84
:10EBF00088ED94E10E94E15E8DEC94E10C94335930
:10EC00008091FE149091FF1408950C947359CF9342
:10EC1000DF93E0914203F09143030995EC010097E3
:10EC200029F06A817B8181E00E94C862CE01DF9178
:10EC3000CF9108950F931F93CF93DF93EC01E09151
:10EC40004403F091450309958C016A817B8181E041
:10EC50000E94C86281E090E0012B11F480E090E016
:10EC6000DF91CF911F910F910895E0914603F091AC
:10EC70004703099420E030E00296FC01329740817E
:10EC8000442331F0FC0131974081240F311DF4CF32
:10EC9000C9010895FC01208130E0322F22278181B3
:10ECA000282B02C0220F331F6A95E2F7832F992782
:10ECB000FA01E85BFC4F208130E08223932328E0B7
:10ECC00030E0241B350B02C0969587952A95E2F714
:10ECD00008956F927F928F929F92AF92BF92CF9240
:10ECE000DF92EF92FF920F931F93CF93DF938C01EC
:10ECF000EB016A0179012830310524F4A901B6013C
:10ED0000CE014AC0590123E0B594A7942A95E1F7B2
:10ED10004115510521F04801612C712C03C0D80127
:10ED2000FB0120C048E050E0B601CE01860D971DE2
:10ED30000E944A76F40181934F01FFEF6F1A7F0A18
:10ED40006A147B047CF3C501B7FE02C080E090E04A
:10ED5000A701477055274115510511F1080F191FDB
:10ED6000B60118C0CF018C1B9D0B8A159B051CF4A6
:10ED700081918D93F7CFC501B7FE02C080E090E08E
:10ED8000A701477055274115510551F0080F191F6C
:10ED900060E070E08C0F9D1F0E944A76F80180832E
:10EDA000DF91CF911F910F91FF90EF90DF90CF9067
:10EDB000BF90AF909F908F907F906F9008958F92AB
:10EDC0009F92AF92BF92CF92DF92EF92FF920F93FA
:10EDD0001F93CF93DF9300D0CDB7DEB70E94B6610B
:10EDE0008C0182E090E00E949461892B19F480E00C
:10EDF00090E05DC0F801818190E0982F8827208104
:10EE0000820F911D0E9484597C01009781F30E941A
:10EE1000B6614C01F7012681822F869586958695ED
:10EE200090E0422F477021E030E011F420E030E024
:10EE3000820F931F0E949461892BC9F2F70104810C
:10EE40001581C12CD12CF8018081882379F1F8013A
:10EE5000A180B12CB60133E0759567953A95E1F73D
:10EE6000A60147705527680D791D883168F0950116
:10EE7000CE0101960E946976BE016F5F7F4FF80157
:10EE800080810E94DC620DC01A8219829501CE0138
:10EE900001960E94697669817A81F80180810E94D9
:10EEA000C862CA0CDB1C0E5F1F4FCDCFC7010F908D
:10EEB0000F90DF91CF911F910F91FF90EF90DF9016
:10EEC000CF90BF90AF909F908F900895DC0150E05D
:10EED000E0E1F0E0E61BF70BE21BF30B02C0440F8E
:10EEE000551FEA95E2F78C91852B8C9311968C91A6
:10EEF0001197842B11968C9308956F927F928F9225
:10EF00009F92AF92BF92CF92DF92EF92FF920F93B8
:10EF10001F93CF93DF938C016B01EA0179012830B5
:10EF200031051CF44881C8015CC0390153E0759477
:10EF300067945A95E1F76115710521F04E01A12CF6
:10EF4000B12C03C0D801FE0127C0F40141914F014B
:10EF500028E030E0B601C8018A0D9B1D0E9466774B
:10EF6000FFEFAF1ABF0AA614B7047CF3C30177FE04
:10EF700002C080E090E0970127703327211531050A
:10EF800009F43FC0C80FD91F488150E0B601621B89
:10EF9000730B685F7F4F1CC0CF018C1B9D0B8615C8
:10EFA00097051CF481918D93F7CFC30177FE02C0C2
:10EFB00080E090E09701277033272115310509F192
:10EFC000C80FD91F488150E068E070E0621B730BE6
:10EFD00002C0559547956A95E2F760E070E0800FB2
:10EFE000911FDF91CF911F910F91FF90EF90DF90D4
:10EFF000CF90BF90AF909F908F907F906F900C9428
:10F000006677DF91CF911F910F91FF90EF90DF9086
:10F01000CF90BF90AF909F908F907F906F9008950A
:10F020006F927F928F929F92AF92BF92CF92DF9218
:10F03000EF92FF920F931F93CF93DF9300D0CDB742
:10F04000DEB78C01FC018681E82EE694E694E69416
:10F05000F12C282F277081E090E011F480E090E0FF
:10F06000E80EF91EC70102960E941862009709F483
:10F0700045C00E94BD61F8012281FC012083F80196
:10F080002381FC0121830E94BD6102965C01A701DE
:10F0900060E070E00E94B498F80104811581E12CD1
:10F0A000F12CF8018081882339F1F8018180912CBD
:10F0B000670163E0D594C7946A95E1F73701F7E0FB
:10F0C0006F227724CA0CDB1C883128F00E94E6628C
:10F0D0009401AC0108C00E94D3629A838983940191
:10F0E000AE014F5F5F4FB301C6010E947D77E80C10
:10F0F000F91C0E5F1F4FD5CF81E090E00F900F906D
:10F10000DF91CF911F910F91FF90EF90DF90CF9003
:10F11000BF90AF909F908F907F906F900895E091F7
:10F120006303F09164030994E0913C03F0913D0383
:10F130000994E0916703F09168030994E0916903F1
:10F14000F0916A03099480E090E008950895E091B9
:10F150003403F0913503099480E090E008950F9313
:10F160001F93CF93DF93CDB7DEB7E0970FB6F89438
:10F17000DEBF0FBECDBF0E9403628C010E94B6614C
:10F18000AE014F5F5F4F602F0E947F80882309F49C
:10F1900046C088A99801281B3109C9010E949461C1
:10F1A000892BE9F12E8121110CC0BE016A5E7F4FCF
:10F1B00088E10E94DC62E0915703F09158030995C1
:10F1C0002EC08A859B858D3C3BEA930711F0019602
:10F1D00031F5223019F088E090E002C082E090E042
:10F1E00001979C012F5F3F4F12161306F4F6E1E0E2
:10F1F000F0E0EC0FFD1FE80FF91F23852F3F81F38F
:10F20000BE01645F7F4F89E10E94DC6289E10E9458
:10F21000E66263EA74E30E94D258892B31F6E096E5
:10F220000FB6F894DEBF0FBECDBFDF91CF911F9117
:10F230000F910895AF92BF92CF92DF92EF92FF921B
:10F240000F931F93CF93DF93CDB7DEB7E0970FB641
:10F25000F894DEBF0FBECDBF8C016B01CE010196CD
:10F260007C0180E3F70111928A95E9F781E08983B7
:10F270008CE00E94D3628C831D821F8280910215D4
:10F2800091E0980F90930215898783E0B82EB88695
:10F290008DEC9BEA9B878A8789E10E94E66260E1A8
:10F2A00073E00E94D258892B31F082E08E838FEF79
:10F2B0008C878D8709C089E10E94E662BC01CE017E
:10F2C0000C960E94C958BE828DEC9BEA9D8B8C8B5C
:10F2D00063EA74E3CE0146960E94C9580E94B66163
:10F2E0009FA78EA70E94036288ABC7010E94787F08
:10F2F000B82E90E00E941862892B31F10E94BD6106
:10F30000BC014B2DC7010E94967FE0902A03F0902C
:10F310002B030E940D625C010E94BD61B501F701E3
:10F3200009950115110581F0009739F0019761F4F5
:10F3300041E050E064E070E004C041E050E060E093
:10F3400070E0C601F8010995E0960FB6F894DEBFAB
:10F350000FBECDBFDF91CF911F910F91FF90EF9026
:10F36000DF90CF90BF90AF9008950E94F87A80937D
:10F370000215E0913403F09135030994892B29F0AB
:10F38000E0913403F091350304C0E0913603F0912D
:10F3900037030994CF93DF93EC01899199910097FA
:10F3A00029F060E070E00E941D5BF7CFDF91CF9104
:10F3B0000895CF93DF93EC0189919991009719F00B
:10F3C0000E946F5AF9CFDF91CF910895CF93DF93C9
:10F3D000EC017B836A830E94916B99838883DF9120
:10F3E000CF910895FC018081918122813381820F28
:10F3F000931F918380830895CF93DF93EC010E9444
:10F40000916B99838883DF91CF910895CF93DF9398
:10F41000EC010E94916B28813981821B930B9C0126
:10F420002F5F3F4F81E090E04A815B814217530795
:10F4300010F080E090E0DF91CF910895CF93DF93BB
:10F44000FC01C281D38180819181C80FD91F0E94A4
:10F45000916B9E01281B390BC901DF91CF91089553
:10F46000CF93DF93ECE1F7E3CEEDD6E3A0E1B7E392
:10F470001192119219921992199219921D9287E381
:10F48000E433F807A9F7DF91CF910895CF93DF9385
:10F49000FC01E05FF84C40819C01220F331F220FDA
:10F4A000331F442301F1A0919400B0919500FC0119
:10F4B000EE0FFF1FE45EF84C80819181AD01481B87
:10F4C000590BCA01E901C252D94C488159816A815C
:10F4D0007B81480F591F611D711D488359836A83C1
:10F4E0007B83B183A083F901E252F94C6081718181
:10F4F00082819381DF91CF91089560E070E0CB012C
:10F500000895FC01EE0FFF1FEE0FFF1FE252F94CB2
:10F5100040835183628373830895CF93DF9320E107
:10F5200037E3CEEDD6E3ECE1F7E3D9018D919D0110
:10F530008823B9F040919400509195008081918189
:10F54000BA01681B790B88819981AA81BB81860FDA
:10F55000971FA11DB11D88839983AA83BB83518303
:10F56000408324963296B7E32C313B07F1F6DF91C6
:10F57000CF9108950C94077F0F931F93FC01CB014B
:10F58000409103155091041533832283158304831E
:10F5900071836083F0930415E0930315452B11F4F8
:10F5A0000E94217F80E090E01F910F91089580914B
:10F5B0000315909104150097C1F010920415109254
:10F5C0000315DC0114966D917C9115971296ED91BF
:10F5D000FC9113970995E0910315F091041530976C
:10F5E00021F0808191810C94217F08950C943E95A7
:10F5F0000C943A9582EE92E00E94545B8AED92E080
:10F600000C94545BCF93DF930E94C361892BA9F0C4
:10F610008AED92E00E94725BEC01009721F10E945A
:10F620000362998388830E94FE619B838A83CE0153
:10F6300004960E943F618CAB14C082EE92E00E945F
:10F64000725BEC01009779F002960E9451619983F8
:10F650008883BE016E547F4FCE018E579F4F0E940C
:10F66000A662CE0102C080E090E0DF91CF910895C4
:10F67000BC016E547F4F8E579F4F0C94A662CF9360
:10F68000DF93EC01BC0182EE92E00E94BC5BBE0104
:10F69000892B19F082EE92E009C08AED92E00E9477
:10F6A000BC5B892B39F0BE018AED92E0DF91CF91EE
:10F6B0000C94975BDF91CF9108950F931F93CF9395
:10F6C000DF93EC01BC0182EE92E00E94BC5B892BCF
:10F6D00091F0FE0161917191CF010E946262BE01C1
:10F6E0006E547F4FCE018E579F4FDF91CF911F9168
:10F6F0000F910C94B762BE018AED92E00E94BC5B50
:10F70000892BD1F00E944F62688179818A819B8127
:10F710000E9462628CA990E00E9418620CA910E01D
:10F720000E94BD61BE016C5F7F4FA801DF91CF9148
:10F730001F910F910C94AB98DF91CF911F910F9176
:10F740000895CF93DF93EC01BC0182EE92E00E941A
:10F75000BC5B892B19F0CE0102960CC0BE018AED6C
:10F7600092E00E94BC5B892B19F08A819B8102C0C8
:10F7700080E090E0DF91CF910895FC01808191813C
:10F780000895860F911D860F911D8E579F4F0895E6
:10F79000860F911D860F911D8E579F4FFC01808112
:10F7A00091810895089582E69BE10E94965D892BE0
:10F7B00021F082E69BE10C94835D0895E0914E1B5D
:10F7C000F0914F1B309709F0099480E00895EF9273
:10F7D000FF920F931F93CF93DF937C01EA01FC010B
:10F7E00080819181009741F08C30934071F1F70155
:10F7F0001182108283E0F2C080E024E0829FF00159
:10F800001124E05BF44E118210828F5F8430A8F3E4
:10F8100080934D1B80918812909189129093611B67
:10F820008093601B0E94685A8093343760E470E0D4
:10F8300082E69BE10E946F5D0E94F4818CE093E080
:10F84000F7019183808381E0C9C06230D9F480914F
:10F85000353790913637892B89F38091463786303A
:10F8600029F480915E3781FD0E94D37B81E00E9464
:10F8700031838091353790913637892BF9F20E9488
:10F88000F77DDCCF633060F5611114C02097B1F2D1
:10F89000D093433CC093423C83E00E9431838091EB
:10F8A000353790913637892B11F00E94DE7B0E940C
:10F8B000D37BC4CF613011F6209709F4BFCFD0932A
:10F8C0003F3CC0933E3C85E00E94318380913537B8
:10F8D00090913637892B09F4B1CF0E94DE7BAECFF1
:10F8E0006738E9F510924C1B00E51BE180914C1B39
:10F8F0008430B8F4F801828193818C179D0749F414
:10F90000808191810E94FE82F8011182108213820F
:10F9100012820C5F1F4F80914C1B8F5F80934C1B9A
:10F92000E5CFEDE5FCE3838194818C179D0719F405
:10F93000148213821082B0962CE3ED3DF20799F702
:10F94000EAEDFCE3818592858C179D0711F4158201
:10F9500014823D968DE3EC35F807A1F76FCF683838
:10F9600009F06CCFC256DB4109F068CF82E69BE11B
:10F970000E94965D892B09F461CF10924C1BE09197
:10F980004C1BE43008F05ACF20E2E29FF001112432
:10F99000EC5BF34C818D8823D9F082E69BE10E94D9
:10F9A000835D80914C1BE0E28E9FC00111248C5B33
:10F9B000934C9093433C8093423C82E00E9431837D
:10F9C0008091353790913637892B11F00E94DE7B7C
:10F9D00080914C1B8F5F80934C1BD1CFDF91CF91D7
:10F9E0001F910F91FF90EF90089590934F1B80937C
:10F9F0004E1B0895209188123091891260E0E0E555
:10FA0000FBE1643098F4408151814817590759F45B
:10FA1000428153814217530731F460934B1B11828B
:10FA200010820C94FE8234966F5FEBCF60934B1B79
:10FA3000089540E0E0E5FBE14430A8F451E0540FC4
:10FA400020813181232B61F440934A1B9183808371
:10FA50002091881230918912338322830C94188369
:10FA60003496452FE9CF40934A1B08952091881280
:10FA700030918912FC01358F248F778F668F08951E
:10FA80002091881230918912FC0132872187748776
:10FA900063870895CF93DF93EA010E94A1820097C4
:10FAA00049F02091881230918912FC013287218718
:10FAB000D487C387DF91CF9108950F931F93CF937E
:10FAC000DF9300D000D0CDB7DEB78C01AB018FEF54
:10FAD00089838A838B838C83B801CE0101960E942F
:10FAE0004A7D009719F0FC01158304830F900F9055
:10FAF0000F900F90DF91CF911F910F91089540E0EB
:10FB000050E062E08AEE92E00E940E5B109236377F
:10FB1000109235370895AC0161E08AEE92E00C94C2
:10FB2000F05AAC0160E08AEE92E00C94F05A0F9328
:10FB30001F93CF93DF938A010E942082EC010097EC
:10FB400059F080918812909189129D8F8C8F1F8F10
:10FB50000E8FCE010E94917DCE01DF91CF911F913A
:10FB60000F910895CF93DF93A091423CB091433C15
:10FB7000109719F0ED016C9605C0C0913E3CD091F4
:10FB80003F3C299680913D3C86FF22C01092491B44
:10FB900040E0E0E5FBE14430B8F420813181149687
:10FBA0008D919C9115972817390759F4828193817B
:10FBB000009739F04093491B998388831B821A82EE
:10FBC00005C034964F5FE7CF4093491B0E94D37B1B
:10FBD00088819981009741F04A815B816091343737
:10FBE000DF91CF910C940E5BDF91CF9108950F932D
:10FBF0001F93CF93DF9380914637863009F071C011
:10FC000080913537909136378115954009F069C05C
:10FC1000C4E9D2E0D0933637C093353702E0009381
:10FC20003F3714E9109340371092623710926137D2
:10FC30000E94EE8180959095909362378093613712
:10FC400010924837109247370E94DD818095909539
:10FC500090934837809347370E94DE7BD0933637A6
:10FC6000C093353700933F3710934037A091403C05
:10FC7000B091413CFD01E459FD4F8CE692E00190CA
:10FC80000D920197E1F76CE672E085E597E30E943B
:10FC90009C81809139378093553780913A37809392
:10FCA000563780913B378093573780913C3780930C
:10FCB000583710926237109261370E94EE8180951A
:10FCC00090959093623780936137109248371092E5
:10FCD00047370E94DD8180959095909348378093B7
:10FCE0004737DF91CF911F910F910C94DE7BFC0180
:10FCF000680F791F80E048E1E617F70781F021914E
:10FD000098E0322F3827532F517030FD8427869585
:10FD1000513009F480682695915099F7EDCF0895F8
:10FD20001F920F920FB60F9211240BB60F922F93C2
:10FD30003F934F935F936F937F938F939F93AF9373
:10FD4000BF93EF93FF9380919400909195009093CF
:10FD500021378093203781E08093123780917100A2
:10FD6000807D809371000E94D77A8091123788231A
:10FD7000D9F1809194009091950040912037509155
:10FD8000213784179507A0F48091E6369091E736E5
:10FD9000A091E836B091E9368C57914EAF4FBF4FE6
:10FDA0008093E6369093E736A093E836B093E93631
:10FDB0002091940030919500241B350B8091E636FC
:10FDC0009091E736A091E836B091E936820F931F03
:10FDD000A11DB11D8093E6369093E736A093E836D7
:10FDE000B093E93610921237FF91EF91BF91AF9126
:10FDF0009F918F917F916F915F914F913F912F9143
:10FE00000F900BBE0F900FBE0F901F9018959FB7CD
:10FE1000F894E1E7F0E08081807D808388B38F6291
:10FE200088BB10929000E1E9F0E0108210929200FD
:10FE300010929500109294008081856080839FBF0E
:10FE400008952FB7F894909399008093980088B301
:10FE50008F6288BBE1E7F0E08081826080832FBF02
:10FE60000895CF93DF93FC01DB0185E0EB0119924C
:10FE70008A95E9F78581837011F082E08C93878100
:10FE8000837021F082E012968C93129785818370A3
:10FE900081F08781837069F0238934898185928517
:10FEA0002817390731F481E0848312961C92129747
:10FEB00001C0148285818370823021F0833021F06B
:10FEC00080E003C082E001C088E011968C93119716
:10FED00087818370823021F0833021F080E003C07D
:10FEE00082E001C088E013968C93DF91CF91089552
:10FEF000CF93DF9300D000D01F92CDB7DEB7BE0105
:10FF00006F5F7F4F0E94317F89819A81890F8D5F5A
:10FF10009B81890F9C81890F9D81890F0F900F9084
:10FF20000F900F900F90DF91CF9108954F925F92B5
:10FF30006F927F928F929F92AF92BF92CF92DF92F9
:10FF4000EF92FF920F931F93CF93DF9300D000D0D7
:10FF500000D0CDB7DEB78C017B01BE016F5F7F4F54
:10FF60004E830E94317FB981AA815B804C808B2FA8
:10FF700090E003962A2F30E0820F931F850D911D8C
:10FF8000642D70E0860F971F5D81850F911D4E8156
:10FF900050E0481759070CF49AC0F801818180FBA2
:10FFA000662460F8712C43E0660C771C4A95E1F7F3
:10FFB000828180FB882480F8912C54E0880C991C65
:10FFC0005A95E1F7862880818770882A838180FB93
:10FFD000AA24A0F8B12C85E0AA0CBB1C8A95E1F7F5
:10FFE0008A28848180FBCC24C0F8D12C96E0CC0CEC
:10FFF000DD1C9A95E1F78C28F7018082F801458194
:020000021000EC
:100000004370F4E04F9FA0011124F80186818370B2
:10001000F0E18F9FC0011124482BF8018781F0E4A3
:100020008F9FC0011124482BF7014183F80180857F
:10003000F7018283B23059F4F8018185F701838397
:10004000F8018285F701848395E0C92E02C083E020
:10005000C82EB0E080E090E0200F311FDB2EDC0CDA
:100060000197BA1761F0A901480F591FFA01B3842B
:10007000A7014D0D511DFA01B082BF5FEFCF9D2D3D
:10008000F2E05F120EC0D701AD0DB11DF8018389FA
:100090008C9381E08D0DD701A80FB11D9E5F8489DF
:1000A0008C9340E020E030E0060F171F842F890F6B
:1000B00021503109441561F0D801A20FB31F5596A4
:1000C0005C91D701A80FB11D5C934F5FEFCF80E02B
:1000D00026960FB6F894DEBF0FBECDBFDF91CF914D
:1000E0001F910F91FF90EF90DF90CF90BF90AF9056
:1000F0009F908F907F906F905F904F900895BF92E8
:10010000CF92DF92EF92FF920F931F93CF93DF93E3
:100110007C01D62EEA0182E0861708F0B1C0F70113
:10012000808186FBBB24B0F89181292F26952695E6
:100130002370C92EC294C694C69453E0C522382FAA
:100140003770388383FB332730F9398384FB3327B7
:1001500030F93A8385FB882780F98B83BC822D8315
:10016000892F829583708E83CF8282818887222314
:1001700089F13381848190E0982F8827830F911D26
:100180009A87898787010B5F1F4F223071F460E1E6
:1001900073E0CE010B960E94C958F70186818B87C8
:1001A00085818C870E5F1F4F20C02330F1F4F7014B
:1001B0003D9680E090E03E2F2F2F4291DE01A80F68
:1001C000B91F1B964C93019688309105B1F7032F08
:1001D000122F0BC087010D5F1F4F60E173E0CE014E
:1001E0000B960E94C9581A861986CC20B9F1B11015
:1001F0000DC0F8012081818190E0982F8827820F1F
:10020000911D9C8B8B8B0E5F1F4F04C089859A8537
:100210009C8B8B8BF2E0CF120EC060E173E0CE01BD
:1002200045960E94C958F80181818D8B80818E8B03
:100230000E5F1F4F1BC0F3E0CF1218C0085F1F4FA7
:10024000F80180E090E02291DE01A80FB91F5596D9
:100250002C93019688309105B1F708C060E173E0F6
:10026000CE0145960E94C9581C8A1B8AC8018E1966
:100270009F092D2D281B2FA71EA70DA7D81608F400
:1002800080E0DF91CF911F910F91FF90EF90DF9071
:10029000CF90BF900895FB0141505109460F571F61
:1002A000E417F50778F4208130E0322F22276181AE
:1002B000260F311D820F931F8217930708F40196B2
:1002C0003296EECFE417F50751F4208130E0322F5B
:1002D0002227820F931F8217930708F4019608952F
:1002E000CF93DF93C0914037D0E0649720913F37A0
:1002F00030E0322F2227C20FD31F48E050E069E4DC
:1003000077E39E01280F311DC9010E944B81AE0188
:1003100061E577E30E944B81009721F098278927B8
:10032000982702C08FEF9FEFDF91CF9108959093B0
:100330007B1B80937A1B0895FC015381560F5093C9
:100340003C37872F99274281480F40933B37A18143
:10035000A0933A37E081E0933937242F30E0281713
:10036000390748F481E08A0F80933A37811103C03E
:10037000EF5FE0933937852F90E07727861797074F
:1003800088F44F5F40933B3741110CC080913A375E
:100390008F5F80933A37811105C0809139378F5F25
:1003A000809339370895AB01BC0180E090E00E9452
:1003B0004B81982789279827089544E150E06DE301
:1003C00077E380E090E00E944B81009721F098272E
:1003D0008927982708958FEF9FEF089586E00C9462
:1003E000708181E10C94708180E0E82FF0E0EE0FE5
:1003F000FF1FEC53F34C118210828F5F8430A8F3FF
:1004000080E090E2899FF0011124EC5BF34C118EA7
:100410008F5F8430B0F380E094E09093751B8093FD
:10042000741B80E09DE0989FF0011124E652F34C8C
:10043000158214828F5F8A30B0F38093731B089506
:10044000CF932091741B3091751B2F5F3F4F211567
:100450004DE7340710F020E030E1522F432FE4E461
:10046000FCE3C0E0C43059F0A18DAA2329F0A48197
:10047000B581A417B50749F3CF5FB096F3CF30939A
:10048000751B2093741B1092731B20E0E0E0F0E0DA
:100490002430E8F430E2239FD0011124AC5BB34C4C
:1004A00059963C915997311104C02093731BFD015B
:1004B00010C0373041F4309739F05A964C915A9722
:1004C000328D341708F0DF012F5FFD01E1CF20935B
:1004D000731B309799F122E0218F2091761B24879E
:1004E0002091771B25872091781B26872091791BE7
:1004F000278728ED34E0338B228B358B248B21E04A
:1005000030E0318B208B138E228F23E0208F168AD0
:1005100020E1278B2091741B3091751B32272327F4
:1005200032273583248377836683DC014D915D9187
:100530006D917C914083518362837383CF01CF910E
:100540000895CF93DF932091741B3091751B2F5F1B
:100550003F4F21154DE7340710F020E030E1522FD6
:10056000432FEEEDFCE3C0E0CA3041F0A081B18141
:10057000CF5F3D96A417B507B9F7E9CF3093751B48
:100580002093741B40E05DE04A30A0F4A1E0A40F8A
:10059000549FF0011124E652F34C24813581232B22
:1005A00039F44093731B309741F480E090E023C00E
:1005B0004A2FEACF4093731BF8CF2091741B3091E0
:1005C000751B32272327322735832483778366835D
:1005D000009729F4108211821282138209C0EC0163
:1005E00088819981AA81BB8180839183A283B3830F
:1005F00080E48087CF01DF91CF91089540E04430BF
:10060000A0F4E42FF0E051E0540FEE0FFF1FEC5385
:10061000F34C208131812817390729F44093731B4B
:10062000118210820895452FEACF4093731B0895DD
:1006300040E0443098F4E42FF0E051E0540FEE0F26
:10064000FF1FEC53F34C20813181232B29F440937D
:10065000731B918380830895452FEBCF4093731BC9
:100660000895AF92BF92CF92DF92EF92FF920F93D5
:100670001F93CF93DF93C091423CD091433C843091
:1006800009F4DCC125E637E33093413C2093403C3C
:100690003093383720933737833059F4898D8F70F2
:1006A000833009F06BC088899989892B09F0DFC6EE
:1006B0007FC0823009F080C08091791B8F5F80936A
:1006C000791B811113C08091781B8F5F8093781BF9
:1006D00081110CC08091771B8F5F8093771B8111F4
:1006E00005C08091761B8F5F8093761B1092363702
:1006F000109235371092D93C1092D83C298D822F18
:100700008D7F853041F48A8D8F5F8A8F843109F027
:10071000AEC6198EACC6222309F4A9C68889998968
:10072000892B09F441C08A8D9FEF980F9A8F811110
:100730009EC68B8D883031F09FEF920F923048F437
:10074000853039F4198E80E880933D3C0E94B27D5B
:1007500047C5853038F493E0082E01C0990F0A94FC
:10076000EAF701C090E39A8F8F5F8B8F822F8F7093
:100770008330A1F048F4813009F44FC3823009F08E
:1007800076C610925E374CC3863009F4C8C48830F0
:1007900009F4C5C4843009F06AC6C1C484E08093FA
:1007A0003D3C0E94B27D4EC52F70233009F05FC6DC
:1007B00088E080933D3C09C5853019F5E0913E3CC9
:1007C000F0913F3C84819581892B09F450C61092A9
:1007D000433C1092423C89E597E39093413C8093DF
:1007E000403C90933837809337371092D93C109221
:1007F000D83C109236371092353788E080933D3CD4
:100800001BC180913D37853409F031C600913F37D7
:1008100010E0102F002780914037080F111D8091A4
:100820003537909136378017910708F420C610931A
:10083000363700933537809143378F7309F017C6E9
:1008400080914437811113C68091D43C9091D53C5E
:10085000C0916D03D0916E038C179D0759F44091A0
:10086000D63C5091D73C20916F03309170034217D2
:100870005307A1F020914D3730914E372817390793
:1008800009F0F5C520914F37309150378091D63C13
:100890009091D73C2817390709F0E9C50E94DD81FE
:1008A000019609F0E4C580914637863009F429C1E4
:1008B0008131E9F1813009F0DAC580915137883012
:1008C00009F0D5C510925137809153379091543724
:1008D000873F3FEF930710F0099601C00896909369
:1008E0005437809353378091493790914A37A0917C
:1008F0004B37B0914C3780934D3790934E37A09340
:100900004F37B09350378091D43C9091D53CA09113
:10091000D63CB091D73C8093493790934A37A09307
:100920004B37B0934C3780E4809345377DC50C51ED
:100930001109109336370093353789E597E3909383
:10094000413C8093403C8091573790915837892B98
:1009500029F00E94F181019609F089C52091533751
:10096000309154372115310509F481C58AED9CE396
:1009700090933F3C80933E3CA0905137B0905237CB
:1009800040916F03509170036091710370917203F5
:10099000A0917303B09174030091493710914A37C5
:1009A000E0904B37F0904C37E0913E3CF0913F3C6B
:1009B0008DE3EC35F80708F05AC5848195810097DE
:1009C00021F12817390709F586819781009719F0D9
:1009D000A816B906D1F4808191818C179D0729F45E
:1009E000C280D380C416D506B1F08617970729F4C4
:1009F000C280D380CA16DB0671F00817190729F4E4
:100A000082819381E816F90631F03D96F0933F3CE0
:100A1000E0933E3CC9CF1092433C1092423C82E0AE
:100A200080933D3C89E597E390933837809337373F
:100A30001092D93C1092D83C0E94B27D8091D83C53
:100A40009091D93C009709F412C59C01245E3F4F58
:100A5000309336372093353730933F3720934037E4
:100A6000E0913E3CF0913F3C20852093453721E1C9
:100A700020934637089698278927982790935637CA
:100A8000809355371092583710925737848195814B
:100A90009093523780935137868197819093543742
:100AA000809353378091D43C9091D53CA091D63C13
:100AB000B091D73C8093493790934A37A0934B37F6
:100AC000B0934C3780819181A281B38180934D375F
:100AD00090934E37A0934F37B093503785E697E306
:100AE0009093413C8093403C0E94F1818095909589
:100AF000009711F48FEF9FEF9093583780935737FB
:100B000093C40E94EE81019609F0B1C480915337DD
:100B100090915437009709F4AAC42091513730912D
:100B200052372115310509F4A2C44091493750913B
:100B30004A3760914B3770914C37EDE5FCE3C4E4E4
:100B4000DCE3F080FF20A9F0AC81BD818A179B0710
:100B500081F4AE81BF812A173B0759F4A881B9817E
:100B60004A175B0731F4AA81BB816A177B0709F436
:100B70006FC1A096B096ACE3C43CDA0711F72091A0
:100B80005E372F732230D9F49093711B8093701BC2
:100B900040E0443090F4E42FF0E0EE0FFF1FEC5300
:100BA000F34C208131814F5F8217930791F71092A8
:100BB000731B20E0C0E0D0E07EC04093731B8091A7
:100BC0005E3782FD54C484E180935E3788E290E012
:100BD000909336378093353780E580935D378091E9
:100BE000583790915C3790935837309157379091A0
:100BF0005B379093573730935B37209156379091FE
:100C00005A379093563720935A379091553790938F
:100C1000731B4091593740935537909359378F5FE5
:100C200080935C3781110FC081E0830F80935B3725
:100C3000811109C081E0820F80935A37811103C06E
:100C40009F5F90935937809151379091523790938D
:100C5000711B8093701B2091533730915437309320
:100C60005237209351379093543780935337809164
:100C7000493790914A37A0914B37B0914C378093C8
:100C80004D3790934E37A0934F37B09350378091A4
:100C9000D43C9091D53CA091D63CB091D73C809368
:100CA000493790934A37A0934B37B0934C37A1C341
:100CB000373089F02F5F2430C0F430E2239FC00129
:100CC0001124FC01EC5BF34C318D3111F1CF2093F9
:100CD000731BEF010CC0209721F0428D3A8D341721
:100CE00048F7EC01CC5BD34CE5CF2093731B2097E6
:100CF00009F4BDC3D093433CC093423C83E08A8F48
:100D0000888F1E8A84E08F8B1B8E80915337909141
:100D100054379D838C8380915137909152379F83B4
:100D20008E838091493790914A37A0914B37B0918B
:100D30004C3788839983AA83BB8381E0898F809114
:100D4000761B8C878091771B8D878091781B8E878F
:100D50008091791B8F8781E090E0998B888B8091BF
:100D600058378B87809157378A8780915637898784
:100D700080915537888781E090E00E949B8A80911E
:100D80005D37282F207F30E0213531050CF445C038
:100D900082958F7090E00597880F991F880F991F93
:100DA0003091721B20E0E22FF0E0E817F9078CF594
:100DB000E35CF84C30A5311105C02093731B1092F1
:100DC000721B2BC0313011F42F5FEDCF3230E1F4C4
:100DD00041A54430C9F42093731B3093721B82A544
:100DE00090E0982F882723A5822B9093711B8093E6
:100DF000701B893DA4E09A0710F088ED94E09B8B6E
:100E00008A8B9D8B8C8B09C041A5442311F0240F44
:100E1000CACF2093731B3093721B80E180935E379F
:100E200080915E37826080935E3782E08093653781
:100E300084E0809366378093673788ED80936837C6
:100E40008CE290E0909336378093353780E67EC20F
:100E5000D093433CC093423C10923D3C90915E370E
:100E600092FF03C0198E80E21AC280915D3782958D
:100E70008F70880F880F8093731B081B1109045112
:100E8000110910933637009335378F2D8F708230CC
:100E900029F4892F8F73823139F41FC0813021F4F6
:100EA000892F8F738230C9F0012B19F4892F837039
:100EB000A1F020915537888528133EC220915637DE
:100EC0008985281339C2209157378A85281334C25F
:100ED000209158378B8528132FC294FF4AC0688908
:100EE00079896115710509F444C0CE010C960E9400
:100EF0009C81309159378091393738133AC020910D
:100F00005A3780913A37281334C090915B378091DB
:100F10003B3798132EC080915C3740913C37841347
:100F200028C03C872D879E878F878B8D81111AC0A3
:100F30002E89888D9A8D891B922F969596959695D8
:100F4000891B280F2E8B87FD81959F89392F369518
:100F50003695931B980F9F8B822F86958695869545
:100F6000890F888F81E080933D3C888D8A8F198A14
:100F7000188A498D842F8F7090E0FC013197E830FA
:100F8000F10508F074C2E057FF4F0C94EA9280918B
:100F90003D3C80FF14C083E0898F80E480933D3C1A
:100FA000198A188A8091353790913637009709F45D
:100FB00008C122E420933D3C0E949B8A02C180919B
:100FC0005E378F73823009F052C227CF80913D3C4B
:100FD00080FF70C080915E378F73823109F06AC0E4
:100FE00080915D37282F207F30E0213531050CF4CA
:100FF00045C082958F7090E00597880F991F880FE4
:10100000991F3091721B20E0E22FF0E0E817F907FA
:101010008CF5E35CF84C30A5311105C02093731BAF
:101020001092721B2BC0313011F42F5FEDCF323094
:10103000E1F441A54430C9F42093731B3093721B33
:1010400082A590E0982F882723A5822B9093711B6F
:101050008093701B893D24E0920710F088ED94E0A6
:101060009B8B8A8B9D8B8C8B09C041A5442311F0EF
:10107000240FCACF2093731B3093721B83E0898F98
:101080008091553788878091563789878091573767
:101090008A87809158378B8781E090E00E949B8AF5
:1010A00082E480933D3C198A188A10923637109258
:1010B000353787C080E280933D3C0E94B27DE0914D
:1010C000423CF091433C118E7ACD80915E3780FF97
:1010D00028C044FD26C088899989892B09F0C7C199
:1010E000809135379091363701960E949B8A2091E6
:1010F0003D3C822F806180933D3C809135379091BB
:101100003637892B19F0226120933D3C0E94B27D35
:1011100081E090E0998B888B88E0898F1B8E81E13C
:101120000CC185FF1CC08091633790E0982F882701
:1011300020916437822B2091403C3091413C280F14
:10114000391F3093413C2093403C209135373091FA
:101150003637281B390B309336372093353780913B
:10116000353790913637009749F044FD07C02091FC
:101170003D3C226020933D3C0E949B8A80915F37DA
:1011800090E0982F882720916037820F911D9093CF
:10119000711B8093701B2C893D892817390710F02B
:1011A000892B21F43093711B2093701B8091701B4D
:1011B0009091711B9B8B8A8B80913D3C837009F4CD
:1011C00056C11092D93C1092D83C0E94B27D8091B9
:1011D0003D3C85FF07C01092D93C1092D83C198E37
:1011E00084E1ABC084FF0AC01092D93C1092D83C75
:1011F00081E090E0998B888B84E08FCF2091D83C60
:101200003091D93C21153105E1F080FF02C0198AE7
:10121000188A88899989009781F48A899B8982171D
:10122000930720F49093D93C8093D83C8091D83C8C
:101230009091D93C998B888B04C09093D93C809332
:10124000D83C1B8E80913737909138379093413C32
:101250008093403C8091D83C9091D93C892B59F0A7
:1012600088899989009739F08896909336378093CA
:10127000353788E10BC080913D3C81FFF8C088E2A2
:1012800090E0909336378093353780E180935E37D6
:101290005CC080913D3C80FFEAC0198E80E1809364
:1012A0003D3C0E94B27DE3C0809135379091363746
:1012B000009711F00E949B8A90915E3780913D3C8F
:1012C00090FF0BC080FF06C087E0898F1A8E198AB5
:1012D000188A19C086E0898F16C080FF1EC085E07D
:1012E000898F198A188AC3C0809135379091363713
:1012F000009711F00E949B8A80915E3780FF0DC09D
:1013000087E0898F1A8E81E090E00E949B8A80E1BD
:1013100080933D3C0E94B27D0FC080913537909103
:101320003637892B49F4A3C080913D3C80FF9FC094
:1013300087E0898F1A8E9BC080E180935E3788E2B8
:1013400090E0909336378093353780E580935D3712
:10135000888580935937898580935A378A85809309
:101360005B378B8580935C378C85809355378D8573
:10137000809356378E85809357378F858093583763
:1013800086E0809346378C819D819093523780937D
:1013900051378E819F81909354378093533780913A
:1013A000D43C9091D53CA091D63CB091D73C809351
:1013B000493790934A37A0934B37B0934C37888185
:1013C0009981AA81BB8180934D3790934E37A0932A
:1013D0004F37B0935037898D84FF05C01092603726
:1013E00010925F3706C084E080935F3788ED80936A
:1013F000603780E480934537809135379091363758
:1014000090933F3780934037109264371092633740
:1014100010926237109261370E94EE81809590950C
:10142000909362378093613785E480933D371092C3
:101430003E37109244371092433780917A1B909137
:101440007B1B019690937B1B80937A1B9093413773
:101450008093423710924837109247370E94DD81BF
:1014600080959095909348378093473704C01092A9
:1014700036371092353710923D3CDF91CF911F9156
:101480000F91FF90EF90DF90CF90BF90AF900895B5
:1014900098278927982708950E94F0920895FC01C3
:1014A00080913737909138372DE33CE3281B390B77
:1014B000AB01261737070CF4A9011416150654F4CE
:1014C0005093D93C4093D83CE817F90719F0BF0175
:1014D0000C94AB98089580E88093610010926100AD
:1014E0000E9425690E94855A0E94036D8091E43410
:1014F0009091E534009729F001979093E53480931B
:10150000E434C090E634D090E734E090E834F090D2
:10151000E9340E94BF6BC616D706E806F90611F338
:101520000E94BF6B6093E6347093E7348093E83495
:101530009093E934D7CF2091423C3091433CBC0199
:10154000C90108960E949C81E091423CF091433C85
:1015500080913937808780913A37818780913B37F6
:10156000828780913C37838708952F923F924F92D4
:101570005F926F927F928F929F92AF92BF92CF9223
:10158000DF92EF92FF920F931F93CF93DF93CDB72C
:10159000DEB763970FB6F894DEBF0FBECDBF7C01F8
:1015A0001B016A01FC0117821682838181FF66C3D9
:1015B000BE016F5F7F4F4B01F7019381F10193FDF6
:1015C000859193FF81911F01882309F453C38532CC
:1015D00039F493FD859193FF81911F01853239F490
:1015E000B70190E00E942E9956016501E5CF10E009
:1015F000512C20E02032A0F48B3269F030F480329C
:1016000059F0833269F420612CC08D3239F0803377
:1016100039F4216026C02260246023C0286021C0E4
:1016200027FD27C030ED380F3A3078F426FF06C08A
:10163000FAE01F9F300D1124132F13C06AE0569E4D
:10164000300D1124532E20620CC08E3221F426FD61
:1016500011C3206406C08C3611F4206802C088369D
:1016600041F4F10193FD859193FF81911F01811157
:10167000C1CF9BEB980F933018F42061805E06C0B9
:101680009BE9980F933008F0AAC12F7E26FF16E041
:101690002F73722E853621F4F22FF0647F2E08C04E
:1016A000863621F4622F6068762E02C01111115027
:1016B00077FE07C01C3348F444244394410E27E0CE
:1016C0000BC0183030F4212F06C027E04CE3442E25
:1016D00003C027E017E0412C560174E0A70EB11CAF
:1016E000F6016081718182819381042DA4010E94A1
:1016F000B3976C01098100FF02C003FF06C071FCB3
:1017000007C072FC08C0612C08C03DE2632E05C012
:101710002BE2622E02C090E2692E802F8C7099F12C
:10172000662011F084E001C083E0851510F0512C93
:101730000BC0581A73FC08C0B70180E290E00E9409
:101740002E995A94C9F7F3CF662029F0B701862D58
:1017500090E00E942E9903FD03C006ED12E102C045
:1017600002ED12E1F72DF0717F2EF80184918823AC
:1017700009F476C271108052B70190E00E942E9950
:101780000F5F1F4FF2CF77FE0FC04C0C04FF04C059
:101790008A81813309F44A94141474F5F8E0F4153D
:1017A00078F588E0482E2CC076FC2AC0812F90E086
:1017B0008C159D059CF06CEFC6166FEFD60674F085
:1017C000772D7068772E0AC0E2E0F0E0EC0FFD1F85
:1017D000E10FF11D8081803319F411501111F4CF04
:1017E00077FE0EC044244394410E812F90E0C8162A
:1017F000D9062CF41C1904C04424439401C010E001
:1018000077FE07C01C141D043CF496012F5F3F4F68
:1018100005C025E030E002C021E030E0662011F094
:101820002F5F3F4F112331F0412F50E04F5F5F4F4B
:10183000240F351F452D50E02417350714F4521A94
:1018400001C0512C872D897049F4552039F0B7011A
:1018500080E290E00E942E995A94F7CF662029F0FA
:10186000B701862D90E00E942E9973FC09C0552087
:1018700039F0B70180E390E00E942E995A94F7CF97
:1018800077FE5FC09C2D8D2DD7FE02C090E080E0DA
:10189000692E782E40E050E0C601841991099D8799
:1018A0008C87960126193709280D391D812F90E064
:1018B000EE27FF27E81BF90BFF87EE87FFEF6F1678
:1018C0007F0669F4B7018EE290E02B8B3A8B488B50
:1018D000598B0E942E99598948893A892B89C614B7
:1018E000D70454F06C857D85661577052CF4F901D5
:1018F000E40FF51F818101C080E371E0671A710870
:101900004F5F5F4FEE85FF856E167F066CF0B70167
:1019100090E02B8B3A8B488B598B0E942E992B8908
:101920003A8948895989CACF6C147D0439F49A815F
:10193000963318F4953311F404FF81E3B70190E076
:101940004BC08A81813309F00F7EB70190E00E947D
:101950002E99111105C074FE18C085E490E017C0DF
:10196000B7018EE290E00E942E9982E06624639493
:10197000680EF401E80FF11D8081B70190E00E942C
:101980002E99115041F3862DF1CF85E690E0B701F5
:101990000E942E99D7FC05C0C114D10439F404FF6C
:1019A00005C0D194C194D1088DE201C08BE2B7018A
:1019B00090E00E942E9980E36AE0C616D1042CF0D4
:1019C0008F5FFAE0CF1AD108F7CFB70190E00E94FD
:1019D0002E99B701C601C0960E942E9941C1833647
:1019E00031F0833779F0833509F058C021C05601B2
:1019F00072E0A70EB11CF6018081898301E010E03E
:101A0000640114C05601F2E0AF0EB11CF601C080B3
:101A1000D18026FF03C0612F70E002C06FEF7FEF1F
:101A2000C6012B8B0E94DA988C012B892F7715C069
:101A30005601F2E0AF0EB11CF601C080D18026FF46
:101A400003C0612F70E002C06FEF7FEFC6012B8BE8
:101A50000E949C988C012B892068722E23FD1AC04D
:101A6000852D90E008171907A8F4B70180E290E0EF
:101A70000E942E995A94F4CFF60177FC859177FE57
:101A800081916F01B70190E00E942E9951105A94F4
:101A9000015011090115110579F7E2C0843611F0E2
:101AA000893651F5560127FF09C0F4E0AF0EB11C8D
:101AB000F60160817181828193810AC0F2E0AF0EEC
:101AC000B11CF60160817181882777FD8095982F80
:101AD000022F0F7697FF08C09095809570956195BD
:101AE0007F4F8F4F9F4F00682AE030E0A4010E9493
:101AF000689AC82EC8183EC0022F853721F40F7E81
:101B00002AE030E01DC0097F8F3691F018F4883547
:101B100059F0B0C0803719F0883711F0ABC00061C0
:101B200004FF09C0046007C024FF08C0066006C0A7
:101B300028E030E005C020E130E002C020E132E0E2
:101B4000560107FF09C0F4E0AF0EB11CF601608139
:101B500071818281938108C0F2E0AF0EB11CF60161
:101B60006081718180E090E0A4010E94689AC82E93
:101B7000C8180F7706FF0BC0202F2E7FC11650F418
:101B800004FF0AC002FD08C0202F2E7E05C0DC2CF9
:101B9000202F03C0DC2C01C0D12E24FF0DC0FE017C
:101BA000EC0DF11D8081803311F4297E09C022FFE4
:101BB00006C0D394D39404C0822F867809F0D394BE
:101BC00023FD13C020FF06C01C2DD51418F4150DDD
:101BD0001D19D52CD51468F4B70180E290E02B8B49
:101BE0000E942E99D3942B89F5CFD51410F45D184B
:101BF00001C0512C24FF12C0B70180E390E02B8B71
:101C00000E942E992B8922FF17C021FF03C088E56F
